:020000040800F2
:10800000E85100200DF10108818D0008838D0008E2
:10801000878D00088B8D00088F8D00080000000000
:10802000000000000000000000000000938D000828
:10803000958D000800000000978D0008998D0008BC
:1080400027F1010827F1010827F1010827F10108AC
:1080500027F1010827F1010827F101081597000809
:1080600027F1010827F1010827F1010827F101088C
:1080700027F1010827F1010827F1010827F101087C
:1080800027F1010827F1010827F1010827F101086C
:1080900027F1010827F1010827F1010817970008C7
:1080A00027F1010827F1010827F1010827F101084C
:1080B00027F1010827F1010827F1010827F101083C
:1080C00027F1010827F1010827F1010827F101082C
:1080D00027F101083B9900089D990008D59A0008EE
:1080E0003798000827F1010827F10108DFF80CD0C4
:1080F00021F060FC0048004701810008E8510020A1
:1081000000F07CFB00F014FC1CF00CFA2948C0784D
:1081100008B91CF0DBFC2748C07820B92648006865
:108120000078592801D017F045FE41E013F0E6FD34
:1081300004F076FC214890F82D00072801D004F0C7
:108140002EFE09F0B0FA04F0C2FD0AF0D3FD11F0E2
:1081500000FE12F082FA01F07DFE04F08EFB13F0B7
:108160004DFE13F00EFF14F050F909F0BAFD13F0B4
:108170009BF91048C07838B90F4800680078592832
:1081800002D11CF0A1F907E00C4890F82D00072857
:1081900002D101200A49C87713F09FF913F046FA7B
:1081A00004F065FC05F026FA04F0E2FC04F0A2FD00
:1081B000BCE70000FE0400202C0200205804002030
:1081C000A003002008B50121082014F08DFE4FF413
:1081D0008040ADF8000010208DF8030003208DF8DA
:1081E00002006946FD4814F0C3FB08BD08B5012133
:1081F000082014F079FE4020ADF8000010208DF822
:10820000030003208DF802006946F44814F0B0FB27
:108210004021F24814F059FC0121082014F064FEBA
:108220004FF40060ADF8000010208DF8030003202B
:108230008DF802006946EA4814F09AFB08BD08B5BB
:108240000121082014F050FE4FF48050ADF80000DA
:1082500010208DF8030003208DF802006946DF48E6
:1082600014F086FB4FF48051DC4814F030FC08BD5C
:108270001FB50121492014F037FE17208DF80000AA
:1082800001208DF801008DF802008DF8030068468A
:1082900014F017FA28208DF8000001208DF8010055
:1082A0008DF802008DF80300684614F00AFA4FF4C6
:1082B0007F40ADF80C0003208DF80E0048208DF8AB
:1082C0000F0003A9C74814F053FB4FF40040ADF86A
:1082D0000C0003208DF80E0048208DF80F0003A934
:1082E000BE4814F045FB0821042014F057FC4FF45D
:1082F0008070019000208DF808000C208DF8090096
:1083000001208DF80A0001A814F052FA0921042076
:1083100014F044FC4FF40070019000208DF8080028
:108320000C208DF8090001208DF80A0001A814F036
:108330003FFA0A21042014F031FC4FF480600190D0
:1083400000208DF808000C208DF8090001208DF820
:108350000A0001A814F02CFA0B21042014F01EFCD2
:108360004FF40060019000208DF808000C208DF87B
:10837000090001208DF80A0001A814F019FA0C2157
:10838000042014F00BFC4FF48050019000208DF875
:1083900008000C208DF8090001208DF80A0001A8C2
:1083A00014F006FA0D21042014F0F8FB4FF40050ED
:1083B000019000208DF808000C208DF809000120A4
:1083C0008DF80A0001A814F0F3F90E21042014F02E
:1083D000E5FB4FF48040019000208DF808000C2050
:1083E0008DF8090001208DF80A0001A814F0E0F9C9
:1083F0000F21042014F0D2FB4FF400400190002024
:108400008DF808000C208DF8090001208DF80A0075
:1084100001A814F0CDF91FBD08B54FF40040ADF828
:10842000000004208DF8030069466E4814F0A0FA9D
:1084300008BD08B50121082014F056FD4FF4005086
:10844000ADF8000010208DF8030003208DF8020025
:108450006946624814F08CFA08BD1FB50121052059
:1084600014F042FD17208DF8000000208DF8010067
:1084700001208DF802008DF80300684614F021F900
:108480004020ADF80C0003208DF80E0004208DF87C
:108490000F0003A9524814F06BFA0220ADF80C004B
:1084A00003208DF80E0010208DF80F0003A94C4812
:1084B00014F05EFA0621002014F070FB40200190B9
:1084C00000208DF808000C208DF8090001208DF89F
:1084D0000A0001A814F06CF91FBD704710B50446DE
:1084E000012C04D181033D4814F0EFFA04E04FF46D
:1084F00080413A4814F0EBFA10BD10B50446012C47
:1085000008D14021354814F0E2FA0221344814F031
:10851000DCFA07E04021314814F0D7FA0221304854
:1085200014F0D5FA10BD08B50121042014F0DCFCCC
:108530000121202014F0D8FC2020ADF800001020EC
:108540008DF8030003208DF802006946264814F0D8
:108550000FFA2021244814F0BAFA4FF48070ADF8D5
:10856000000010208DF8030003208DF802006946FA
:108570001B4814F0FDF94FF48071194814F0A5FA66
:1085800008BD08B50121082014F0AEFC40F202300D
:10859000ADF8000010208DF8030003208DF80200D4
:1085A00069460E4814F0E4F940F202210B4814F039
:1085B0008EFA08BD08B50121102014F095FC0320A7
:1085C000ADF8000010208DF8030003208DF80200A4
:1085D0006946064814F0CCF908BD0000000C0140C3
:1085E0000008014000180140001401400010014043
:1085F00010B50446012C04D1C102B14814F065FA4B
:1086000004E04FF40061AE4814F061FA10BD10B5FB
:108610000446012C03D10103AA4814F058FA10BDF6
:1086200010B50446012C04D14103A64814F04FFABA
:1086300004E04FF40051A34814F047FA10BD08B508
:108640000121042014F050FC4FF40040ADF800006C
:1086500004208DF803008002ADF8000010208DF892
:10866000030003208DF802006946954814F080F954
:108670004FF48051924814F028FA782000F036F92F
:10868000032004F056FA052000F030F908BD08B5C3
:108690000121042014F028FC4FF40040ADF8000044
:1086A00004208DF803008002ADF8000004208DF84E
:1086B00003006946824814F05BF908BD2DE9F041DA
:1086C000044625464FF480517D4814F000FA0520F9
:1086D00000F00CF905F00107002625E0012F0ED16E
:1086E0003903774814F0F1F9062016F021FD39031B
:1086F000734814F0ECF9022016F01AFD0FE04FF465
:1087000080516F4814F0E1F9022016F011FD4FF48A
:1087100080516B4814F0DBF9062016F009FD6D104E
:1087200005F00107701CC6B2082ED7DB4FF480514C
:10873000634814F0CAF9BDE8F08110B562480078CA
:108740000B280AD0614890F8360030B9FFF777FF60
:1087500001205E4981F836000EE05B4800780B2866
:108760000AD15A4890F83600012805D1002057490F
:1087700081F83600FFF78BFF10BD0EB5002054497D
:10878000096800915249091D096801915049083151
:10879000096802910099C9B2009AC2F307221144F4
:1087A000009AC2F307421144009A01EB1261019A48
:1087B000D2B21144019AC2F307228818454AD071F7
:1087C000010A91710199090C51710199090E1171F8
:1087D0000299D1700299090A91700299090C51709D
:1087E0000299090E1170DDE900121144029A114438
:1087F000394A11800121394A11700EBD70B513F04C
:10880000D9FE374800684FF47A72B0FBF2F1B1F14B
:10881000807F00D31DE021F07F40401E4FF0E0221A
:10882000506150170F22002807DA13071D0E2D4B39
:1088300000F00F04241F1D5503E013071C0E2A4BE4
:108840001C5400BF00204FF0E0229061072010610F
:1088500000BFFFF7EEFDFFF700FEFFF7B3FCFFF7E9
:10886000C5FCFFF7ECFCFFF703FDFFF78AFEFFF7FF
:108870005AFE4FF4E13001F054FF4FF4E13001F0C3
:10888000A8FF01F0C9FB01F042FD01F0FFFB13F06E
:108890006FFA0020FFF7C4FE0020FFF71FFE40F232
:1088A0001F31632016F05BFC0120FFF726FE00203D
:1088B000FFF79EFEFFF761FFFFF77CFE70BD000033
:1088C00000080140000C01404F000020A0030020E0
:1088D000E8F7FF1F00000020740000201A010020AC
:1088E0007801002018ED00E000E400E0FD49086098
:1088F00000BFFC4909680029FBD1704708B5FA4A56
:108900000421684603F07AF80020F84988639DF84E
:10891000000000069DF8011000EB01409DF80210D8
:1089200000EB01209DF803100844F049886308BD5E
:1089300008B54021ED4820F0AAFA3C21EC4820F08F
:10894000A6FA8021EB4820F0A2FA8021EA4820F024
:108950009EFA1C21E94820F09AFAFF20E8490871A4
:108960000020887148710870FF2088700020C8704E
:108970004870C871E349087048708870C870087101
:1089800048718871C871D74981F85600962081F8DE
:10899000500081F8510081F8570081F8520081F8A9
:1089A000530081F8540081F855000220D649087020
:1089B0000020487088700220087100204871C8703B
:1089C0008871C871087248728872C8720873012071
:1089D000487300208873C873087448740875487514
:1089E00088750120C8750020087648768876087753
:1089F0004877C87781F8200081F8210081F82200AB
:108A000081F82400022081F82500012081F8260049
:108A100081F8270081F82800002081F8290081F8DA
:108A20002A0081F82B00022081F82C00002081F818
:108A30002D00022081F82F0081F83000002081F8FD
:108A4000310081F8330081F8340081F8350081F875
:108A50003600C87681F8370081F8390081F838008F
:108A600081F82300012081F83A0000209D49086028
:108A70004FF4FA7048600020C86040F6B8300882B1
:108A80004EF6602088604FF47A7088821420488205
:108A900047F23050088341F2883088844FF47A706E
:108AA000C8849A48086242F2D0000885088698482F
:108AB0000068C86264204886964848634FF47A701C
:108AC000A1F84000400008874010488347F230502A
:108AD00088834010A1F8480042F21070A1F84200CB
:108AE000A1F84A00A1F84C0043F69820A1F84E00E6
:108AF00086488865884808664FF47A70A1F8640053
:108B00000320814981F832004FF4967075498887B7
:108B100043F6982088668000C86600207F49087068
:108B20007F49887088714871C872C87008718873ED
:108B30007C4948730B207C49087000207B490870F1
:108B400048708870C870087148718871C8710120B8
:108B50007749087077490870654908707649087048
:108B6000764908700320764908700020754908701E
:108B7000754908700C205D4981F82D00092081F8A5
:108B80002E00002071490870222071490870714937
:108B900008701D207049087040F2E5706F49088028
:108BA00001208870C870002048718871C871FF204A
:108BB0004E49888201F07DFF4EF67D7001F0B0FFD6
:108BC00012F044FF664A02214A4802F017FF494862
:108BD00000780A2802D102F035FF13E003F035FCDB
:108BE00002F030FF00208DF800008DF801008DF8B4
:108BF00002008DF803003C4A0421684602F0D2FED0
:108C000019F0B6FA02F0D0FA564800880A280EDBAE
:108C10005548008828B953480078401E3749C8761F
:108C20000AE051480078401E3449C87604E04D48B7
:108C30000078401E3149C87602F00BFBFFF75EFE5C
:108C400019F086FA494800680068401C47490968DD
:108C500008604748C078012803D14E20454909687B
:108C6000087019F07DFA08BD3B480078082838D113
:108C70001F48008D00EB80004FF6FF7101EA4000B5
:108C80003D4948801A48408D00EB80004FF6FF7147
:108C900001EA4000384988801548808DC880144812
:108CA000408E08811248C08D48811148008E88810D
:108CB0000F48408D00EB80004FF6FF7101EA400045
:108CC0000A4948800A48008D00EB80004FF6FF718A
:108CD00001EA40000549088428480088888400206B
:108CE000C8807047E003002000A006085804002058
:108CF000A8040020B0110020B00900209409002031
:108D00000800002018000020A003002080EE36009C
:108D1000C400002020BF0200E0930400E000002017
:108D2000BF120020B01200204F000020F8000020E9
:108D30003800002098040020480000204A0000204D
:108D400049000020E2000020E30000204E00002047
:108D5000EC000020ED000020C00000202A000020D0
:108D60007E4006089C0000209E000020300200206B
:108D7000FE0400202C020020E4040020D600002085
:108D8000704700BFFEE700BFFEE700BFFEE700BF81
:108D9000FEE770477047704710B5FA48007850B941
:108DA0004FF40051F84813F076FE20B94FF400510B
:108DB000F54813F08AFEF548006820B1F3480068D2
:108DC000401EF2490860F2480078082823D1F14893
:108DD0000078022811D1F04890F8330068B9EB48C8
:108DE000406828B1E9484068401EE849486012E000
:108DF0000120E94981F833000DE04FF48041E74854
:108E000013F049FE38B14FF4FA70E0494860002091
:108E1000E14981F83300E24801880088401EE04AB9
:108E20001080022906DA0120DE4908704FF4FA604A
:108E300011460880DC4801880088401CDA4A10800E
:108E400041F28830814205DD002011460880012072
:108E5000D6490870D648007801280FD1D548018836
:108E60000088401CD34A108041F28830814205DDE1
:108E70000020114608800120CF490870CF48407A71
:108E800004280ED1CE48006828B1CD480068401EA5
:108E9000CB49086005E0CB48C94908600120CA49B0
:108EA0000870C3480078012807D10102C74813F0B1
:108EB000F2FD012801D1C6490870B74800780228A0
:108EC0000FD1B248008A28B1B048008A401EAF498D
:108ED000088206E00120B049087040F6B830AB497E
:108EE0000882BC480088002805DDBA480088401E7A
:108EF000B849088008E04FF47A70B649088001202C
:108F0000B5490870B5490870A048408E28B19F48FF
:108F1000408E401E9D49488616E04FF496709B494E
:108F200048869D48007D012807D100209A49087590
:108F30000121A64813F0CBFD06E0012096490875F3
:108F40000121A24813F0C1FD9048808A28B18F48C2
:108F5000808A401E8D49888206E001208E4908746F
:108F600047F23050894988828B4890F82E000228B9
:108F700014D19B4890F82D000B280FD08348C06D6A
:108F800028B18248C06D401E8049C86506E00120B6
:108F9000814981F82E0093487C49C8657E4890F845
:108FA0002100012804D07C4890F82100022814D127
:108FB0007648B0F8480038B17448B0F84800401E10
:108FC0007249A1F8480008E00020734981F82100A7
:108FD00043F698206D49A1F848006F48807B02282D
:108FE00010D16A48008E28B16848008E401E67493B
:108FF0000886A2E003206849887342F2D0006349E2
:1090000008869AE06448807B0128F2D16248407B60
:1090100002280FD15D48C06A28B15C48C06A401E72
:109020005A49C86206E00220564908706E48006836
:109030005649C8620221544813F02DFD60B16B48B7
:10904000008828B169480088401E6849088003E00C
:1090500002214D4813F03BFD4F4890F82E000628A2
:109060001ED14FF40071484813F015FDC0B160489F
:10907000008848B15E480088401E5D490880012094
:10908000454981F821000BE04FF400713E4813F090
:109090001EFD0220404981F82E00002081F82100A9
:1090A0003848007802280ED15248008828B151482B
:1090B0000088401E4F49088005E001204E49088085
:1090C000C8204C4908802F48007802280ED14B4810
:1090D000008828B149480088401E4849088005E0BA
:1090E00001204749088032204449088025480078FB
:1090F00078B94448008828B142480088401E414958
:10910000088006E00120404908804FF47A703D490C
:1091100008802148007B02280FD11C48008D28B10F
:109120001A48008D401E1949088506E003201A4997
:10913000087342F2D000154908851748407A022882
:109140000ED11248408A28B11048408A401E0F496B
:10915000488205E001201049487214200B494882DA
:109160000D4890F8290058B90848B0F84E0040B1B1
:109170000648B0F84E00401E0449A1F84E0050E0E9
:109180004FE043E028000020000C0140E0030020F5
:10919000C000002010000020A003002000180140A3
:1091A00062000020640000206800002066000020AB
:1091B000200100206A0000206C000020B012002076
:1091C00004010020009F240008010020001001403D
:1091D0007C0000205E000020600000206500002070
:1091E0005804002040771B00C4000020CE0000205F
:1091F000D000002052010020540100205E01002018
:109200005C01002070010020720100200120F7495C
:1092100081F82B0081F8290044F62060F449A1F878
:109220004E00F348806828B1F1488068401EF0493C
:1092300088602BE00120ED498870EE490870EE4807
:10924000407C20B944F62060E949886006E0EA489D
:10925000407C012802D1E948E5498860E84908884E
:109260000988491EE64B19801FF0F0FD1FF0E4FD50
:1092700044F6216190FBF1F201FB120000F6B830D8
:10928000E049086008460068DF490860DE48006879
:1092900028B1DD480068401EDB49086002E0DB4879
:1092A000D9490860D248806E28B1D148806E401EEE
:1092B000CF49886607E00120CC4981F83C0043F69D
:1092C0009820CB498866CA48C06E28B1C848C06E8D
:1092D000401EC749C8660CE00120C44981F83A0025
:1092E000C648C349C866C448407C10B944F62060EB
:1092F000C866BF48006F28B1BD48006F401EBC491A
:10930000086707E00120B94981F83B0041F2883045
:10931000B7490867BE480078F0B1B548408B28B11E
:10932000B348408B401EB249488315E0B9480078E5
:1093300001280ED0B748007805280AD0B548007833
:10934000062806D0B3480078022802D0B148007839
:1093500010B9FF20AE490870AF48407A04281FD1E9
:10936000A348B0F8400038B1A148B0F84000401E12
:109370009F49A1F8400013E09C48407F052803D195
:1093800001209A49487706E09848407F062802D194
:109390000020964948774FF47A709549A1F840002B
:1093A00008F0FCF99D48007801280FD19048006A28
:1093B00028B18F48006A401E8D49086206E08F4838
:1093C0008B4908620020894981F82600944800787A
:1093D000FF2820D14FF48041924813F05CFB98B9EC
:1093E000834890F8500038B1814890F85000401EF2
:1093F0007F4981F850000EE00220894908709620CC
:109400007B4981F8500006E00120854908709620CC
:10941000774981F8500082484078FF2820D14FF4E6
:109420000071804813F037FB98B9714890F85100EB
:1094300038B16F4890F85100401E6D4981F85100D5
:109440000EE00220764948709620694981F8510063
:1094500006E00120724948709620654981F8510064
:109460006F488079FF2820D14FF400516D4813F0E8
:1094700012FB98B95E4890F8520038B15C4890F8F9
:109480005200401E5A4981F852000EE00220644901
:1094900088719620564981F8520006E00120604903
:1094A00088719620524981F852005D480079FF2862
:1094B00020D14FF400415B4813F0EDFA98B94C48C5
:1094C00090F8560038B14A4890F85600401E484976
:1094D00081F856000EE00220514908719620444957
:1094E00081F8560006E001204D4908719620404958
:1094F00081F856004A48C079FF281FD1411C4948CD
:1095000013F0C9FA98B93A4890F8550038B138487C
:1095100090F85500401E364981F855000EE00220B3
:109520003F49C8719620324981F8550006E0012074
:109530003B49C87196202E4981F8550038488078FB
:10954000FF2826D14FF48051364813F0A4FAC0B951
:10955000274890F8530038B1254890F85300401E32
:10956000234981F853002BE02F488078401C2E4976
:10957000887002202A49887096201D4981F853007E
:109580001EE00120264988709620194981F8530071
:1095900016E026488078012812D1154890F853002B
:1095A00038B1134890F85300401E114981F8530018
:1095B00006E000201D49887096200D4981F853006F
:1095C0001748C078FF2845D14FF40061154813F0C3
:1095D00062FA68BB064890F8540050B3044890F80B
:1095E0005400401E024981F854004AE0A0030020C4
:1095F000E00300200F010020FE040020804F120035
:10960000740000207800002070000020C0D4010009
:109610004D0000204E000020B0120020DB00002092
:109620000800002000180140180000202000002041
:1096300008E0FFE70220FE49C8709620FD4981F846
:1096400054001EE00120FA49C8709620F94981F8BB
:10965000540016E0F848C078012812D1F54890F877
:10966000540038B1F34890F85400401EF14981F895
:10967000540006E00020F049C8709620ED4981F8BA
:109680005400EB484079FF2820D14FF48061EB482B
:1096900013F001FA98B9E74890F8570038B1E54857
:1096A00090F85700401EE34981F857000EE0022071
:1096B000DF4948719620DF4981F8570006E0012014
:1096C000DB4948719620DB4981F85700DC48C07DB2
:1096D00002281ED1D748808B28B1D648808B401EE7
:1096E000D449888315E0D7480078092807D0D548A1
:1096F00000780A2803D0D3480078082802D1002037
:10970000D04908700120CE49C87547F23050C94988
:10971000888310BD704710B5402013F0AFF80028C3
:1097200062D0C74890F82700012857D1C648007872
:10973000022853D1C248807B022823D1C348008B22
:10974000401CC24908830846008B012846DB0020E4
:1097500008834FF40051BE4813F0B7F90020BA490E
:1097600008700120B6498873BA4908704FF47A70BE
:10977000B94908800020B949088040F6B830AD49A1
:10978000C8822BE0AE48807B012827D1AF48008BF0
:10979000401CAE4908830846008B02281EDB0020CF
:1097A0000883084690F82D00062808D1A44890F8B0
:1097B0003500012803D10220A349087007E00020EA
:1097C000A14908704FF40051A14813F07EF942F20C
:1097D000D0009849088501209949C873402013F0AA
:1097E00049F8402013F05BF84FF4807013F046F80E
:1097F00068B18F48C07910B9FF208D49C8714FF406
:10980000807013F037F84FF4807013F048F84FF47D
:10981000007013F033F868B18548407810B9FF2024
:10982000834948704FF4007013F024F84FF400702F
:1098300013F035F810BD10B58348007850B94FF4D7
:109840000051834813F027F920B94FF400518048A4
:1098500013F03BF94FF4806013F010F868B17448CE
:10986000407910B9FF20724948714FF4806013F0BD
:1098700001F84FF4806013F012F84FF4006012F01A
:10988000FDFF68B16A48C07810B9FF206849C87008
:109890004FF4006012F0EEFF4FF4006012F0FFFF93
:1098A0004FF4805012F0EAFF68B16148807810B937
:1098B000FF205F4988704FF4805012F0DBFF4FF4B7
:1098C000805012F0ECFF4FF4005012F0D7FF68B157
:1098D0005748807910B9FF20554988714FF40050DE
:1098E00012F0C8FF4FF4005012F0D9FF4FF480403F
:1098F00012F0C4FF68B14E48007810B9FF204C49FF
:1099000008704FF4804012F0B5FF4FF4804012F021
:10991000C6FF4FF4004012F0B1FF68B1444800792F
:1099200010B9FF20424908714FF4004012F0A2FF25
:109930004FF4004012F0B3FF10BD10B540F22551B6
:10994000474813F0F5FC012827D1454813F070FC77
:109950004449454A1278885408460078AA281CD100
:1099600008464078801C40490978884205DD3E4819
:109970000078401C3C4908700FE03A483A490978A1
:10998000405C552806D100203749087001202C4939
:10999000887102E000203449087010BD10B540F213
:1099A0002551324813F0C4FCE8B13148D0F8000426
:1099B00040F2FF31884203D300202D49C1F8000452
:1099C0002A48001D0088C1B22948D0F80024D0F8E8
:1099D0000004401C264BC3F8000418468154202183
:1099E000224813F09CFC10BD10B51748007850B900
:1099F0004FF40051164813F04EF820B94FF40051BF
:109A0000134813F062F840F22551184813F090FC07
:109A100001285DD140F22551114813F0B3FC1348E1
:109A200013F006FCC1B2134802780078401C23E012
:109A300008000020E0030020200000200018014062
:109A4000A00300204F000020280000205804002020
:109A5000000C01406E000020700100207201002007
:109A600000380140A2080020990000200044004076
:109A7000E01500209A0000202D4B18702D488154CD
:109A80000078AD2821D118460078022800DA10BDF0
:109A900028484078FC280FD125480078052817DD94
:109AA00023480178234800F042FF00202049087035
:109AB0000120214948700BE000201D4908701D4815
:109AC00041781EA020F09CF902E00020184908709F
:109AD00000BFDCE710B540F225511A4813F028FC0E
:109AE000012824D1174813F0A3FBC1B2164802780D
:109AF0000078401C144B1870144881540078AA2830
:109B00000ED11248407855280AD110488078C01CE0
:109B10001946097888420ADC00201946087006E0D8
:109B200009480078022802DB00200749087010BDB0
:109B30009A000020E4080020A003002025780D0AE8
:109B400000000000004800409B0000207409002035
:109B50000146CA1701EB92729210A1EB820292B9F0
:109B6000642091FBF0F200FB121050B94FF4C87062
:109B700091FBF0F200FB121008B9012070470020A1
:109B8000FCE70120FAE70020F8E7F0B503460C46B1
:109B90001546642093FBF0F0C6B2642093FBF0F707
:109BA00000FB1730C1B2132E02DD01F16400C1B217
:109BB0000846CF1701EB977701EBA707BAB207204A
:109BC00092FBF0F700FB172082B25719601EDFF8F6
:109BD00014C41CF80000384482B2CF1701EB977709
:109BE000BF10A1EB87071FB9032C01DA501E82B208
:109BF000072092FBF0F700FB1720C0B2F0BD2DE963
:109C0000F05F06460F4690469946DDE90AAB002410
:109C100040F2DF70864203DB40F63300864202DD0D
:109C20000120BDE8F09F40F2B2750AE02846FFF738
:109C30008FFF10B1EC48044401E0EC480444681C78
:109C400085B2B542F2DB781EC7B2002510E0E848C5
:109C5000405D40F2A321484304EBC0143046FFF7B7
:109C600077FF18B1012D01D1E2480444681C85B288
:109C7000BD42ECDBA8F1010040F2A321484304EB14
:109C8000C014C9EB4910C0EB092004EB0014CAEB67
:109C90000A1004EB80045C4413F0EAFB204613F046
:109CA000B4FB0121080713F02CF9012014F041FB4B
:109CB00013F0DEFB0121084613F07EFB0020B0E725
:109CC00070B500260024002513F096FB0646C9480F
:109CD000B6FBF0F4C8480088A04235D0C6490C80D5
:109CE00040F2B2750AE02846FFF732FF10B1A4F542
:109CF000B77401E0A4F26D14681C85B2B4F5B67FA8
:109D0000F1D8BE480580002516E0BC490888FFF759
:109D10001FFF30B1012D04D11D2C01D31D3C09E0E2
:109D20000CE0B348405DA04203D8B148405D241A1E
:109D300000E003E0681C85B21C2CE6D200BF681C62
:109D4000AE498870601CC870AA48B6FBF0F100FBF1
:109D500011644FF46160B4FBF0F0A84948714FF40E
:109D60006160B4FBF0F100FB11403C21B0FBF1F06D
:109D7000A24988714FF46160B4FBF0F100FB11401F
:109D80003C21B0FBF1F201FB12009C49C87100209C
:109D900070BD1CB5042014F05CFB4AF2A55188424A
:109DA0003BD001214FF0C05013F0ABF8012014F06C
:109DB000C0FA14F019FB012013F003F8002401E0AD
:109DC000601C84B241F288308442F9DB00BF41203C
:109DD00012F05FFF0028FAD04FF4807013F00DF8F6
:109DE000012013F010F813F04CFB13F041FB47F681
:109DF000FF7013F017FB13F03BFB4AF2A551042050
:109E000014F01BFB00200090034601221146019034
:109E100040F2DF70FFF7F3FE1BE001214FF0C0506E
:109E200013F06FF8002401E0601C84B241F2883026
:109E30008442F9DB7B2012F02CFF10B97A2012F05B
:109E400028FF13F08FF80121084613F0B5FA13F03C
:109E50000FFB1CBD10B56A48007C012813D169486E
:109E600090F82D0007280ED06748007800B110BD8B
:109E700011F0ECFD65480078032801D164490870B1
:109E800000205F49087400BFF1E708B503208DF892
:109E900000008DF8010000208DF8020001208DF8EF
:109EA0000300684612F00DFC08BD10B501214FF00B
:109EB000C05013F026F8012014F03BFA14F094FA85
:109EC000012012F097FF00BF612012F0E2FE00288F
:109ED000FAD04FF4007012F090FF012012F093FFBF
:109EE00013F0CFFA13F0C4FA0121022013F064FA40
:109EF00013F0BEFA49F6404013F094FA13F0B8FAA2
:109F0000FFF7C3FF13F078FA841C204613F098FA89
:109F100013F0AEFA10BD1CB501214FF0C05012F085
:109F2000F0FF012014F005FA14F05EFA012012F09F
:109F300061FF00BF612012F0ACFE0028FAD04FF4A0
:109F4000007012F05AFF012012F05DFF13F099FA31
:109F500013F08EFA49F6404013F064FA13F088FAD1
:109F60004FF4003012F09BFC04208DF80400C00375
:109F7000009008208DF8050001208DF80600684645
:109F800012F016FC1CBD10B54FF4803012F05EFECE
:109F900012F09BFE1F4908700846007801280FD177
:109FA00012F0C8FE00BF392012F073FE0028FAD06C
:109FB000022012F0C2FE00BF12F0C8FE0828FBD13A
:109FC00010BD70B5044613F017FA0519284613F0B2
:109FD00037FA13F04DFA0221002014F0BDF9FFF713
:109FE000D2FF70BDFCA802080085E2018033E101C8
:109FF00008A9020880510100800000202A000020EA
:10A00000A0030020580400204D000020ED00002097
:10A01000EC0000207E00002008B50121202012F075
:10A0200063FF40F21F30ADF8000010208DF80300F0
:10A0300003208DF802006946134812F099FC08BD10
:10A0400070B5044600251BE04FF400710E4812F075
:10A050003EFD04F0800028B14FF480710A4812F0F0
:10A0600034FD04E04FF48071074812F030FD6006C3
:10A07000040E4FF40071044812F027FD681CC5B2AD
:10A08000082DE1DB304670BD0014014010B50024FE
:10A0900000F06DF9D02000F0FFF90446012C02D049
:10A0A00000F08EF910BD00F0BCF9802000F0F4F94A
:10A0B0000446012C02D000F083F9F3E700F0B1F977
:10A0C00000F07EF900BFEDE770B500F050F9D12047
:10A0D00000F0E2F900F0A5F900F012FA044600F0F1
:10A0E00087F900F00DFA054600F082F900F008FA51
:10A0F000064600F065F905EB042086B2304670BDD7
:10A1000070B500206A4908806A4908806A4890F85A
:10A110002800012828D16848407A28B9FFF7B6FFFF
:10A12000022065494872C0E06348407A0128FAD1AC
:10A13000FFF7CAFF5F49088000205F4948725D4809
:10A140000088502803DD01205C49087070BD594823
:10A1500000885B495B4A128821F812005948008840
:10A16000401C58490880A0E05648008818B9534858
:10A1700000780128D7D100205049087001205249A9
:10A1800008708870012429E04D4830F814004849CF
:10A19000088000251AE04A4830F815100246681C6D
:10A1A00032F8100081420FDD104630F815004049AA
:10A1B00008801146681C31F8100021F815003C4851
:10A1C0000188681C22F81010681C85B23D48008880
:10A1D000401C001BA842DEDC601C84B239480088A9
:10A1E0008442D1DB37480088401E354931F81000E1
:10A1F0003649888108468089502801DD0020888101
:10A200004FF448712E481EF042FE2E480088304917
:10A21000088000202B4908802E480078012844D16E
:10A2200000202A4989892C4A2C4B1B7822F81310CC
:10A230002A490978491C294A1170114609780429CC
:10A2400032DD01251FE0002417E0234931F81420F6
:10A250000B46611C33F811108A420CDD1A46611C52
:10A2600032F81100114631F81420611C23F8112036
:10A27000194621F81400611C8CB2C5F10501A142F8
:10A28000E3DC691C8DB2052DDDDB1349C988144A56
:10A2900011800021114A11700E4A11700121114ADA
:10A2A00011700021104A117000BF00BF4EE700007E
:10A2B0009400002096000020A003002098000020B9
:10A2C0001005002086000020F8000020580400201F
:10A2D00092000020D90000205808002090000020A3
:10A2E0008E000020910000200C0100200F2000BFF4
:10A2F0000100A0F10102D0B2FAD170474FF4FA7018
:10A3000000BF0100A0F1010290B2FAD1704708B578
:10A310000121042012F0E8FD3020ADF800001420E7
:10A320008DF8030003208DF802001020FA49086020
:10A33000202008606946F848103812F019FB012106
:10A34000402012F0D1FD0C20ADF8000014208DF853
:10A35000030003208DF802000820F0490860042063
:10A3600008606946ED48103812F002FB08BD00B5E0
:10A370001020E9490860FFF7B9FF2020E64908608E
:10A38000FFF7B4FFE4480838006800F0100008B98F
:10A39000012000BD1020E049091D0860FFF7A6FF5D
:10A3A000DD480838006800F0100008B10220F0E72E
:10A3B0002020D949091D0860FFF798FF0020E8E731
:10A3C00000B52020D449091D0860FFF78FFF102039
:10A3D000D149091D0860FFF789FF2020CE49086098
:10A3E000FFF784FF1020CC490860FFF77FFF00BD16
:10A3F00000B52020C849091D0860FFF777FF10202D
:10A40000C549091D0860FFF771FF2020C249086097
:10A41000FFF76CFF2020C049091D0860FFF766FFA9
:10A4200000BD00B52020BC49091D0860FFF75EFF94
:10A430002020B9490860FFF759FF1020B64908608D
:10A44000FFF754FF2020B449091D0860FFF74EFFB5
:10A4500000BD00B52020B049091D0860FFF746FF88
:10A460001020AD490860FFF741FF2020AA4908608D
:10A47000FFF73CFFA8480838006800F0100028B13A
:10A480002020A549091D0860002000BD2020A24908
:10A49000091D08600120F8E710B5034620209E49F9
:10A4A000091D086000241BE020209B49091D08604D
:10A4B000FFF71CFF03F0800018B1102096490860D8
:10A4C00003E010209449091D08605806030EFFF7A9
:10A4D0000DFF202090490860FFF708FF601CC4B200
:10A4E000082CE1DB20208C49091D08608A480838C7
:10A4F000006800F0100008B1002010BD0120FCE74A
:10A5000010B5002310208449086000BF00241AE021
:10A510005806030E20208049091D0860FFF7E6FE5B
:10A5200020207D490860FFF7E1FE7B48083800687D
:10A5300000F0100008B143F0010320207649091D06
:10A540000860601CC4B2082CE2DB184610BD00B5E0
:10A5500008207249086004200860FFF7CFFE6F48AA
:10A560000838006800F0080008B9012000BD082084
:10A570006A49091D0860FFF7C1FE6848083800688D
:10A5800000F0080008B10220F0E704206349091D2B
:10A590000860FFF7B3FE0020E8E700B504205F493C
:10A5A000091D0860FFF7AAFE08205C49091D086024
:10A5B000FFF7A4FE042059490860FFF79FFE08201A
:10A5C00056490860FFF79AFE00BD00B504205349C4
:10A5D000091D0860FFF792FE08205049091D086018
:10A5E000FFF78CFE04204D490860FFF787FE04202A
:10A5F0004A49091D0860FFF781FE00BD00B504202F
:10A600004649091D0860FFF779FE082043490860A4
:10A61000FFF774FE042041490860FFF76FFE042035
:10A620003E49091D0860FFF769FE00BD00B5042022
:10A630003A49091D0860FFF761FE082037490860A4
:10A64000FFF75CFE042035490860FFF757FE3348EA
:10A650000838006800F0080028B104202F49091DBF
:10A660000860002000BD04202C49091D086001205D
:10A67000F8E710B5034600241BE004202749091D14
:10A680000860FFF73BFE03F0800018B10820234963
:10A69000086003E008202149091D08605806030EE0
:10A6A000FFF72CFE04201D490860FFF727FE601C01
:10A6B000C4B2082CE1DB04201849091D0860FFF72B
:10A6C000B5FF08B9002010BD0120FCE710B500233C
:10A6D000082012490860002416E05806030E0420E2
:10A6E0000E49091D0860FFF709FE04200B490860A8
:10A6F000FFF704FE09480838006800F0080008B1B8
:10A7000043F00103601CC4B2082CE6DB04200349BB
:10A71000091D0860184610BD1008014010180140BE
:10A72000704710B586B004460121880312F0DCFBA7
:10A730000121042012F0D8FB4FF40070ADF8140092
:10A7400003208DF8160018208DF8170005A9A348DE
:10A7500012F00EF94FF48060ADF8140048208DF827
:10A76000170005A99D4812F003F90121880312F092
:10A77000D5FB00214FF4804012F0D0FB0194002063
:10A78000ADF80800ADF80A00ADF80C00ADF8100007
:10A790000C20ADF80E0001A9914812F04CFC2520C8
:10A7A0008DF8000003208DF801008DF802000120D3
:10A7B0008DF80300684611F084FF012240F2255114
:10A7C000874812F0D0FC0121854812F0C0FC06B089
:10A7D00010BD10B586B004460121480412F091FB6B
:10A7E0000121042012F080FB0420ADF81400182091
:10A7F0008DF8170003208DF8160005A9774812F090
:10A80000B7F80820ADF8140048208DF8170005A906
:10A81000724812F0ADF80121480412F08CFB0021BF
:10A820004FF4003012F087FB01940020ADF80800CF
:10A83000ADF80A00ADF80C00ADF810000C20ADF832
:10A840000E0001A9674812F0F6FB26208DF80000E3
:10A8500000208DF801008DF8020001208DF8030022
:10A86000684611F02EFF012240F225515D4812F09A
:10A870007AFC01215B4812F06AFC06B010BD10B5ED
:10A8800086B004460121082012F02EFB0121880425
:10A8900012F037FB4FF48060ADF8140018208DF8EB
:10A8A000170003208DF8160005A94F4812F060F834
:10A8B0004FF40060ADF8140004208DF8170005A9CE
:10A8C000494812F055F80121880412F034FB0021A8
:10A8D0004FF4802012F02FFB01940020ADF8080007
:10A8E000ADF80A00ADF80C00ADF810000C20ADF882
:10A8F0000E0001A93D4812F09EFB27208DF80000B4
:10A9000003208DF801008DF8020001208DF803006E
:10A91000684611F0D6FE012240F22551334812F06C
:10A9200022FC0121314812F012FC06B010BD70B5B6
:10A9300004460D4600260DE000BF4021284812F0D5
:10A94000E1FC0028F9D014F8011B254812F06CFC3A
:10A95000701CC6B2AE42EFD300BF4021204812F0B7
:10A96000D1FC0028F9D070BD70B504460D46002614
:10A970000DE000BF40211B4812F0C4FC0028F9D0B4
:10A9800014F8011B174812F04FFC701CC6B2AE42FF
:10A99000EFD300BF4021134812F0B4FC0028F9D0D7
:10A9A00070BD70B504460D4600260DE000BF402185
:10A9B0000E4812F0A7FC0028F9D014F8011B0B4830
:10A9C00012F032FC701CC6B2AE42EFD300BF402181
:10A9D000064812F097FC0028F9D070BD000801402D
:10A9E0000038014000440040000C01400048004095
:10A9F00010B50820FB4908606420FDF777FF0820A8
:10AA0000F849091F08603220FDF770FF10BD10B52E
:10AA100004461020F3490860042008602046FFF730
:10AA20000FFB10BD10B504461020EE49086004204D
:10AA3000091F08602046FFF703FB1020E949091FA2
:10AA4000086010BD70B505460C462846FFF7EAFFC2
:10AA50002046FFF7E7FF70BD2DE9F04104460D46A3
:10AA600016461F464020FFF7D2FFB020FFF7CFFF6A
:10AA70001020FFF7CCFF0020FFF7C9FFE1B2201242
:10AA8000FFF7E0FFF1B23012FFF7DCFFB020FFF775
:10AA9000BEFF1020FFF7BBFF0020FFF7B8FFE9B2B1
:10AAA0002812FFF7CFFFF9B23812FFF7CBFFBDE84E
:10AAB000F08110B5FFF79CFFE220FFF7A8FFA2206E
:10AAC000FFF7A5FFA120FFF7A2FFC820FFF79FFF18
:10AAD0002720FFF79CFFF820FFF799FF0020FFF7E2
:10AAE00096FF8120FFF793FF5420FFF790FF2C2063
:10AAF000FFF78DFF2E20FFF78AFF2F20FFF787FF3C
:10AB00004020FFF784FFB020FFF781FF1020FFF700
:10AB10007EFF0020FFF77BFFAF20FFF778FF10BD1F
:10AB200070B506464020FFF772FF00251AE045F099
:10AB3000B000FFF76CFF002410E0102141EA241060
:10AB4000FFF765FF04F00F00FFF761FF0020FFF73C
:10AB500069FF0020FFF766FF601CC4B2832CECDBAA
:10AB6000681CC5B2092DE2DB70BD2DE9F047064631
:10AB70000F469046994600251DE0A8EB0501C9B295
:10AB800041F0B000FFF743FF344610E0102141EAE6
:10AB90002410FFF73CFF04F00F00FFF738FF002000
:10ABA000FFF740FF0020FFF73DFF601CC4B2BC422E
:10ABB000ECDB681CC5B24D45DFDBBDE8F08770B546
:10ABC00004460D464020FFF722FFE9B241F0B000F5
:10ABD000FFF71DFF102141EA2411C8B2FFF717FF4C
:10ABE00004F00F00FFF713FF70BD2DE9F041074699
:10ABF0000D4614464020FFF70AFFB820FFF707FF75
:10AC0000102141EA2411C8B2FFF701FF04F00F0040
:10AC1000FFF7FDFE002607E03846FFF703FF284652
:10AC2000FFF700FF701CC6B2052EF5DBBDE8F08112
:10AC30002DE9F04104460F4615464020FFF7E7FE98
:10AC400000261DE0B91BC9B241F0B000FFF7DFFEDE
:10AC5000102141EA2420FFF7DAFEE0B2FFF7D7FE29
:10AC60004FF0000807E02878FFF7DCFE6D1C08F1C4
:10AC7000010000F0FF08B8F1180FF4DB701CC6B239
:10AC8000032EDFDBBDE8F0812DE9F04104460F46DD
:10AC900015464020FFF7BBFE00261FE0B91BC9B2D6
:10ACA00041F0B000FFF7B3FE102141EA2411C8B211
:10ACB000FFF7ADFE04F00F00FFF7A9FE4FF000080C
:10ACC00007E02878FFF7AEFE6D1C08F1010000F0E8
:10ACD000FF08B8F1100FF4DB701CC6B2022EDDDBEA
:10ACE000BDE8F0812DE9F04104460F4615464020AD
:10ACF000FFF78DFE00261FE0B91BC9B241F0B0007E
:10AD0000FFF785FE102141EA2411C8B2FFF77FFE4C
:10AD100004F00F00FFF77BFE4FF0000807E02878F3
:10AD2000FFF780FE6D1C08F1010000F0FF08B8F18C
:10AD30000C0FF4DB701CC6B2022EDDDBBDE8F08127
:10AD40002DE9F047044688461546E7B24020FFF754
:10AD50005EFE002622E0E7B2A8EB0601C9B241F090
:10AD6000B000FFF754FE102141EA2710FFF74FFE15
:10AD700007F00F00FFF74BFE4FF0000909E02878BD
:10AD8000FFF750FE6D1C781CC7B209F1010000F0FE
:10AD9000FF09B9F1050FF2DB701CC6B2012EDADB38
:10ADA000BDE8F0872DE9F047044688461546E7B22E
:10ADB0004020FFF72CFE002625E0E7B2A8EB0601B5
:10ADC000C9B241F0B000FFF722FE102141EA27107E
:10ADD000FFF71DFE07F00F00FFF719FE4FF0000907
:10ADE0000CE00000141401402878FFF71BFE6D1CD6
:10ADF000781CC7B209F1010000F0FF09B9F1060F94
:10AE0000F2DB701CC6B2022ED7DBBDE8F0872DE95D
:10AE1000F047044688461546E7B24020FFF7F7FDA5
:10AE2000002622E0E7B2A8EB0601C9B241F0B0006B
:10AE3000FFF7EDFD102141EA2710FFF7E8FD07F0CD
:10AE40000F00FFF7E4FD4FF0000909E02878FFF755
:10AE5000E9FD6D1C781CC7B209F1010000F0FF0983
:10AE6000B9F1080FF2DB701CC6B2022EDADBBDE8C6
:10AE7000F087000070B50024FE488079012870D169
:10AE8000FD48807810286ED1AA222046611CCCB2E1
:10AE9000FA490A5417222046611CCCB2F7490A54D9
:10AEA00011222046611CCCB2F4490A54002508E066
:10AEB000F348425D2046611CCCB2F0490A54681C3C
:10AEC000C5B2102DF4DBEF488168007B4FF07F4363
:10AED00019400020020242EA1160C2B22046611C01
:10AEE000CCB2E6490A54E7488168007B1B0A194046
:10AEF0000020020442EA1140C2B22046611CCCB2DA
:10AF0000DE490A54DF490889097B1B1218400021D9
:10AF1000000A40EA0160C2B22046611CCCB2D749A7
:10AF20000A54D848027A2046611CCCB2D3490A544C
:10AF3000D44882782046611CCCB2D0490A54D1480A
:10AF400002792046611CCCB2CC490A5455222046D5
:10AF5000611CCCB2C9490A541A21C848FFF7E7FC62
:10AF60001EE120E1FFE7C44880782028F8D1AA221A
:10AF70002146601CC4B2C14842541D222046611CB7
:10AF8000CCB2BE490A5421222046611CCCB2BB4936
:10AF90000A54BC488168007B4FF07F431940002071
:10AFA000020242EA1160C2B22046611CCCB2B3492F
:10AFB0000A54B4488168007B1B0A1940002002042F
:10AFC00042EA1140C2B22046611CCCB2AB490A54DD
:10AFD000AC480189007B1A1211400020020642EAA7
:10AFE0001120C2B22046611CCCB2A4490A54A54823
:10AFF000027A2046611CCCB2A0490A54A14882784A
:10B000002046611CCCB29D490A549E4802792046D4
:10B01000611CCCB299490A549B490888C11700EBBE
:10B020001161C1F307232146621CD4B2934A5354E1
:10B0300095490888C11700EB11610912A0EB0121A5
:10B04000CBB22146621CD4B28C4A53548E488278CB
:10B050002046611CCCB289490A548B4802792046AB
:10B06000611CCCB285490A54874882792046611C0C
:10B07000CCB282490A548448027A2046611CCCB280
:10B080007E490A5480494889C11700EB1161C1F318
:10B0900007232146621CD4B2784A53547A4948891E
:10B0A000C11700EB11610912A0EB0121CBB22146BF
:10B0B000621CD4B2714A53547348827C2046611C8E
:10B0C000CCB26E490A547048C27C2046611CCCB296
:10B0D0006A490A546C48027D2046611CCCB267491B
:10B0E0000A546948427D2046611CCCB263490A5427
:10B0F00065498889C11700EB1161C1F30723214617
:10B10000621CD4B25D4A53545F498889C11700EB71
:10B1100011610912A0EB0121CBB22146621CD4B20D
:10B12000564A53545849C889C11700EB1161C1F3FD
:10B1300007232146621CD4B2504A53545249C8894D
:10B14000C11700EB11610912A0EB0121CBB221461E
:10B15000621CD4B2494A53544B49088AC11700EBC8
:10B160001161C1F307232146621CD4B2434A5354F0
:10B170004549088AC11700EB11610912A0EB0121B2
:10B18000CBB22146621CD4B23C4A535455222046CD
:10B19000611CCCB239490A5421463848FFF7C7FB35
:10B1A00000203449887170BD1CB5002000900190CA
:10B1B000364A0621684600F021FC9DF8000034491B
:10B1C0000880084600884FF6FF7101EA00203049E8
:10B1D00008809DF80100098808442D4908809DF8E1
:10B1E00002002C490880084600884FF6FF7101EAEA
:10B1F0000020284908809DF8030009880844254953
:10B2000008809DF8040024490880084600884FF60D
:10B21000FF7101EA0020204908809DF80500098897
:10B2200008441D4908801A4800880A2802DD0020C9
:10B2300017490880174800880A2802DD00201549B0
:10B24000088015480088642802DD00201249088023
:10B250001CBD70B5002400250B48C07E4FF6FF7161
:10B2600001EAC0250D482A184FF400610C4800F08F
:10B27000C5FB17E0A0030020A20800206208002000
:10B28000A9040020980400209409002000980608D2
:10B290009C0000209E000020A2000020004806081C
:10B2A000B00900202146641CFC48405CFC49088031
:10B2B000084600884FF6FF7101EA0020F84908802F
:10B2C000084602882146641CF448405C1044F44956
:10B2D000088008460088B0F57A7F01DB00200880EE
:10B2E0002046611CCCB2ED49085CED494880084617
:10B2F00040884FF6FF7101EA0020E949488008467E
:10B3000042882046611CCCB2E449085C1044E44900
:10B31000488008464088632801DD00204880204698
:10B32000611CCCB2DD49085CDD4988800846808814
:10B330004FF6FF7101EA0020D949888008468288CB
:10B340002046611CCCB2D549085C1044D4498880A1
:10B3500008468088B0F57A7F01DB0020888020468F
:10B36000611CCCB2CD49085CCD49C8800846C08874
:10B370004FF6FF7101EA0020C949C8800846C2881B
:10B380002146601CC4B2C548405C1044C449C88012
:10B390000846C088B0F57A7F01DB0020C8802046CF
:10B3A000611CCCB2BD49085CBD49088108460089D2
:10B3B0004FF6FF7101EA0020B94908810846028969
:10B3C0002046611CCCB2B549085C1044B4490881E0
:10B3D00008460089632801DD002008812046611CA1
:10B3E000CCB2AE49085CAE494881084640894FF668
:10B3F000FF7101EA0020AA49488108464289214696
:10B40000601CC4B2A548405C1044A5494881084668
:10B4100040895A2801DD002048812046611CCCB2B9
:10B420009E49085C9E4908820846008A4FF6FF71D3
:10B4300001EA00209A4908820846028A2146601CD7
:10B44000C4B29648405C1044954908820846008A78
:10B4500042F20F71884202DD0020914908822046A5
:10B46000611CCCB28D49085C8D4988810846808971
:10B470004FF6FF7101EA00208949888108468289D8
:10B480002046611CCCB28549085C104484498881FF
:10B4900008468089B0F57A7F01DB0020888120464C
:10B4A000611CCCB27D49085C7D49C8810846C089D1
:10B4B0004FF6FF7101EA00207949C8810846C28928
:10B4C0002146601CC4B27548405C10447449C88170
:10B4D0000846C089B0F57A7F01DB0020C88120468C
:10B4E000611CCCB26D49085C6D4988740846807C4B
:10B4F0000C2801DD012088742046611CCCB267490C
:10B50000085C6749C8740846C07C1F2801DD01201B
:10B51000C8742046611CCCB26049085C604908755B
:10B520000846007D172801DD002008752046611CB3
:10B53000CCB25A49085C5A4948750846407D3B28B8
:10B5400001DD002048752046611CCCB25349085CDF
:10B55000534988750846807D0C2801DD01208875D7
:10B560002046611CCCB24D49085C4D49C87508465F
:10B57000C07D1F2801DD0120C8752046611CCCB2AA
:10B580004649085C464908760846007E172801DDD2
:10B59000002008762046611CCCB24049085C404936
:10B5A00048760846407E3B2801DD0020487620464C
:10B5B000611CCCB23949085C394988760846807EDE
:10B5C000082801DD0020887670BD1CB500200090A1
:10B5D0000190344800880A2812DD32480088C828C3
:10B5E0000EDA0A202F4908802F480088401C2E4977
:10B5F0000880084600880A2809DB0020088006E049
:10B6000028480088C82802DB0020264908802748EF
:10B610000088642802DD64202449088021490888C4
:10B62000C11700EB1161090A8DF800101D49088847
:10B63000C11700EB11610912A0EB0121C9B28DF80D
:10B64000011019490888C11700EB1161090A8DF82A
:10B65000021015490888C11700EB11610912A0EB0F
:10B660000121C9B28DF8031010490888C11700EBF9
:10B670001161090A8DF804100C490888C11700EB04
:10B6800011610912A0EB0121C9B28DF80510084A19
:10B690000621684600F086F91CBD0000B0090020B4
:10B6A000940900209C0000209E000020A2000020A1
:10B6B0000098060870B500240025B049088DC11710
:10B6C00000EB1161C1F307232246641CAC498B5483
:10B6D000AA49088DC11700EB11610912A0EB0121E5
:10B6E000CBB22246641CA6498B54A449488DC1178D
:10B6F00000EB1161C1F307232246641CA0498B545F
:10B700009E49488DC11700EB11610912A0EB012180
:10B71000CBB22246641C9A498B549A49C888C117F7
:10B7200000EB1161C1F307232246641C94498B543A
:10B730009449C888C11700EB11610912A0EB0121DF
:10B74000CBB22246641C8E498B548E494889C1175E
:10B7500000EB1161C1F307232246641C88498B5416
:10B7600088494889C11700EB11610912A0EB01213A
:10B77000CBB22146621CD4B2814A53548149888994
:10B78000C11700EB1161C1F307232146621CD4B23B
:10B790007B4A53547B498889C11700EB1161091218
:10B7A000A0EB0121CBB22146621CD4B2744A53549F
:10B7B00074490889C11700EB1161C1F307232146C1
:10B7C000621CD4B26E4A53546E490889C11700EB0B
:10B7D00011610912A0EB0121CBB22146621CD4B247
:10B7E000674A53546849888CC11700EB1161C1F353
:10B7F00007232146621CD4B2614A53546249888CA3
:10B80000C11700EB11610912A0EB0121CBB2214657
:10B81000621CD4B25A4A53545B49088DC11700EBDD
:10B820001161C1F307232146621CD4B2544A535418
:10B830005549088DC11700EB11610912A0EB0121D8
:10B84000CBB22146621CD4B24D4A53544E49488D66
:10B85000C11700EB1161C1F307232146621CD4B26A
:10B86000474A53544849488DC11700EB11610912EA
:10B87000A0EB0121CBB22146621CD4B2404A535402
:10B88000424882782046611CCCB23D490A543F4868
:10B89000C2782046611CCCB239490A543B484279EF
:10B8A0002046611CCCB236490A5438488279204679
:10B8B000611CCCB232490A54354802782046611CDA
:10B8C000CCB22F490A54324842782046611CCCB28F
:10B8D0002B490A542E4882782046611CCCB2284954
:10B8E0000A542B48C2782046611CCCB224490A5421
:10B8F000274802792046611CCCB221490A5404E051
:10B9000000201F490855601CC4B2202CF8DB2148D8
:10B9100000880A2812DB2048008838B91D480088B2
:10B92000401E4FF6FF7101EAC0250EE01A4800885C
:10B93000401E4FF6FF7101EAC02506E01548008859
:10B94000401E4FF6FF7101EAC02514482A186421F1
:10B950000B4800F027F870BD0E480088401C0D49C8
:10B9600008800F480088401C0D4908800846008860
:10B97000642801DD6420088070470000A8040020CE
:10B98000B0090020E4040020580400202A00002010
:10B99000330000209C0000209E0000200048060884
:10B9A000A20000202DE9F04105460E46174612F090
:10B9B0009CFD342013F034F8384612F0DBFD0024EF
:10B9C00013E015F814804FF6FF7000EA08280120F4
:10B9D00000EB4400285C40441FFA80F807EB440069
:10B9E000414612F0CAFE601C84B206EBD671B4EB7D
:10B9F000610FE6DB12F085FDBDE8F081F0B503468E
:10BA00000C4615460021002015E035F810100A46B6
:10BA1000CE1701EB1666C6F3072603F81060CE17A3
:10BA200001EB16663612A1EB0626012707EB40074D
:10BA3000DE55421C90B204EBD476B0EB660FE4DB2B
:10BA4000F0BD00002DE9F04100240026FE4A8021CF
:10BA5000FE48FFF7D3FF002506E02046611CCCB26C
:10BA6000FA490E5C681CC5B2102DF6DB2046611C3D
:10BA7000CCB2F649085CF64948742046611CCCB249
:10BA8000F249095CF24881742046611CCCB2EF494E
:10BA9000095CEF48C174002505E00021EC48113035
:10BAA0004155681CC5B2032DF7DB00250DE020468B
:10BAB000611CCCB2E549085CE64948550846415D41
:10BAC000E3481E304155681CC5B2092DEFDB002547
:10BAD0000DE02046611CCCB2DC49085CDD494855CC
:10BAE0000846415DDA4818304155681CC5B2032D3F
:10BAF000EFDB00250DE02046611CCCB2D349085C89
:10BB0000D44948550846415DD1481B304155681C11
:10BB1000C5B2032DEFDB2046611CCCB2CB49085CDB
:10BB2000CB4908850846008D4FF6FF7101EA0020D9
:10BB3000C74908850846028D2046611CCCB2C3491E
:10BB4000085C1044C24908850846008DB0F57A7F2C
:10BB500001DB002008852046611CCCB2BB49085C93
:10BB6000BB4948850846408D4FF6FF7101EA002029
:10BB7000B74948850846428D2046611CCCB2B3497E
:10BB8000085C1044B24948850846408D632801DDB1
:10BB9000002048852046611CCCB2AC49085CAC4909
:10BBA00088850846808D4FF6FF7101EA0020A8497C
:10BBB00088850846828D2046611CCCB2A349085C6A
:10BBC0001044A34988850846808DB0F5FA7F01DDD1
:10BBD000002088852046611CCCB29C49085C9C49A9
:10BBE000C8850846C08D4FF6FF7101EA00209849CC
:10BBF000C8850846C28D2046611CCCB29349085CBA
:10BC000010449349C8850846C08D642801DD002092
:10BC1000C8852046611CCCB28C49085C8C490886DA
:10BC20000846008E4FF6FF7101EA00208849088619
:10BC30000846028E2046611CCCB28449085C104440
:10BC4000834908860846008E642801DB01200886A7
:10BC50002046611CCCB27D49085C7D494886084677
:10BC6000408E4FF6FF7101EA002079494886084668
:10BC7000428E2046611CCCB27449085C1044744961
:10BC800048860846408EC82801DD5A20488620464E
:10BC9000611CCCB26D49085C6D4988860846808E6F
:10BCA0004FF6FF7101EA0020694988860846828EB6
:10BCB0002046611CCCB26549085C10446449888602
:10BCC0000846808E632801DD002088862046611C9E
:10BCD000CCB25E49085C5E49C8860846C08E4FF605
:10BCE000FF7101EA00205A49C8860846C28E2046E4
:10BCF000611CCCB25549085C10445549C8860846B9
:10BD0000C08E632801DD0020C8862046611CCCB2AD
:10BD10004E49085C4E4908870846008F4FF6FF7170
:10BD200001EA00204A4908870846028F2046611C24
:10BD3000CCB24649085C1044454908870846008F44
:10BD4000632802DC0846008F10B9012040490887AB
:10BD50002046611CCCB23D49085C3D4948870846F5
:10BD6000408F4FF6FF7101EA0020394948870846A5
:10BD7000428F2046611CCCB23449085C10443449DF
:10BD800048870846408FB0F57A7F01DB002048875E
:10BD90002046611CCCB22D49085C2F49087008462A
:10BDA0000078012803DB08460078032802DD032021
:10BDB00029490870002029494880002513E02748B8
:10BDC000418823481830405D08442449488008468B
:10BDD000408800EB80004FF6FF7101EA40001F49E8
:10BDE0004880681CC5B21C480078401EA842E6DCAA
:10BDF0001A48418816481830405D08441749488061
:10BE00002046611CCCB21149085C1349C870084631
:10BE1000C078012801DD0020C8702046611CCCB22A
:10BE20000A49085C0C49487008464078012803DB41
:10BE300008464078032802DD0320074948700020A7
:10BE40000649888000251EE000400608B011002049
:10BE5000A804002030120020FE04002098040020D6
:10BE6000FE488188FE48405D0844FC4988800846B9
:10BE7000808800EB80004FF6FF7101EA4000F7492F
:10BE80008880681CC5B2F7484078401EA842E7DCAD
:10BE9000F2488188F248405D0844F0498880204695
:10BEA000611CCCB2F049085CEE4908710846007983
:10BEB000012801DD002008712046611CCCB2EA494E
:10BEC000085CE849C8810846C0894FF6FF7101EA5D
:10BED0000020E449C8810846C2892046611CCCB2D2
:10BEE000E149085C1044DF49C8810846C0896428DC
:10BEF00001DD6420C8812046611CCCB2DA49085CAF
:10BF0000D849487108464079012801DD0020487170
:10BF10002046611CCCB2D449085CD24988700846DE
:10BF20008078012803DB084680780A2802DD092092
:10BF3000CC4988700020C94A9060D06000251BE081
:10BF4000C648D0E90230C649C91C495D591840F1BC
:10BF50000000C24AC2E9021010460A23D0E90212C8
:10BF60000020A1FB037C02FB03C201FB0020BB49B4
:10BF7000C1E90270681CC5B2BA488078401EA84268
:10BF8000DEDCB648D0E90230B549C91C495D591814
:10BF900040F10000B14AC2E902102046611CCCB257
:10BFA000B149085CAF49887108468079012801DDF4
:10BFB000002088712046611CCCB2AB49085CA949BD
:10BFC000C8720846C07A012801DD0020C8722046E8
:10BFD000611CCCB2A449085CA249C8710846C0796A
:10BFE000012801DD0020C8712046611CCCB29E49A9
:10BFF000085C9C4988720846807A012801DD00208F
:10C0000088722046611CCCB29749085C9549087239
:10C010000846007A012801DD002008722046611CD4
:10C02000CCB29149085C8F4908730846007B01280F
:10C0300001DD012008732046611CCCB28A49085CEE
:10C04000884948720846407A012801DD002048727C
:10C050002046611CCCB28449085C824908740846B9
:10C06000007C012801DD002008742046611CCCB250
:10C070007D49085C7B4948740846407C012801DD05
:10C0800000204874BDE8F0812DE9F041002400252E
:10C0900009E073481A38425D2046611CCCB27249EF
:10C0A0000A54681CC5B2102DF3DB00206F4A1063E0
:10C0B000506300251BE06D48D0E90C3068491A39FF
:10C0C000495D591840F10000684AC2E90C10114658
:10C0D0000A23D1E90C020021A0FB036702FB0372D3
:10C0E00000FB01206149C1E90C60681CC5B20F2D3D
:10C0F000E1DB5E48D0E90C3059491B39097C5918FD
:10C1000040F10000594AC2E90C1055481B38427CE6
:10C110002046611CCCB254490A5451481B38827CD9
:10C120002046611CCCB250490A544D481B38C27C91
:10C130002046611CCCB24C490A54002514E0494801
:10C140008078A84208DD4648C01C425D2046611C3C
:10C15000CCB245490A5405E000222046611CCCB20D
:10C1600041490A54681CC5B2092DE8DB002514E0DA
:10C170003C480078A84208DD3948C01E425D204690
:10C18000611CCCB238490A5405E000222046611CEB
:10C19000CCB235490A54681CC5B2032DE8DB002532
:10C1A00013E030484078A84207DD2D48425D204624
:10C1B000611CCCB22C490A5405E000222046611CC7
:10C1C000CCB229490A54681CC5B2032DE9DB2448C6
:10C1D0001B38008D020A2046611CCCB222490A5449
:10C1E0001F481B3890F828202046611CCCB21E49FD
:10C1F0000A541B481B38408D020A2046611CCCB2F1
:10C2000019490A5416481B3890F82A202046611C08
:10C21000CCB215490A5412481B38808D020A2046B8
:10C22000611CCCB210490A540D481B3890F82C20E0
:10C230002046611CCCB20C490A5409481B38C08DF9
:10C24000020A2046611CCCB207490A5404481B3834
:10C2500090F82E202046611CCCB209E09804002002
:10C26000C3040020FE040020B01100205804002068
:10C27000FE490A54FE48008E020A2046611CCCB2D8
:10C28000FA490A54FA4890F830202046611CCCB292
:10C29000F6490A54F648408E020A2046611CCCB288
:10C2A000F2490A54F24890F832202046611CCCB280
:10C2B000EE490A54EE48808E020A2046611CCCB238
:10C2C000EA490A54EA4890F834202046611CCCB26E
:10C2D000E6490A54E648C08E020A2046611CCCB2E8
:10C2E000E2490A54E24890F836202046611CCCB25C
:10C2F000DE490A54DE48008F020A2046611CCCB297
:10C30000DA490A54DA4890F838202046611CCCB249
:10C31000D6490A54D648408F020A2046611CCCB246
:10C32000D2490A54D24890F83A202046611CCCB237
:10C33000CE490A54CF4802782046611CCCB2CB4982
:10C340000A54CC48C2782046611CCCB2C7490A5472
:10C35000C84842782046611CCCB2C4490A54C5483A
:10C3600002792046611CCCB2C0490A54C148C08938
:10C37000020A2046611CCCB2BC490A54BD48827BEB
:10C380002046611CCCB2B9490A54BA4842792046C9
:10C39000611CCCB2B5490A54B64882782046611C6B
:10C3A000CCB2B2490A54B34882792046611CCCB25F
:10C3B000AE490A54AF48C27A2046611CCCB2AB49A0
:10C3C0000A54AC48C2792046611CCCB2A7490A5431
:10C3D000A848827A2046611CCCB2A4490A54A548D8
:10C3E000027A2146601CC4B2A0484254A148027B94
:10C3F0002046611CCCB29D490A549E48427A204690
:10C40000611CCCB299490A549A48027C2146601CAE
:10C41000C4B2964842549748427C2046611CCCB234
:10C4200092490A5404E0FF2090490855601CC4B2A8
:10C43000802CF8DB0A208D4981F87E008E4A80210D
:10C440008A48FFF7AFFABDE8F0812DE9F0410024FA
:10C4500000250BE000218648401C4155425D2046E6
:10C46000611CCCB281490A54681CC5B2102DF1DBA5
:10C470000020824A1063506300251FE000217C48A1
:10C48000401C41557D48D0E90C317948401C405D45
:10C49000181841F10001794AC2E90C011146D1E9AD
:10C4A0000C010A230022A0FB036701FB037100FBC0
:10C4B00002107249C1E90C60681CC5B20F2DDDDBAA
:10C4C0006E48D0E90C306A49097C591840F10000E7
:10C4D0006A4AC2E90C10002065494874002164488A
:10C4E0008174C174427C2046611CCCB25F490A54FD
:10C4F0005F48827C2046611CCCB25C490A545C488F
:10C50000C27C2046611CCCB258490A54002516E072
:10C5100058488078A8420ADD002155481E30415510
:10C52000425D2046611CCCB250490A5405E000220D
:10C530002046611CCCB24D490A54681CC5B2092D75
:10C54000E6DB002516E04B480078A8420ADD002112
:10C55000474818304155425D2046611CCCB24349E2
:10C560000A5405E000222046611CCCB23F490A541F
:10C57000681CC5B2032DE6DB002516E03D48407877
:10C58000A8420ADD00213A481B304155425D204651
:10C59000611CCCB235490A5405E000222046611CDA
:10C5A000CCB232490A54681CC5B2032DE6DB002226
:10C5B0002046611CCCB22D490A542046611CCCB2E5
:10C5C0002A490A542046611CCCB228490A54204604
:10C5D000611CCCB225490A542046611CCCB22349C7
:10C5E0000A542046611CCCB220490A542046611CE2
:10C5F000CCB21E490A542046611CCCB21B490A54D5
:10C600002046611CCCB219490A542046611CCCB2A8
:10C6100016490A542046611CCCB214490A5401221E
:10C620002046611CCCB211490A5400222046611CEC
:10C63000CCB20E490A542046611CCCB20B490A54B4
:10C640002046611CCCB209490A542146601CC4B280
:10C65000064842542046611CCCB204490A54204684
:10C66000611CCCB201490A54214609E0B0110020F6
:10C67000A8040020FE040020004006085804002002
:10C68000601CC4B23A4842542046611CCCB23849BE
:10C690000A5403222046611CCCB235490A540022B8
:10C6A0002046611CCCB232490A5403222046611C48
:10C6B000CCB22F490A5400222046611CCCB22C492E
:10C6C0000A5401222046611CCCB229490A54002296
:10C6D0002046611CCCB226490A542046611CCCB2CB
:10C6E00023490A542046611CCCB221490A542046F1
:10C6F000611CCCB21E490A542046611CCCB21C49B4
:10C700000A5401222046611CCCB219490A54204621
:10C71000611CCCB216490A542046611CCCB21449A3
:10C720000A542046611CCCB211490A542046611CAF
:10C73000CCB20F490A542046611CCCB20C490A54B1
:10C740002046611CCCB20A490A5404E0FF20084983
:10C750000855601CC4B2802CF8DB0A20044981F81B
:10C760007E00044A80210248FFF71CF9BDE8F081F1
:10C77000B01100200040060800B58BB0012108462A
:10C7800010F0A5FB914812F097FB9148009091485A
:10C79000019000200290012003900020049080204E
:10C7A000059040000690800007902020089000022D
:10C7B000099000200A906946844812F01FFC01216C
:10C7C000824812F046FC0BB000BD00B587B00121D5
:10C7D0004FF4047010F088FB0420ADF80400002032
:10C7E0008DF8070003208DF8060001A97A4810F0A3
:10C7F000BFF80020029001208DF80C008DF80D008C
:10C800004FF4602004900020059001208DF818005E
:10C8100002A96F484C3812F04EF9052301220C2171
:10C820006B484C3812F0DFF9FFF7A6FF012168488A
:10C830004C3812F077F9012165484C3812F067F94D
:10C8400063484C3812F085F900BF61484C3812F04B
:10C8500085F90028F9D15E484C3812F089F900BFFB
:10C860005B484C3812F089F90028F9D10121584869
:10C870004C3812F08CF907B000BD2DE9F0410027CB
:10C880000026564890F8290001280BD1544800781A
:10C8900048B10020514981F8290042F210705149F5
:10C8A000A1F84E008FE0052301220C214E4812F022
:10C8B0009AF901214C4812F06AF900BF02214A4856
:10C8C00012F0D6FA0028F9D0474812F0F3F90746DB
:10C8D00040F6D3107843070B07EB47004FF6FF7184
:10C8E00001EA40004149424A127821F812004048CA
:10C8F0000078401C3E49087008460078072862DB33
:10C9000000200870022521E0384830F81560022424
:10C9100016E0364830F814100246601C32F8100059
:10C9200081420BDD104630F814600146601C31F87E
:10C93000100021F81400601C21F81060601CC4B2C3
:10C94000C5F10800A042E4DC681CC5B2072DDBDBA2
:10C950002648C0882549098908442449498908444A
:10C96000032190FBF1F086B241F2243086422ADCAA
:10C9700020480680008841F29411884203DD084671
:10C980001C49088008E01B48008840F6B8318842FE
:10C9900002DA0846174908801648008841F29411C7
:10C9A000081A6421484340F2DC5190FBF1F0C0F1D9
:10C9B0006400C0B2104988820020084981F829002B
:10C9C00001200E490870BDE8F08100000800024017
:10C9D0004C240140A400002000100140A0030020CE
:10C9E00028000020E003002000280140AC000020C7
:10C9F000BC000020BA00002058040020BD00002028
:10CA000070B504460D46E1B2FA4810F00DFC00BFC7
:10CA1000F848008800F080000028F9D0204670BD5A
:10CA2000F5480078012808D1F4480078012804D19D
:10CA30000020F249087001200871704710B50446C3
:10CA400054B94FF40051EE4810F03FF84FF48071A4
:10CA5000EC4810F03CF809E04FF40051E84810F0C1
:10CA600036F84FF48071E74810F02FF810BD10B57C
:10CA7000E548C079012855D1E448007807284FD20D
:10CA8000DFE800F00408374E4E1F20000020FBF7BF
:10CA900025FD46E00120FBF721FDDD48007830B997
:10CAA0006420DC4948830120D949087008E0D8484F
:10CAB0000078FF2804D10020D4490870D4490870B8
:10CAC0002FE000BF0120FBF709FDD148007830B905
:10CAD0003220D04948830120CD49087008E0CC4875
:10CAE0000078FF2804D10020C8490870C8490870A0
:10CAF00017E00120FBF7F2FCC548007830B9C820E8
:10CB0000C44948830120C249087008E0C048007841
:10CB1000FF2804D10020BD490870BD49087000E01D
:10CB200000BF05E00020FBF7D9FC0020B8490870E1
:10CB300010BD10B504461CB9FE20FBF7BFFD16E082
:10CB4000012C03D10120FBF7B9FD10E0022C03D129
:10CB50000820FBF7B3FD0AE0032C03D1EF20FBF71D
:10CB6000ADFD04E0052C02D10420FBF7A7FD10BDAC
:10CB700010B5A548C079012805D1A74800780B2831
:10CB800001D0FBF7DAFDA048C079012870D19B489D
:10CB900090F836000128F9D19F4800780B2868D218
:10CBA000DFE800F0068F8F2D2E8F8F8F0D4E6F00D8
:10CBB0000020FFF7BEFF0B209749087082E08F48E6
:10CBC000007E012805D100208C49C875FFF7B1FF10
:10CBD00078E08A48C07D01280AD10220FFF7A9FF2A
:10CBE00002208649C8754FF47A708A49888305E027
:10CBF0008248C07D10B90020FFF79BFF62E000BFB4
:10CC00007E48007E012805D100207C49C875FFF7C9
:10CC100090FF57E07948C07D01280AD10220FFF734
:10CC200088FF02207549C87542F2107079498883DF
:10CC300005E07248C07D10B90020FFF77AFF41E09F
:10CC40006E48007E012805D100206C49C875FFF7A9
:10CC500070FF37E06948C07D01280BD1FFF769FFFD
:10CC600002206649C8754FF47A706A49888307E0E4
:10CC700029E026E06148C07D10B90020FFF759FF88
:10CC800020E05E48007E012805D100205B49C87580
:10CC9000FFF74FFF16E05948C07D01280AD1052053
:10CCA000FFF747FF02205549C8754FF47A7059497C
:10CCB000888305E05148C07D10B90020FFF739FF97
:10CCC00000E000BF02E00020FFF733FF10BD10B509
:10CCD0004A4890F82700012804D0484890F82800D6
:10CCE000012803D10120FBF708FC02E00020FBF73C
:10CCF00004FC10BD10B5414890F82400012822D151
:10CD00004648007801280DD141023D480FF0DDFE74
:10CD10004FF480713A480FF0DAFE022138480FF0E4
:10CD2000D6FE10E03D48007868B94FF400713448F1
:10CD30000FF0CDFE4FF4807131480FF0C8FE022194
:10CD40002F480FF0C4FE364890F82D00072804D075
:10CD5000334890F82D00042811D13248407A042835
:10CD600004D04FF4007126480FF0B1FE4FF48071EB
:10CD700023480FF0ACFE022121480FF0A8FE1F4807
:10CD800090F82100012802D1FBF732FC06E01B4895
:10CD900090F8210010B90020FBF72AFC10BD10B557
:10CDA0002148007830B1012808D0022844D0FF285B
:10CDB0007AD178E000201D49087076E01C480078A0
:10CDC0000D2803DB0220194908700AE01848007892
:10CDD000012803DB01201549087002E000201349F7
:10CDE00008700020124908700F490870012011498D
:10CDF00008705AE000380140C0000020A003002065
:10CE0000000C014000080140FE0400204E000020FC
:10CE10004D000020E00300204F000020DC00002037
:10CE200058040020B012002008000020100000204C
:10CE300018000020E9000020FC480078401CFB4955
:10CE4000087008460078012809D1F948007818B11F
:10CE5000F7480078FF2802D10520F6490870F3480A
:10CE600000780D2803DB0220F349087006E0EF4844
:10CE70000078052802DB0020F0490870EB480078B4
:10CE8000FF2802D10D20E9490870FF20EC49087005
:10CE90000120EC4981F8210043F69820EA49A1F8E5
:10CEA000480002E000E000E000BF00BFE448007975
:10CEB00030B1012808D002281FD0FF2846D144E015
:10CEC0000020DD49087142E0D84800790D2803DBD5
:10CED0000220D94908710AE0D4480079012803DB0F
:10CEE0000120D549087102E00020D34908710020D3
:10CEF000CE490871D249087129E0CC480079401C1C
:10CF0000CA49087108460079012809D1C848007843
:10CF100018B1C7480078FF2802D10520C54908701C
:10CF2000C24800790D2803DB0120C549087102E0E1
:10CF3000FF20C34908710120C24981F8210043F64E
:10CF40009820C149A1F8480001E000E000BF00BFFF
:10CF5000BB48407830B1012808D002281FD0FF28F4
:10CF600046D144E00020B449487042E0AF484078E0
:10CF70000D2803DB0220B04948700AE0AB48407836
:10CF8000012803DB0120AC49487002E00020AA49D7
:10CF900048700020A5494870A949487029E0A34875
:10CFA0004078401CA149487008464078012809D1C2
:10CFB0009F48007818B19E480078FF2802D10520CC
:10CFC0009C490870994840780D2803DB01209C4952
:10CFD000487002E0FF209A4948700120994981F881
:10CFE000210043F698209849A1F8480001E000E0AC
:10CFF00000BF00BF9248807930B1012808D00228D4
:10D0000028D0FF2861D15FE000208B4988715DE066
:10D010004FF400518D480FF03EFDD0B184480078A8
:10D02000B8B9824880790D2803DB012082498871D4
:10D030000AE07E488079012803DB01207E4988715F
:10D0400002E000207C4988710020784988717C4981
:10D0500088713BE075488079401C74498871764836
:10D060008079042804D100208871754988712AE0EC
:10D070006E48807901280AD16D48007818B16C4853
:10D080000078FF280CD105206A49087008E067483D
:10D0900080790D2803DB02206749887100E000BF1A
:10D0A00062488079FF2802D10D2060498871FF20F5
:10D0B000634988710120634981F8210043F6982073
:10D0C0006149A1F8480001E000E000BF00BF5C48F2
:10D0D000C07930B1012808D0022825D0FF2861D1BD
:10D0E0005FE000205449C8715DE04FF480715748FB
:10D0F0000FF0D1FCB8B14D48C0790D2803DB0220F8
:10D100004D49C8710AE04948C079012803DB012074
:10D110004949C87102E000204749C87100204349CD
:10D12000C8714749C8713EE04048C079401C3F493A
:10D13000C8710846C07901281ED13D48007818B151
:10D140003B480078FF2817D13E48407E012803D095
:10D150000520384908700FE03A48407E01280BD17D
:10D160003848007E012804D0394890F82D00042862
:10D1700002D105202F4908702C48C0790D2803DB07
:10D1800001202F49C87102E0FF202D49C8710120FC
:10D190002C4981F8210043F698202B49A1F848003A
:10D1A00001E000E000BF00BF2548807830B10128D1
:10D1B00008D0022821D0FF2875D173E000201E4935
:10D1C000887071E0194880780D2803DB02201A4925
:10D1D00088700CE015488078012805DB012016498D
:10D1E00088701C49887002E0002013498870002074
:10D1F0000E4988701249887056E00F4880780428DC
:10D2000005D10020094988700D49887048E0074819
:10D210008078012820D10648007818B104480078A9
:10D22000FF282AD105200349087026E018000020B5
:10D230004D0000204E00002010000020E9000020DA
:10D2400008000020A0030020E00300200018014097
:10D250005804002020000020FA4880780D2803DBC5
:10D260000220F949887008E0F6488078052804DB38
:10D270000120F5498870F5498870F2488078FF28C8
:10D2800002D10D20EF498870FF20F14988700120FC
:10D29000F04981F8210043F69820EF49A1F84800B1
:10D2A00002E000E000E000BF00BFE948C07830B114
:10D2B000012808D0022821D0FF2862D160E0002098
:10D2C000E149C8705EE0DF48C0780D2803DB02202A
:10D2D000DD49C8700CE0DB48C078012805DB01207F
:10D2E000D949C870D949C87002E00020D649C87031
:10D2F0000020D449C870D649C87043E0D148C078EE
:10D30000401CD049C870D048C078042804D10020FF
:10D31000C870CF49C87032E0CA48C07801280AD125
:10D32000CE48007818B1CD480078FF2814D10520E8
:10D33000CB49087010E0C348C0780D2803DB0220F9
:10D34000C149C87008E0BF48C078052804DB012047
:10D35000BD49C870BD49C870BA48C078FF2802D11D
:10D360000D20B849C870FF20B949C8700120B949DB
:10D3700081F8210043F69820B749A1F8480001E060
:10D3800000E000BF00BFB248407930B1012808D0AA
:10D3900002281FD0FF2858D156E00020AA49487122
:10D3A00054E0A84840790D2803DB0220A6494871C3
:10D3B0000AE0A4484079012803DB0120A249487112
:10D3C00002E00020A049487100209E494871A04910
:10D3D00048713BE09B484079401C9A4948719A4803
:10D3E0004079042804D100204871994948712AE005
:10D3F0009448407901280AD19848007818B1974894
:10D400000078FF280CD105209549087008E08D4868
:10D4100040790D2803DB02208B49487100E000BFF2
:10D4200088484079FF2802D10D2086494871FF20A5
:10D43000874948710120874981F8210043F69820E7
:10D440008549A1F8480001E000E000BF00BF7E4828
:10D450008079022836D100207B4988718148007884
:10D4600008282FD07F48007809282BD07948007EE3
:10D4700060B900207749C8750120087605F0D1FB16
:10D480000020734988716F4988711BE07148007EE4
:10D49000012817D100206F49087605F0C2FB002053
:10D4A0006E4908706F4800780D2803D10020694943
:10D4B000C87502E001206749C87500206449887179
:10D4C00060498871674800780A2807D06548007865
:10D4D0000B2803D0634800780E2826D15A4840799B
:10D4E000022822D10020584948715A4890F820005B
:10D4F00030B90120574981F8200005F048FB05E0CC
:10D500000020544981F8200005F041FB01205149D9
:10D5100081F8390047F230504F49088300204D49C7
:10D5200048744B4948714749487110BD10B50020F7
:10D53000FBF776F80020FAF7D1FF0020FAF7DDFFBD
:10D540000020FBF755F80020FFF7F3FA4648407A31
:10D55000042804D1002044494872444908703D48D9
:10D56000C07F50B902203B49C87742F210703A4957
:10D57000886001203749887009E03648C07F01285B
:10D5800005D107203A4981F82E00FAF745FF10BD72
:10D5900001203349087000203049087001203549C6
:10D5A000087030490870344908700C20304981F8FF
:10D5B0002D00704710B52748807F012819D12948D0
:10D5C00000781D2808D10720294981F82D0081F80D
:10D5D0002E00FAF721FF0CE00120264908700720F1
:10D5E000234981F82D002220234908701E201D495F
:10D5F000087010BD10B5174890F82E0001280FD103
:10D600000A201E4908704FF400711D480FF05DFAA2
:10D610004FF4FA701B49088006200E4981F82E004D
:10D6200010BD012804D0022832D003285FD145E084
:10D630004FF46161144A116011460968134A116080
:10D6400056E00000180000201000002020000020FC
:10D6500008000020A0030020E00300204D0000206F
:10D660004E000020C0000020B0120020DC0000208E
:10D67000580400204B000020EC0000204F00002048
:10D68000000C0140D0000020C4000020C800002091
:10D69000FE49C98831B90021FD4A1160FD49FE4AA1
:10D6A00011600AE0F949C988FC4A92FBF1F1F84A95
:10D6B000116011460968F84A116019E0F849C989F2
:10D6C00031B90021F24A1160F249F34A11600DE0CC
:10D6D000F349C98901EB81014900F04A92FBF1F15C
:10D6E000EB4A116011460968EB4A116000E000BF87
:10D6F00000BFE749096829B10221EA4A1170EA4AE4
:10D70000517305E00021E74A11700121E64A517387
:10D71000704710B5E44890F82500012812D1002088
:10D72000E14981F82500E14890F82E00FF2809D052
:10D73000DF48007800B110BD0A20DC4981F82E00D6
:10D740000DF074FF00BFF6E710B5D748807B0128C5
:10D7500002D00CF0F1FC38E0D6480079022814D150
:10D76000D4488078022810D10420D2498870012042
:10D77000D14908701A20D14908701F20D04908707B
:10D780000920CA4981F82D001FE0C5484079E0B959
:10D79000C8480078022818D10120C749087009201C
:10D7A000C24981F82D0041F28830C649C882022062
:10D7B000C24908700920C24908700020B9490870A0
:10D7C0000120B94948730020087310BD10B5B9484D
:10D7D000007801280BD1B84908700320B7490870B8
:10D7E0000220B749087041F28830B649C882B14872
:10D7F0008078012855D10320AE49887041F28830E5
:10D80000B049C882B048008818B90020AF490870F4
:10D8100029E0AE480078AC490988884205DAAB486F
:10D820000078401CA94908701DE00120A749087034
:10D83000A54800880A2816DDA548008828B9A5480B
:10D840000078401EA449C87604E0A1480078401E34
:10D85000A149C876FDF7FDFC02209849087009200F
:10D860009749087010BD9C48C07E002805DD9A4885
:10D87000C07E401E9849C8760BE09648008818B9CB
:10D8800000209549C87604E092480078401E9249ED
:10D89000C876FDF7DEFC0220884908700920884917
:10D8A00008708448C07801284AD103208149C87093
:10D8B00041F288308349C8828348008818B9002023
:10D8C000824908701DE081480078012805DD7F4805
:10D8D0000078401E7D49087013E07B4800787B4942
:10D8E0000870794800880A280BDD00207A49C8763C
:10D8F000FDF7AFFC022071490870092070490870DB
:10D90000B0E77448008818B900207349C8760FE062
:10D910007148C17E6F480088401E814205DA6E481A
:10D92000C07E401C6C49C87602E000206A49C87677
:10D93000FDF78FFC022061490870092060490870DA
:10D940005C48007902280CD101205B49087007204F
:10D95000564981F82D002220594908701E20574948
:10D96000087000BF7EE753480078012807D152496C
:10D9700008700420514908700320514908704D482F
:10D98000007902280CD101204B4908700720474933
:10D9900081F82D0022204A4908701E20474908704E
:10D9A0007047414890F82E0030B902203E4981F876
:10D9B0002E004A484349C8653E48007801280BD1EB
:10D9C0003D49087007203D49087006203C49087011
:10D9D0000020354981F82E003648807802284CD145
:10D9E0000420344988703E4800883E4908803C48FD
:10D9F000807888703A48C078C870394800790871D2
:10DA00003748407948713648807988713448C07900
:10DA1000C871084680780D281DD2DFE800F01C0789
:10DA200011081509160A0B170C180D0000BF00BFCE
:10DA300000BF00BF00BF00BF1F202B4908700EE0D1
:10DA40001D20294908700AE000BF00BF00BF1E204A
:10DA50002549087003E01E202349087000BF00BF5D
:10DA60000120154908700520144908700420144944
:10DA7000087000200C4981F82E000E480079022819
:10DA80003DD101200C49087007202FE0E40400205C
:10DA9000C4000020407E0500C800002080EE360053
:10DAA000FE04002028000020A003002058040020CD
:10DAB0004D000020100000204B000020C00000207E
:10DAC000EC000020E0030020A2000020E80000207D
:10DAD0009E0000209C0000209409002040771B003D
:10DAE0002A0000203A00002032000020FC4981F882
:10DAF0002D002220FB4908701E20FB49087070474A
:10DB000010B5FA4890F82E0030B90220F74981F894
:10DB10002E00F748F749C865F7480078012859D121
:10DB2000F648007806284FD2DFE800F04E030A11CD
:10DB3000171E0220F14908700420EA49087044E0E9
:10DB40000320EE4908700420E64908703DE00420F7
:10DB5000EA490870E349087037E00520E749087092
:10DB60000420E049087030E0E5480088E549088075
:10DB7000E34880788870E248C078C870E04800794F
:10DB80000871DF4840794871DD488079887100204C
:10DB9000C8710DF0BBFF0120D8490870DA49087040
:10DBA0000020DA49087041F28830D249C882032047
:10DBB000CC4908700420CC4908700020D449087072
:10DBC0000220D449087000E000BF00BF0020C74910
:10DBD00081F82E00C8484078012803D0C6488079D3
:10DBE00001285AD10020C14981F82E00C34800788D
:10DBF000062850D2DFE800F04F03343B4249C048CA
:10DC00000088C0490880BE4880788870BC48C078C9
:10DC1000C870BB4800790871B94840794871B84864
:10DC200080798871B648C079C8710DF06FFF012006
:10DC3000B2490870B44908700020B449087041F234
:10DC40008830AC49C8820320A64908700420A64940
:10DC500008700020AE4908700220AE4908701BE031
:10DC60000120A649087004209E49087014E0022093
:10DC7000A249087004209B4908700DE003209F49C9
:10DC8000087004209749087006E004209B4908703A
:10DC90009449087000E000BF00BF974880780128D1
:10DCA00003D095488078022876D103209249887065
:10DCB00000208E4981F82E009048007806286CD20A
:10DCC000DFE800F0B603095398A48D480088401C93
:10DCD0008B490880ADE08A488078401C884988706C
:10DCE000084680780C2801DD0120887084488078FF
:10DCF0000D282AD2DFE800F0290711082209230A9B
:10DD00000B240C250D0000BF00BF00BF00BF00BFEB
:10DD100000BF1F20804908701BE079490888C1179F
:10DD200000EB91718910A0EB810119B11C207A4997
:10DD3000087002E01D20784908700AE000BF00BFAB
:10DD400000BF1E207449087003E01E20724908704D
:10DD500000BF00BF6A48C0786F490978884203DD78
:10DD60006D4800786649C87063E0654880780D2882
:10DD70002CD2DFE800F02B0713082409250A0B2614
:10DD80000C270D0000BF00BF00BF00BF00BF00BFD9
:10DD90001F20614908701DE052E049E05849088899
:10DDA000C11700EB91718910A0EB810119B11C2002
:10DDB0005949087002E01D20574908700AE000BF69
:10DDC00000BF00BF1E205449087003E01E205249C6
:10DDD000087000BF00BF4A48C078401C4849C8705E
:10DDE0000846C0784C490978884202DD0120444940
:10DDF000C8701EE042484079401C414948710846BD
:10DE00004079172801DD0020487112E03C488079F4
:10DE1000401C3B498871084680793B2801DD002081
:10DE2000887103202F49087004202F49087000E0F2
:10DE300000BF00BF05202C49087004202949087044
:10DE40002D48C078012803D02B48C078022846D13D
:10DE500003202949C8700020244981F82E00274852
:10DE60000078062875D2DFE800F0D4030975B8C63B
:10DE700023480088401E22490880CBE02048807853
:10DE8000012803DC0C201E49887004E01C488078BF
:10DE9000401E1B4988701A4880780D2849D2DFE857
:10DEA00000F0480711084109420A0B430C440D00D9
:10DEB00000BF00BF00BF00BF00BF00BF1F2016494A
:10DEC00008703AE00E490888C11700EB917189107B
:10DED000A0EB810111B31C200F49087021E0A0E0E4
:10DEE00058040020EC000020C0000020A003002007
:10DEF00040771B00E00300201000002038000020C5
:10DF00003A0000202A0000204B000020C200002020
:10DF1000500000204E000020320000201D20FE494D
:10DF200008700AE000BF00BF00BF1E20FA49087059
:10DF300003E01E20F849087000BF00BFF748C07812
:10DF4000F5490978884203DDF3480078F349C87041
:10DF500060E05EE0F14880780D282AD2DFE800F02A
:10DF6000290711082209230A0B240C250D0000BFE4
:10DF700000BF00BF00BF00BF00BF1F20E649087000
:10DF80001BE0E6490888C11700EB91718910A0EBEE
:10DF9000810119B11C20E049087002E01D20DE4912
:10DFA00008700AE000BF00BF00BF1E20DA490870F9
:10DFB00003E01E20D849087000BF00BFD748C078D2
:10DFC000012804DCD4480078D449C87004E0D34860
:10DFD000C078401ED149C8701CE0D0484079002864
:10DFE00003DC1720CD49487104E0CC484079401E3D
:10DFF000CA4948710EE0C9488079002803DC3B20FB
:10E00000C649887104E0C5488079401EC3498871BB
:10E0100000E000BF00BF0520C14908700420C149CD
:10E020000870C148007902280CD10120BF4908704E
:10E030000720BF4981F82D002220BA4908701E2010
:10E04000B749087010BD30B500210022B64B1B78CF
:10E05000012B53D1B74B1B78072B4DD2DFE803F0D0
:10E060004C0405060708140000BF00BF00BF00BF36
:10E07000B04B1B785B1CAF4C23700623A84C23705D
:10E080000523A84C237038E00123AA4C23700020FC
:10E0900009E0A94B1B5CA94C245CA34201D00121DF
:10E0A00003E0431CD8B20328F3DB00BF71B901239E
:10E0B0009E4C237008239A4C23709A4C23700023A3
:10E0C0009F4C237002239F4C23700BE00623944C3B
:10E0D00023700523934C237003239B4C237001234F
:10E0E0009A4CE375944B1B7803EB83035A00924BD5
:10E0F0005B781344DAB200E000BF00BF8A4B5B7864
:10E10000012B1FD18B4B1B78072B13D2DFE803F0B9
:10E11000120408090A0B0C000123864C23700AE044
:10E1200000BF00BF00BF00BF824B1B785B1E814C4D
:10E13000237000E000BF00BF0623794C2370052345
:10E14000784C2370784B9B78012B03D0764B9B78CF
:10E15000022B4CD10323744CA370764B1B78072BF6
:10E160003DD2DFE803F03C0405062021220000BF79
:10E1700000BF704B1B785B1E6F4CE35C092B0BDA06
:10E180006C4B1B785B1EE35C5B1CDCB2694B1B7841
:10E190005B1E694DEC5405E00024664B1B785B1E4A
:10E1A000654DEC541CE000BF00BF624B1B781B1F89
:10E1B000624CE35C092B0BDA5E4B1B781B1FE35CA4
:10E1C0005B1CDCB25B4B1B781B1F5C4DEC5405E009
:10E1D0000024584B1B781B1F584DEC5400E000BF27
:10E1E00000BF06234E4C237005234E4C23704E4B2C
:10E1F000DB78012B03D04C4BDB78022B4CD1032373
:10E20000494CE3704B4B1B78072B3DD2DFE803F002
:10E210003C0405062021220000BF00BF454B1B78AF
:10E220005B1E454CE35C002B0BDD424B1B785B1EF9
:10E23000E35C5B1EDCB23F4B1B785B1E3E4DEC5437
:10E2400005E009243B4B1B785B1E3B4DEC541CE066
:10E2500000BF00BF374B1B781B1F384CE35C002B03
:10E260000BDD344B1B781B1FE35C5B1EDCB2314BB8
:10E270001B781B1F314DEC5405E009242D4B1B78F6
:10E280001B1F2E4DEC5400E000BF00BF0623244CA2
:10E2900023700523234C2370234B1B79022B0CD1B5
:10E2A0000123224C23700723214C84F82D30222394
:10E2B0001C4C23701E231A4C237030BD234890F849
:10E2C0002E0030B90220214981F82E002048214932
:10E2D000C86515480078012866D100201B4981F8DF
:10E2E0002E001D480078012806D106200D4908702F
:10E2F00002201949087057E01848C07858B91348E7
:10E3000090F8340001283DD108490870124908707E
:10E310000820074924E03FE0320000203A000020B6
:10E32000C0000020EC000020100000204B00002066
:10E3300058040020F2000020420000204500002088
:10E34000500000204E0000204F000020A0030020BD
:10E3500040771B00E003002098040020FE0400200A
:10E3600081F82D000020FC4908704FF47A70FB49B9
:10E3700088600820FA490870FA4908700120FA49B3
:10E38000087011E00120F84908702020F449087055
:10E390002620F449087007E00120F449087008209D
:10E3A000EF490870EF490870F1484078012803D020
:10E3B000EF488079012811D10020EE4981F82E0024
:10E3C000E9480078022806D10620E64908700120B5
:10E3D000E549087002E00120E3490870E4488078CC
:10E3E000022812D10420E24988700020E14981F816
:10E3F0002E000120DD4908701C20D9490870212019
:10E40000D84908700120DC490870D94800790228F1
:10E410000CD10120D54908700720D84981F82D007A
:10E420002220D04908701E20CD490870704770B571
:10E43000D04890F82E0030B90220CE4981F82E0045
:10E44000CF48C649C865CA48007801287DD1002058
:10E45000C84981F82E00C4480078012802D002285B
:10E4600074D15DE0C7488078C349097888420BDDE4
:10E47000C1480078401CC04908701C20B849087089
:10E480002120B849087046E00021B74A9160D16068
:10E4900000241AE0B448D0E90231BB48005D1818E6
:10E4A00041F10001B04AC2E902011046D0E9022060
:10E4B0000A210023A2FB015600FB016002FB0300BE
:10E4C000A949C1E90250601CC4B2AE488078401E20
:10E4D000A042DFDCA448D0E90231AB48005D181847
:10E4E00041F10001A04AC2E90201FDF7CDFD07207C
:10E4F0009B49087006209B49087002209A490870C1
:10E5000001209D4908709949087000209F490870B2
:10E5100002209F4908700120964981F834007AE072
:10E52000984800789749497808449349097888427F
:10E530000DDD91480078401C8F4908701C208849E7
:10E54000087021208749087063E065E062E00020E0
:10E5500085494880002413E0834841888A48801F09
:10E56000005D0844804948800846408800EB8000F0
:10E570004FF6FF7101EA40007B494880601CC4B23D
:10E5800080480078401EA042E6DC774841887E48FB
:10E59000801F005D08447449488000208880002462
:10E5A00013E0714881887848C01E005D08446E49B8
:10E5B00088800846808800EB80004FF6FF7101EAF2
:10E5C000400069498880601CC4B26E484078401E93
:10E5D000A042E6DC644881886B48C01E005D0844A8
:10E5E00061498880FDF750FD07205D4908700620CD
:10E5F0005C49087001206049087002205A4908707F
:10E6000001205A49087000206049087002206049C2
:10E61000087000E000BF00BF55484078012803D0D3
:10E620005348807901286FD10020524981F82E008B
:10E630004D480078012802D002287DD15BE04E4889
:10E640000078012847D10021474A9160D160002419
:10E650001AE04548D0E902314B48005D181841F1F5
:10E660000001414AC2E902011046D0E902100A2223
:10E670000023A1FB025600FB026001FB03003A49A4
:10E68000C1E90250601CC4B23E488078401EA042DE
:10E69000DFDC3548D0E902303B49095D591840F1CB
:10E6A0000000314AC2E90210FDF7EEFC07202C49B8
:10E6B000087006202B49087002202B4908700120A1
:10E6C0002D4908702949087000203049087002203F
:10E6D0002F4908700AE028480078401E2649087033
:10E6E0001C201F49087021201E4908700120214963
:10E6F00081F8340094E02048007801287ED1002081
:10E7000019494880002414E08BE0174841881E48CE
:10E71000801F005D0844144948800846408800EB8B
:10E7200080004FF6FF7101EA40000F494880601CED
:10E73000C4B21448007800E071E0401EA042E4DC5E
:10E74000094841881048801F005D084406494880F8
:10E7500000208880002430E0E4000020E003002056
:10E76000C0000020EC000020980400204B00002096
:10E7700010000020A0030020F20000205804002018
:10E7800040771B00FE040020C6040020500000203B
:10E790004E000020F8488188F848005D0844F6499A
:10E7A00088800846808800EB80004FF6FF7101EA00
:10E7B0004000F1498880601CC4B2F1484078401E96
:10E7C000A042E7DCEC488188EC48005D0844EA4957
:10E7D0008880FDF759FC0720EA4908700620EA49BD
:10E7E00008700120E94908700220E34908700120FF
:10E7F000E74908700020E749087000E003E00220C4
:10E80000E54908700AE0E1480078401EDF490870D9
:10E810001C20DC4908702120DB49087000E000BFA3
:10E8200000BFDE488078012803D0DC4880780228C9
:10E8300079D10320D94988700020D94981F82E0068
:10E84000CD480078012802D0022864D11AE0CF48D0
:10E850000078401EC949C91C085C09280ADACB485F
:10E860000078401E085C401CC2B2C8480078401EB8
:10E870000A5406E00022C5480078401EBF49C91C62
:10E880000A5449E0BE480078C049097888421ADB3A
:10E89000BE480078401EB949C91E085C09280ADA3A
:10E8A000BA480078401E085C401CC2B2B7480078E5
:10E8B000401E0A542DE00022B4480078401EAF49A3
:10E8C000C91E0A5425E0AE480078B0490978081AF4
:10E8D000401EAA49085C092812DAA9480078AB4909
:10E8E0000978081A401EA549085C401CC2B2A44819
:10E8F0000078A6490978081A401EA0490A5408E081
:10E9000000229F480078A1490978081A401E9B49B7
:10E910000A5401E007E000BF00BF1C2099490870BD
:10E920002120994908709D48C078012803D09B4850
:10E93000C078022879D103209849C87000209849EE
:10E9400081F82E008C480078012802D0022864D17A
:10E950001AE08E480078401E8849C91C085C0028CF
:10E960000ADD8A480078401E085C401EC2B2874813
:10E970000078401E0A5406E0092284480078401EB0
:10E980007E49C91C0A5449E07D4800787F490978CE
:10E9900088421ADB7D480078401E7849C91E085C11
:10E9A00000280ADD79480078401E085C401EC2B28B
:10E9B00076480078401E0A542DE0092273480078FA
:10E9C000401E6E49C91E0A5425E06D4800786F4903
:10E9D0000978081A401E6949085C002812DD684859
:10E9E00000786A490978081A401E6449085C401E8C
:10E9F000C2B26348007865490978081A401E5F4929
:10EA00000A5408E009225E48007860490978081A2B
:10EA1000401E5A490A5401E007E000BF00BF1C2015
:10EA2000584908702120584908705C48007902282C
:10EA30000CD101205649087007205A4981F82D0051
:10EA40002220514908701E204E49087070BD54485C
:10EA500090F82E0030B90220514981F82E0052481A
:10EA60005249C8654D488079012803D04B48407809
:10EA700001280FD100204A4981F82E000120444985
:10EA8000087007203F49087006203F4908700120A0
:10EA9000394908704148007902280CD101203C49CD
:10EAA000087007203F4981F82D0022203649087060
:10EAB0001E2034490870704710B5394890F82E0070
:10EAC00030B90220364981F82E0037483749C865E9
:10EAD0000220334981F82C003548344988652F4895
:10EAE000007801286AD13348007801287ED10320BC
:10EAF0002A49087000202A4981F82E002E48007803
:10EB000050BB1E481B380078072823D2DFE800F0EE
:10EB1000220409130E181D00022018491B39087021
:10EB200019E0042015491B39087014E0032013492B
:10EB30001B3908700FE0052010491B3908700AE0E6
:10EB400006200E491B39087005E001200B491B39CE
:10EB5000087000E000BF44E008481B380078801EC1
:10EB600005283CD2DFE800F0032F2B3337000420C8
:10EB700002491B39087033E098040020C3040020C8
:10EB8000FE040020C0000020EC000020F200002065
:10EB90004B000020500000204E00002010000020FC
:10EBA000A00300205804002040771B00E003002051
:10EBB00080EE3600E9000020E600002016E0032089
:10EBC000FE4908700CE00520FC49087008E00620AA
:10EBD000FA49087004E00220F849087000E000BF1C
:10EBE00000BF0820F6490870F6490870F64800781A
:10EBF00002285CD10020F54981F82E00084690F8E3
:10EC00003300012853D1F248007818BBEB48007854
:10EC100007281DD2DFE800F01C0408100C141800AF
:10EC20000220E649087014E00420E449087010E06E
:10EC30000320E24908700CE00520E049087008E074
:10EC40000620DE49087004E00120DC49087000E07D
:10EC500000BF1FE0D9480078801E052818D2DFE8E1
:10EC600000F0030B070F13000420D449087010E0D4
:10EC70000320D24908700CE00520D049087008E054
:10EC80000620CE49087004E00220CC49087000E05C
:10EC900000BF00BF0020CD4981F833004FF4FA7067
:10ECA000CC4948600820C6490870C6490870C64863
:10ECB000807901284FD10020C44981F82E00C44832
:10ECC000007818BBBD48007807281DD2DFE800F0A7
:10ECD0001C0408100C1418000620B849087014E031
:10ECE0000120B649087010E00220B44908700CE019
:10ECF0000420B249087008E00320B049087004E01D
:10ED00000520AE49087000E000BF1FE0AB48007866
:10ED1000801E052818D2DFE800F0030B070F130050
:10ED20000620A649087010E00220A44908700CE0F3
:10ED30000420A249087008E00320A049087004E0FC
:10ED400005209E49087000E000BF00BF08209C49D4
:10ED500008709C4908709C48407801287DD19E49E4
:10ED60000870FDF791F9F9F77FFF01209B490870C2
:10ED700000209B4908709B4908809B4908709B496B
:10ED8000087001209A4908709A48407C18B944F6E6
:10ED90002060904988608948408D68B10120FEF765
:10EDA00040FC0120944981F82D000B208549087012
:10EDB0000A20834908700CE00220FEF732FC022092
:10EDC0008D4981F82D000C207E4908700B207C496C
:10EDD0000870002089494873894908708649C883AA
:10EDE00042F2D0007B49088586480068C86200204E
:10EDF00081490881754948767F49C88248830883DC
:10EE0000888301208049087000208049087080486C
:10EE10007049086200207849C88401206B4981F854
:10EE200026000020487447F230506A4908830020C9
:10EE300066494875C87476486649086242F210709F
:10EE4000886001207349087000207349087002200F
:10EE50007249087000205D4900E001E081F82E0051
:10EE600059488078012803D057488078022874D107
:10EE70000320554988700020544981F82E004F48DE
:10EE8000007807287FD2DFE800F07E041422446077
:10EE900070004A48008D40F2E731884203DB0020D1
:10EEA0004649088504E04548008D401C43490885D3
:10EEB0006AE04248408D322803DB00203F49488504
:10EEC00004E03E48408D401C3C4948855CE03B489E
:10EED000808D642805DA3948808D401C3749888543
:10EEE00016E03648808DB0F5FA7F09DA3348808D18
:10EEF000642805DB3148808D0A303049888507E079
:10EF00002E48808DB0F5FA7F02DB00202B498885E2
:10EF10003AE02A48C08D642803DB00202749C885D1
:10EF200012E02648C08D3C2809DB2448C08D6428A7
:10EF300005DA2248C08D0A302049C88504E01F4800
:10EF4000C08D401C1D49C8851EE01C48008E6328EA
:10EF500005DB00201949088606E01BE013E017488E
:10EF6000008E401C154908860EE01448408E5A2831
:10EF700003DB01201149488604E01048408E401C04
:10EF80000E49488600E000BF00BF08200C49087009
:10EF90000C4908700C48C078012803D00A48C07892
:10EFA00002286ED103200849C8700020074981F863
:10EFB0002E0002480078072873D231E0A804002010
:10EFC000C0000020EC00002010000020A003002062
:10EFD000E6000020E0030020E5000020D90000202A
:10EFE000690100208E000020900000209100002088
:10EFF00010010020FE04002058040020B012002060
:10F00000E0000020C4000020F2000020A00000204A
:10F0100080EE36004B000020500000204E00002003
:10F02000DFE800F08004132148647200FE48008D80
:10F03000002804DC40F2E730FB49088504E0FA4888
:10F04000008D401EF84908856DE0F748408D002886
:10F0500003DC3220F449488504E0F348408D401E2B
:10F06000F14948855FE0F048808D64280ADCEE486D
:10F07000808D002806DDEC48808D401EEA49888599
:10F0800017E056E0E848808DB0F5FA7F0ADCE648E4
:10F09000808D642806DDE448808D0A38E249888541
:10F0A00007E03FE0E048808D18B94FF4FA70DE4980
:10F0B000888538E0DC48C08D002803DC6420DA490C
:10F0C000C88512E0D848C08D642809DCD648C08DB8
:10F0D0003C2805DDD448C08D0A38D349C88504E0F2
:10F0E000D148C08D401ED049C8851CE0CE48008E56
:10F0F000002803DC6320CC49088604E0CA48008E5F
:10F10000401EC94908860EE0C748408E012803DC2E
:10F110005A20C549488604E0C348408E401EC24973
:10F12000488600E000BF00BF0820C0490870C04901
:10F130000870C048007902280CD10120BE4908702F
:10F140000720BE4981F82D002220B94908701E20F1
:10F15000B6490870B7484079012815D1FCF794FFEB
:10F160000020B6490880B64908700920AF490870E8
:10F170000720AF4908700120B2490870AE490870F5
:10F180000020B14981F82E0010BD0620AB4981F85E
:10F190002D00AD4890F82E0030B90220AA4981F820
:10F1A0002E00AA48AA49C865A2484079022803D07F
:10F1B000A048407901281BD1A34890F83500B8B980
:10F1C0000120A14981F8350004209A4948710020A6
:10F1D0009D4981F82E0003209649487102209849E4
:10F1E000087000209549C8830880062081F82D000A
:10F1F00092480088142808D0934890F835000128D8
:10F2000027D18C484079012823D100208E4981F8EC
:10F21000350081F82E000320864988710820834933
:10F2200008700120844908700820814908708948C5
:10F230000078012803D102207B49087002E00120F8
:10F2400079490870FF207D4981F82D0000207E4912
:10F2500008737848807901281FD17B4890F83500E1
:10F26000D8B90020784981F82E0008206F4908702D
:10F2700001207149087008206D49087075480078B0
:10F28000012803D102206849087002E00120664984
:10F290000870FF20694981F82D00704718B50021DA
:10F2A000644A1278012A79D16B4A694B5A63654ADC
:10F2B0001278012A04D0022A0CD0032A6CD113E060
:10F2C0000222604B1A700D22584B1A700F22584BB5
:10F2D0001A7062E003225B4B1A700D22534B1A70B6
:10F2E0000F22534B1A7058E005228DF8002002229D
:10F2F0008DF8012000228DF80220002009E0574AF5
:10F30000125C1DF800309A4201D0012103E0421C3A
:10F31000D0B20328F3DB00BF01290FD100200AE09F
:10F320004E4A125C4E4B1B5C9A4201D0022104E013
:10F330000021421CD0B20328F2DB00BFE9B9012250
:10F34000404B1A70404B5A75464A12781E2A04D117
:10F3500007223A4B83F82D2003E00422374B83F831
:10F360002D20404A1278314B1A703F4A1278304BA8
:10F370001A700122304B1A700BE00322314B1A70C5
:10F380000D222A4B1A700F22294B1A7000222E4B85
:10F390005A7502E002E0FFE700BF00BF254A9279FC
:10F3A000012A03D0234A5278012A2AD12A4A284B1B
:10F3B0005A63244A1278012A17D0022A0BD0032A52
:10F3C0001DD102221F4B1A700D22184B1A700F22EA
:10F3D000174B1A7014E001221A4B1A700D22134BAE
:10F3E0001A700F22124B1A700AE00122154B1A7084
:10F3F0000D220E4B1A700F220D4B1A7000E000BF49
:10F4000000BF0C4A9278012A03D00A4A9278022A55
:10F4100055D10322074B9A700F4A0D4B5A63094A84
:10F420001278012A27D021E0A8040020C000002083
:10F43000EC000020100000204B00002058040020A9
:10F4400028000020F2000020A003002040771B00CD
:10F45000E0030020E600002020BF0200450000205D
:10F4600042000020D2000020EE000020022A03D03B
:10F47000032A1CD101E000BF00BFFE4A1278521ED1
:10F48000FD4B9A5C092A0BDAFA4A1278521E9A5CF2
:10F49000521CD3B2F74A1278521EF74CA35405E01F
:10F4A0000023F44A1278521EF34CA35400E000BF2C
:10F4B00000BF0D22F14B1A700F22F14B1A70F14A66
:10F4C000D278012A03D0EF4AD278022A32D103221D
:10F4D000EC4BDA70EC4AED4B5A63E64A1278012A9B
:10F4E00004D0022A03D0032A1CD101E000BF00BFD0
:10F4F000E04A1278521EE04B9A5C002A0BDDDD4A8E
:10F500001278521E9A5C521ED3B2DA4A1278521EF8
:10F51000D94CA35405E00923D64A1278521ED64C82
:10F52000A35400E000BF00BF0D22D44B1A700F227D
:10F53000D34B1A7018BD08B5D548407D01280AD1B3
:10F540000720D44981F82D001E20CC4908702220C4
:10F55000CB49087008BDCF484088B8B90120CE49D2
:10F5600008700220CB4981F82D000C20C449087096
:10F570000B20C24908700120C8490870C44890F89F
:10F580003200012801D1C64908705EE10020C2495D
:10F590000870BF48407C00287DD1BA4840780228D6
:10F5A0001CD147F23050B9490883BA4890F82D0071
:10F5B00001284FD1B6494873002008730B20B04989
:10F5C00008700420B34981F82D0042F21070AF4951
:10F5D00088600120AE4981F839003BE0A9484078B5
:10F5E000012837D147F23050A8490883A94890F83C
:10F5F0002D0004282ED10120AA4908700020AA4914
:10F6000008700120A94908700020A9490880A9496B
:10F610000870A94908700120FEF703F800209D49F1
:10F62000C88342F2D00099490885A4480068C8629E
:10F630000B20934908700A209049087001209549D1
:10F6400081F82D0042F210709049886001209049A5
:10F6500081F839008F4890F82D0004287ED1894820
:10F660000079022857D100208649087147F23050AE
:10F67000864908830120894908708648806B000EFE
:10F680008DF800008348806B000C8DF801008148E4
:10F69000008F000A00E0BDE08DF802007D4890F880
:10F6A00038008DF80300864A04216846FCF77AF991
:10F6B0008448007830B9FCF74FF9FBF786FF01204A
:10F6C00080490870FBF7F6FF7F488079C0B90D20AC
:10F6D0006A4908700F206A4908701E207B4908702B
:10F6E00022207B4908700A207A4908700B207A4949
:10F6F000087065486549486301205E49087029E73C
:10F700000720644981F82D001E205C4908702220E2
:10F710005B4908701EE75B48007802285DD1012034
:10F720006E49087002206E49087000205549087023
:10F7300047F230505549088301204E490870574917
:10F7400008705448806B000E8DF800005148806BA3
:10F75000000C8DF801004F48008F00E03DE0000AEA
:10F760008DF802004B4890F838008DF80300544A99
:10F7700004216846FCF716F95248007830B9FCF7C6
:10F78000EBF8FBF722FF01204E490870FBF792FFD0
:10F790004D488079C0B90D20384908700F2038498C
:10F7A0000870082049490870494908700A204949E9
:10F7B00008700B20484908700420364981F82D0054
:10F7C000314832494863C5E608202C4908702C4965
:10F7D000087004202F4981F82D00424880780128C4
:10F7E00033D14048C07801282FD1C1023E480DF0E6
:10F7F00052F950B300203B498870C8700120244959
:10F80000487447F23050214908830120204981F88B
:10F8100039001AE033488078012816D13148C07881
:10F82000012812D1C10230480DF035F968B100202D
:10F830002C498870C8701649487447F230501349F3
:10F8400008830120124981F839001248808C274929
:10F850004988884263DB00202549087001200C4953
:10F8600048730020087304202249087040F6C41031
:10F87000064941E0F200002045000020C0000020C1
:10F88000EC0000201000002020BF0200E003002058
:10F89000A003002058040020DB0000204B000020C3
:10F8A0000F0100201001002069010020D900002074
:10F8B0008E0000209000002091000020C400002055
:10F8C00000A00608A0000020FE040020D2000020B6
:10F8D000EE000020D3000020EF000020E600002012
:10F8E000A80400202000002000180140E4040020AB
:10F8F000280000204F000020A1F842000120FD490F
:10F9000081F824000E20FC4908701020FB49087083
:10F910000120F849C875FA490870FA49087000BF13
:10F9200018E608B5F348407D01280CD1F549087068
:10F930000720F54981F82D001E20EF49087022208C
:10F94000EE49087008BDF148407B012837D0F048E7
:10F950000078032821DBE74890F82C0001282ED1FD
:10F960000320EA49487342F21070EA498860022095
:10F97000E04981F82C00E548407B032809D10120AB
:10F98000E2494873DB4890F83200012801D1E2498E
:10F9900008700020DE49087011E0D64890F82C006D
:10F9A00068B9DB480078032809DADC48D94988655A
:10F9B0000320D04981F82C000020D5490870CD489B
:10F9C000407C002879D1D648407802283BD147F2C4
:10F9D0003050D0490883CC4890F82D00022813D12C
:10F9E0000C20C64908700420C74981F82D0042F256
:10F9F0001070C84988600120BE4948730020087310
:10FA0000012081F839006EE0BF4890F82D000328EE
:10FA100069D10C20B94908700120BA490870042046
:10FA2000B94981F82D0042F21070BA49886000206F
:10FA3000B549C8800120AF494873002008730120F0
:10FA400081F839004FE0B6488079012803D0B448E6
:10FA50004078012847D147F23050AE490883AA4880
:10FA600090F82D0004283ED10120AE4908700020F6
:10FA7000AD4908700120AD4908700020AC490880EC
:10FA8000A149C88342F2D000A2490885A94800686C
:10FA9000C862A9480078012802D09B48C08868B194
:10FAA0000020A54908700320A4490870FDF7B9FD9E
:10FAB0000320954981F82D000DE09FE10220FDF71C
:10FAC000B0FD0C208D4908700B208B490870022076
:10FAD0008D4981F82D000120864981F8390042F2D4
:10FAE00010708C49886096488078012818D1944815
:10FAF000C078012814D1C10292480CF0CCFF78B133
:10FB000000208F498870C87001207A49487447F2F4
:10FB10003050804908830120764981F8390029E076
:10FB20007F488078012825D17D48C07810BB03200C
:10FB30007B49887047F23050764908836D48807E53
:10FB400058B901206B49887681F8220081F823009A
:10FB500042F210706F4948870CE0002065498876B2
:10FB600081F8220042F210706A49488701206149F9
:10FB700081F82300644890F82D0004287ED168485D
:10FB80000078022865D101206F49087002206F4972
:10FB9000087000206249087047F230505D490883C0
:10FBA000012057490870574908705748806B000E6C
:10FBB0008DF800005448806B000C8DF8010052480D
:10FBC000008F000A8DF802004F4890F838008DF839
:10FBD00003005F4A04216846FBF7E4FE5D480078B5
:10FBE00030B9FBF7B9FEFBF7F0FC0120594908706A
:10FBF000FBF760FD5848807910BB0D203E49087026
:10FC00000F203E4908700820544908705449087074
:10FC10003D48C08830B10B2052490870232052491A
:10FC2000087005E00B204F4908700C204E49087001
:10FC30000420354981F82D004C483649486381E657
:10FC400008202D4908702D49087004202E4981F89C
:10FC50002D003348007902284AD10020304908712C
:10FC60002948806B000E8DF800002748806B000C3F
:10FC70008DF801002448008F000A00E094E08DF820
:10FC80000200214890F838008DF80300304A042122
:10FC90006846FBF787FE2F48007830B9FBF75CFE1B
:10FCA000FBF793FC01202B490870FBF703FD47F29B
:10FCB000305018490883012012490870264880797D
:10FCC000A8B90D200C4908700F200C4908701E209F
:10FCD000224908702220224908700B48C08840B190
:10FCE0000B202049087023201F49087046E050E08F
:10FCF00083E03DE0A0030020C0000020EC000020D5
:10FD0000F20000204B00002058040020B012002018
:10FD1000E0000020E00300200F01002080EE36000C
:10FD2000100000201001002069010020D9000020EF
:10FD30008E000020C4000020DD000020C100002053
:10FD40002000002000180140E6000020A804002048
:10FD500000A00608A0000020FE040020D200002021
:10FD6000EE000020D3000020EF00002020BF0200A2
:10FD70000B20F74908700C20F64908700420F6495A
:10FD800081F82D00F548F64948630120F5490870CF
:10FD9000D8E50720F04981F82D001E20F2490870AF
:10FDA0002220F2490870CDE5F148007802284DD1B3
:10FDB000E94890F82D00032848D047F23050E84930
:10FDC00008830020EB494874012048730020087321
:10FDD0000420E14981F82D0042F21070E04988606A
:10FDE0001620E14908701820E04908700120E24916
:10FDF0000870DC490870E149087027E0E048807825
:10FE0000012823D1DE48C07801281FD1C102DD4876
:10FE10000CF041FED0B10020D9498870C870D54996
:10FE2000487447F23050CE4908830120D14981F807
:10FE30003900D54800780C2802D1CC49087005E07B
:10FE4000D1480078232801D1C8490870C24890F8E9
:10FE50002D00042850D0C648C07901287CD100204C
:10FE6000C349C871C348407E012846D0C148C07C00
:10FE7000012842D0C548408988B30120BD49C874D3
:10FE80000320FDF7CEFB42F2D000B5490885C048FB
:10FE90000068C8620220BF4908702320B349087077
:10FEA0000120B64908700320AB4981F82D000846AF
:10FEB000008D401C0885B5484089C8800846008DE3
:10FEC000012802D1AB4981F82C00B348407B0128BE
:10FED00006D0B2480078401CB049087003E00CE03E
:10FEE0000020AE490870A34890F82C00032833D1B5
:10FEF0000120A04981F82C002EE09E48407E012878
:10FF00002AD19548408D401C934948850220A1493B
:10FF1000087001209749C8750846407E012806D11F
:10FF2000087781F8380041F288308D49C8878A48BF
:10FF300090F82D0003280CD123208C490870012053
:10FF40008C49887681F8220042F2107084494887F3
:10FF500002E00C20854908708648C07C012845D104
:10FF60007D48C088E0BB0120824948768748808967
:10FF700079490881854880894EF66021484378494F
:10FF8000C86000207B49C8740220FDF74AFB42F29A
:10FF9000D000734908857E480068C8620C20734908
:10FFA0000870012075490870724890F832000128E5
:10FFB00006D142F210706A498860012078490870C1
:10FFC000654890F82D00032803D076480078012872
:10FFD00007D10220604981F82D0000207149087086
:10FFE0001CE004205C4981F82D0017E06148C07CCA
:10FFF000A0B9594890F82D00042805D101205D4989
:020000040801F1
:1000000048730020087309E00220FDF70AFB6048EE
:1000100000685349C86202205649C8744E48808C13
:100020005A494988884222DB00205F490870012034
:1000300050494873002008730120C87504205B49AB
:10004000087040F6C4104649A1F842000120494911
:1000500081F824000E20444908701020434908709C
:1000600001204449C8753F4908704449087000BFE1
:1000700068E410B5384890F82D0001280ED03648B5
:1000800090F82D00022809D0334890F82D0003285D
:1000900004D0314890F82D00042837D105202E498E
:1000A00081F82D0001204249087008460078012897
:1000B00008D1002008702F4890F83200012801D1A3
:1000C0000AF064FE42F2107025498860002032492F
:1000D000C871012008723748007830B9FBF73CFC42
:1000E000FBF773FA012033490870334880783349AD
:1000F00008703148C07848702F48407988702E4881
:100100008079C87008200871FBF7D4FA1848007885
:10011000022863D11620144908701820134908706A
:100120000120154908700F49087014490870002013
:100130001E4908701848407A042841D140F6C4107E
:100140000749A1F8420001200A4981F8240045E04E
:10015000D3000020EF0000205804002020BF020040
:10016000E0030020F2000020C0000020EC0000208E
:1001700010000020A0030020480000204B000020B9
:100180002000002000180140ED000020E4040020C1
:10019000C40000204E000020B0120020E00000202B
:1001A0000F010020DE000020280000204F0000206A
:1001B000E7000020A00000202A00002033000020DB
:1001C0004FF40071F9480CF082FC40F6C410F84975
:1001D000A1F842000020F74981F82400F648007990
:1001E000022818D1FBF766FA0120F44908700720AD
:1001F000F34981F82D004FF49670ED498860002096
:10020000EC49C875EF4908702220EF4908701E209C
:10021000EE49087010BD00BFFCE7E74800780128F0
:1002200029D1EB48007807281DD2DFE800F01C0434
:10023000080C101418000220E549087014E003208F
:10024000E349087010E00420E14908700CE0052043
:10025000DF49087008E00620DD49087004E0062048
:10026000DB49087000E000BF00BF1620D7490870C6
:100270001820D5490870D0484078012803D0CE48CE
:100280008079012829D1D248007807281DD2DFE8DB
:1002900000F01C04080C101418000120CC49087050
:1002A00014E00120CA49087010E00220C849087013
:1002B0000CE00320C649087008E00420C449087017
:1002C00004E00520C249087000E000BF00BF16200E
:1002D000BE4908701820BC490870B74880780128CA
:1002E00003D0B5488078022874D10320B2498870C1
:1002F000B7480078072865D2DFE800F064041526C7
:1003000037465500B3480078032803DB0020B14985
:10031000087004E0AF480078401CAE49087018200F
:10032000A949087055E0AB484078022803DB00205B
:10033000A849487004E0A7484078401CA549487087
:100340001820A149087044E0A2488078022803DB05
:100350000020A049887004E09E488078401C9D4998
:10036000887018209849087033E007209849087071
:100370001820964908701A20934908700120964960
:1003800008708E49087024E00B20914908701720EE
:100390008E49087019208C49087001208E49087018
:1003A0008649087015E00E20894908701920874990
:1003B00008701B20844908700120874908707F4914
:1003C000087006E001208249087018207E490870F4
:1003D00000BF00BF7848C078012803D07648C078B5
:1003E00002283AD103207449C8707948007801285E
:1003F00004D0022810D003282AD11BE075480078C9
:10040000002803DC03207349087004E07148007879
:10041000401E704908701CE06E484078002803DCDC
:1004200002206C49487004E06A484078401E6949DF
:1004300048700EE067488078002803DC0220654998
:10044000887004E063488078401E6249887000E04C
:1004500000BF00BF18205C49087057480079022887
:100460000CD10120554908700720554981F82D000D
:100470002220554908701E205449087070474E4884
:10048000007801282ED1524800780B2804D00C287F
:1004900009D00D2821D10DE00C204D4908701920FC
:1004A000494908701DE00D20494908701920464946
:1004B000087016E006204649087018204249087066
:1004C00016204249087001203C4908700020434929
:1004D000087002203B49087003E019203A4908706F
:1004E00000BF00BF34484078012803D032488079EB
:1004F000012822D1364800780B2804D00C2809D0D6
:100500000D2815D10DE00B203149087019202E4916
:10051000087011E00B202E49087019202A49087034
:100520000AE00C202A49087019202749087003E0C6
:1005300019202549087000BF00BF1F488078012896
:1005400003D01D488078022855D103201A498870AD
:100550001F4800780B2804D00C2810D00D2845D156
:100560001BE01C48C079032803DB03201949C8712C
:1005700004E01848C079401C1649C87137E0154896
:10058000007A032803DB03201249087204E01148B3
:10059000007A401C0F49087229E00E48407A03286F
:1005A0001EDB03200B4948721FE00000000C0140D5
:1005B000E0030020A0030020100000204B000020DA
:1005C000580400204E000020EC000020C000002055
:1005D00048000020F2040020F2000020500000201B
:1005E000FA48407A401CF949487200E000BF00BF59
:1005F0001920F7490870F748C078012803D0F5485A
:10060000C07802283AD10320F249C870F248007835
:100610000B2804D00C2810D00D282AD11BE0EB4861
:10062000C079002803DC0020E849C87104E0E748ED
:10063000C079401EE549C8711CE0E448007A0028F2
:1006400003DC0020E149087204E0E048007A401E23
:10065000DE4908720EE0DD48407A002803DC002005
:10066000DA49487204E0D948407A401ED7494872B6
:1006700000E000BF00BF1920D5490870D5480079B7
:1006800002280CD10120D54908700720D44981F8EF
:100690002D002220CE4908701E20D24908707047D4
:1006A000CC480078012837D1CB480078072806D0FD
:1006B000082812D0092809D00A2828D114E00920D6
:1006C000C54908701A20C249087024E00820C249B0
:1006D00008701A20BE4908701DE00A20BE49087043
:1006E0001A20BB49087016E00520BB490870182085
:1006F000B74908701620BB4908700120B749087037
:100700000020B94908700220B849087003E01A2097
:10071000AF49087000BF00BFAE484078012803D041
:10072000AC48807901282BD1AB480078072806D047
:10073000082812D0092809D00A281CD114E0072063
:10074000A54908701A20A249087018E00720A2499C
:1007500008701A209E49087011E009209E4908700F
:100760001A209B4908700AE008209B4908701A204B
:100770009749087003E01A209549087000BF00BF30
:1007800094488078012803D09248807802284AD182
:1007900003209049887090480078072806D00828E0
:1007A00020D0092810D00A2838D129E08748C078FD
:1007B000022803DB02208549C87004E08348C07822
:1007C000401C8249C8702AE080484079022803DB37
:1007D00002207E49487104E07C484079401C7B49F6
:1007E00048711CE079480079022803DB0220774930
:1007F000087104E075480079401C744908710EE0E6
:1008000072488079022803DB02207049887104E075
:100810006E488079401C6D49887100E000BF00BFC0
:100820001A206B4908706B48C078012803D06948CA
:10083000C07802284AD103206649C870664800780B
:10084000072806D0082820D0092810D00A2838D137
:1008500029E05E48C078002803DC00205B49C870AE
:1008600004E05A48C078401E5849C8702AE05748EA
:100870004079002803DC00205449487104E05348C3
:100880004079401E514948711CE0504800790028C9
:1008900003DC00204D49087104E04C480079401EFB
:1008A0004A4908710EE049488079002803DC00209D
:1008B0004649887104E045488079401E4349887163
:1008C00000E000BF00BF1A2041490870414800798C
:1008D00002280CD10120414908700720404981F8C5
:1008E0002D0022203A4908701E203E4908707047AA
:1008F00038480078012822D1374800780E2804D0E3
:100900000F2809D0102818D110E00F2032490870A4
:100910001B202F49087011E010202F4908701B2060
:100920002B49087002203149087007E011202A493C
:1009300008701B202649087000E000BF00BF254852
:100940004078012803D024480078112824D10620BB
:10095000214908702248808C25494988884212DB49
:1009600040F6C4102349A1F842000120224981F831
:1009700024001020164908700E201A49087004201F
:100980001E49087005E00B20164908700C2010491C
:1009900008700120114908700E488079012831D172
:1009A0000D4800780E2802D00F2829D106E00E202D
:1009B000094908701B200649087022E00E200649EC
:1009C00008701B20024908701BE00000F2040020A0
:1009D000EC00002010000020480000204B00002008
:1009E00058040020C0000020500000204E000020CD
:1009F000E4040020E0030020A00300204F000020BA
:100A000000BF00BFFB488078012803D0F9488078F8
:100A1000022819D10320F7498870F74800780E287A
:100A20000DD1F648807A0A2803DB0A20F349887240
:100A300004E0F248807A401CF049887200E000BF70
:100A400000BF1B20EE490870EA48C078012803D097
:100A5000E848C078022819D10320E649C870E64862
:100A600000780E280DD1E548807A002803DC0020AC
:100A7000E249887204E0E148807A401EDF498872CA
:100A800000E000BF00BF1B20DD490870D948007995
:100A900002280CD10120DB4908700720DA4981F8CF
:100AA0002D002220D64908701E20D84908707047B2
:100AB00008B5D048407802287ED10020CD49487042
:100AC000D3494871D3490870D3490870D349087095
:100AD000CF49087048708870D148407A012800D109
:100AE00008BDCF48807B012800D1F9E7CC48407A87
:100AF000042809D140F6C410CA49A1F842000120D7
:100B0000C94981F8240003E00020C74981F8240086
:100B1000C348007901280FD10020C1490871BA48A3
:100B2000808CC2494988884203DB0820C04908718B
:100B300002E00020BF490870B9484079012804D17B
:100B40000020B7494871BB490870B5488079012831
:100B500004D10020B2498871B6490870B048C07A03
:100B6000012804D10020AE49C872B2490870AC48CF
:100B7000C07801280CD10020A949C8700220AA49D8
:100B800081F82F00AC48A74908660020A9490870E1
:100B90000020AA49087042F21070A2498860002023
:100BA000A74908700420984981F82D00084640881C
:100BB00058B10A20954900E024E008700B209049C4
:100BC000087001208F49087018E08F48C08860B114
:100BD00001209C4908700B208C490870232088490B
:100BE000087001208749087008E00B2087490870C9
:100BF0000C208349087001208249087042F210706D
:100C0000884988607B480079022852D17E48806BF1
:100C1000000E8DF800007C48806B000C8DF8010000
:100C20007948008F000A8DF80200774890F8380064
:100C30008DF80300844A04216846FAF7B3FEFAF7F8
:100C400039FD01206F49087004206F4981F82D009B
:100C50007E48807910BB01206A4908700D206B49DD
:100C600008700F206649087000206F49C8757849E0
:100C700008701E207749087022207749087077484D
:100C80000078774908707748007877490870774886
:100C90006449486301207649087021E707205A49D2
:100CA00081F82D001E2059490870222054490870EF
:100CB00016E76248007830B9FAF74EFEFAF785FC7D
:100CC00001205E4908706B480078012804D1FAF7CA
:100CD000F1FC002067490870534890F82F00002865
:100CE0007ED102206449087047484088E0B340F64E
:100CF000C4104C49A1F842004948407A042808D160
:100D000040F6C410A1F842000120474981F82400B0
:100D10000AE00020444981F824004D4908704FF44E
:100D2000007156480BF0D3FE002045490870544925
:100D300008703B49C8700A20344908700B203049BC
:100D4000087001202F4908704E490870FCF769FCB3
:100D500042F2D000334908854B480068C862012040
:100D6000294981F82D00CFE0FFE72748C088C0B3AC
:100D700001202D49C8742A48407A042809D140F638
:100D8000C4102849A1F842000120274981F8240015
:100D90000AE00020244981F824002D4908704FF40E
:100DA000007136480BF093FE40F6C4101D49A1F8BF
:100DB0004200002022490870314908701849C87063
:100DC0000B201249087023200D49087003200E499A
:100DD00081F82D0001200B4908700320294901E00A
:100DE00096E053E00870FCF71CFC42F2D0000D497D
:100DF000088589E01000002048000020F20400204F
:100E0000EC0000204B00002058040020C00000200F
:100E1000F80000206B0100206A0100205901002029
:100E2000B0120020E0030020A0030020E404002012
:100E3000330000204F000020E0930400A0000020B9
:100E40004E000020DD00002000A00608FE04002067
:100E5000DC000020D2000020EE000020D5000020A1
:100E6000D3000020F1000020EF00002020BF02008E
:100E7000F20000200901002028000020000C0140A1
:100E80004D000020C1000020C4000020F748407A37
:100E9000042809D140F6C410F549A1F84200012008
:100EA000F44981F824000AE00020F24981F8240086
:100EB000F14908704FF40071F0480BF008FE40F65D
:100EC000C410EB49A1F842000020ED490870ED493B
:100ED0000870E649C8700B20EB4908700C20EB49FC
:100EE00008700220EA4981F82D000120E9490870C4
:100EF0000220E9490870FCF794FBE8480068DC49E7
:100F0000C86242F2D00008850520DA4981F82F0036
:100F1000D84890F83000012829D1D4488079012898
:100F200017D0D2484079012813D0D048C07A012880
:100F30000FD0CE48C07801280BD0CC4800790128CA
:100F400007D0CA48807B012803D0C848407A0128CE
:100F50000DD10B20CE4981F82D000120C549C8755F
:100F60000320CF4908700020C24981F8300000BF3B
:100F7000B6E508B5CB480079022859D1C448806B42
:100F8000000E8DF80000C248806B000C8DF8010047
:100F9000BF48008F000A8DF80200BD4890F8380065
:100FA0008DF80300C04A04216846FAF7FBFCBF48ED
:100FB000007830B9FAF7D0FCFAF707FB0120BB49FB
:100FC0000870FAF777FB0120B24908700420B04995
:100FD00081F82D00B6488079F8B90D20AA4908702B
:100FE0000F20AA4908700020A249C875A2490870BC
:100FF0001E20B04908702220AF490870AF48007821
:10100000AF490870AF480078AF490870AF489849B9
:1010100048630120AE49087008BD07209C4981F84B
:101020002D001E2098490870222098490870F3E787
:1010300000BFF1E708B59B48007801287ED1A5489C
:101040000078C01E102877D2DFE800F00816320FB3
:10105000761D2B43515F4A3C2458666F06209D49FC
:1010600008701F208949087067E0042099490870BA
:101070001F208649087060E00820964908701F20EC
:101080008249087059E00F20924908701F207F495B
:10109000087052E009208F4908701F207B490870B2
:1010A0004BE005208B4908701F207849087044E008
:1010B0000E20884908700120764908702020734965
:1010C00008703AE00A208349087020206F490870B0
:1010D00033E00D207F49087020206C4908702CE017
:1010E0000B207C49087020206849087025E01020FA
:1010F000784908702020654908701EE00C20754969
:10110000087020206149087017E0112071490870AB
:1011100020205E49087010E012206E4908702020DF
:101120005A49087009E009E006E012206949087090
:1011300020205649087000E000BF00BF59484078A1
:10114000012803D05748807901287ED16148007872
:10115000C01E102877D2DFE800F00816320F761D87
:101160002B43515F4A392458666F03205949087050
:101170001F204649087067E00320564908701F2069
:101180004249087060E00620524908701F203F491C
:10119000087059E004204F4908701F203B4908702F
:1011A00052E008204B4908701F20384908704BE076
:1011B0000F20484908701F203449087044E0092076
:1011C000444908701F20314908703DE00120314931
:1011D000087003203F4908701F202C49087033E035
:1011E0000E203C4908702020284908702CE00A2075
:1011F0003849087020202549087025E00D20354920
:1012000008702020214908701EE00B203149087029
:1012100020201E49087017E010202E490870202059
:101220001A49087010E00C202A490870202017493C
:10123000087009E009E006E0112026490870202026
:101240001249087000E000BF00BF164880780128EE
:1012500003D014488078022875D103201149887082
:101260001C480078C01E10286ED235E0B012002055
:10127000E0030020A0030020DC000020000C01405F
:101280004E0000204D000020C0000020EC00002097
:10129000580400204B000020C1000020C4000020A2
:1012A0004F0000201000002000A00608A000002031
:1012B000FE040020D2000020EE000020D500002017
:1012C000D3000020F1000020EF00002020BF02002A
:1012D000F200002049000020DFE800F00824531944
:1012E000CC48647A8FAB846F379AB6C1FB480078DC
:1012F000032803DB0120F949087004E0F74800786F
:10130000401CF64908701F20F5490870B3E0F34807
:10131000C078012802D10020F049C8701F20F04990
:101320000870A8E0ED484078032803DB0120EB4972
:10133000487004E0E9484078401CE84948701F20A4
:10134000E749087097E097E094E0E448C089642892
:1013500003DB0020E149C88104E0E048C089401C6B
:10136000DE49C8811F20DE49087084E0DB484079EF
:10137000012802D10020D94948711F20D84908709E
:1013800079E0D6488078092803DB0120D3498870AA
:1013900004E0D2488078401CD04988701F20D04992
:1013A000087068E0CD488079012802D10020CB493F
:1013B00088711F20CA4908705DE0C848C07A0128BA
:1013C00002D10020C549C8722020C549087052E0EA
:1013D000C248C07910B90120C049C8712020C04955
:1013E000087048E0BD48807A012802D10020BB493E
:1013F00088722020BA4908703DE0B848007A012878
:1014000002D10020B54908722020B549087032E0A9
:10141000B248007B012808D10020B04908730120A0
:10142000B04908700020B04908702020AC4908700D
:1014300021E0AA48407A012802D10020A749487239
:101440002020A749087016E0A448007C012802D19A
:101450000020A24908742020A14908700BE09F4891
:10146000407C012802D100209C49487420209C49DE
:10147000087000E000BF00BF9C48C078012803D07E
:101480009A48C078022873D103209849C8709848B8
:101490000078C01E10286CD2DFE800F008234F1936
:1014A000C34560768BA5816C3495AFB98B480078C5
:1014B000012803DC03208949087004E0874800788C
:1014C000401E864908701F2085490870AAE083489D
:1014D000C07810B901208149C8701F208049087068
:1014E000A0E07E484078012803DC03207B49487057
:1014F00004E07A484078401E784948701F207849B7
:1015000008708FE07548C089002803DC64207349A7
:10151000C88104E07148C089401E7049C8811F20FD
:101520006F4908707EE06D48407910B901206B4921
:1015300048711F206A49087074E068488078012863
:1015400003DC09206549887004E064488078401E07
:10155000624988701F206249087063E05F488079A3
:1015600010B901205D4988711F205D49087059E05C
:1015700059E056E05948C07A10B901205749C8725D
:101580002020574908704DE05448C079012802D105
:1015900000205249C87120205149087042E04F484C
:1015A000807A10B901204D49887220204C4908707A
:1015B00038E04A48007A10B90120484908722020D2
:1015C000474908702EE04548007B40B90120434957
:1015D0000873002043490870012043490870202007
:1015E0003F4908701EE03D48407A10B901203B4950
:1015F000487220203A49087014E03848007C10B93D
:101600000120364908742020354908700AE0334823
:10161000407C10B9012031494874202030490870BD
:1016200000E000BF00BF3148007902283AD1012014
:1016300030490870FAF728FD2848007B012812D1AC
:1016400029480078012823D100208DF800008DF86A
:1016500001008DF802008DF80300274A0421684636
:10166000FAF7A0F914E01F480078012810D10020F3
:101670008DF8000002208DF8010046208DF8020050
:1016800008208DF803001C4A04216846FAF78AF9FD
:1016900007201A4981F82D002220114908701E20C8
:1016A0001749087008BD10B515480078212872D276
:1016B000DFE800F0712B2E313437713A4043494C4A
:1016C00071464F5E6162636467655255585B6A712B
:1016D0003D1128666E00FBF75BFF5DE0FE04002015
:1016E000EC000020E2000020E300002010000020B9
:1016F000490000204B00002000A0060858040020EC
:10170000C0000020FBF712FF46E0FCF71DF843E0A5
:10171000FCF75CF840E0FCF726F93DE0FCF741F906
:101720003AE0FCF7EDF937E0FCF7C8FD34E0FCF7F0
:101730007EFE31E0FDF7C0F92EE0FDF726FD2BE03F
:10174000FDF7ACFD28E0FDF7F6FE25E0FEF7E9F831
:1017500022E0FEF78EFC1FE0FEF75FFD1CE0FEF7C7
:101760008EFE19E0FEF79CFF16E0FFF7C1F813E0CC
:10177000FFF7FFFB10E000BF00BF00BF00BF00BFCE
:1017800000BFFFF795F907E0FFF754FC04E002E023
:10179000FDF75DF900E000BF00BF10BDFE48007816
:1017A0000A287AD006DC01280BD0022855D003285D
:1017B00074D176E00B2872D00D2871D01928F7D19A
:1017C000A2E1F648807B012846D1F548C08A28B1BD
:1017D000F348C08A401EF249C8823DE0F1480078D3
:1017E000401CF049087008460078022815DB0020EC
:1017F00008700320E84908700220EB49087041F2A4
:101800008830E749C8820920E84981F82D00012085
:10181000E2494873002008731EE0E548007802287A
:1018200004D141F28830DE49C88215E00020DD494C
:1018300008700320D84908700220DB49087041F283
:101840008830D749C8820920D84981F82D00012065
:10185000D24948730020087373E1D148C08A28B187
:10186000CF48C08A401ECE49C88215E0D1480078D2
:10187000092803D10A20CC49087006E0CD48007839
:101880000A2802D10920C84908700220C2490870FC
:1018900041F28830C249C88253E138E050E163E048
:1018A00010E1BF48C08A28B1BD48C08A401EBC496B
:1018B000C8822BE0BB480078401CBA490870084633
:1018C000007802280CDB002008700420B249087060
:1018D0000320B549087041F28830B149C88215E04B
:1018E000B3480079022804D141F28830AC49C8825B
:1018F0000CE00020AB4908700420A74908700320C1
:10190000A949087041F28830A549C88219E1A34865
:10191000407C88B9A248008B28B1A148008B401EAA
:101920009F49088308E0A44880899D4908830120D5
:101930009A49487481F839009C4890F82D00042891
:1019400011D09748008F28B19548008F401E9449C8
:10195000088708E001209149887581F839004FF423
:101960007A708F490887ECE00120944908708B4811
:1019700090F82C0001280CD18948806D28B1884846
:10198000806D401E8649886503E00020834981F808
:101990002C008248807E012831D18148408F28B3B5
:1019A0007F48408F401E7E4948870846408F4FF44D
:1019B000FA7190FBF1F201FB120000BB774890F83E
:1019C000220030B90120754981F8220081F82300F6
:1019D00015E0724890F82200022810D106206F49C5
:1019E00081F82200012081F8230008E000206B49E3
:1019F000887681F8220042F210706949488767486A
:101A0000007F012831D16648C08F28B36448C08F59
:101A1000401E6349C8870846C08F4FF4FA7190FB97
:101A2000F1F201FB120000BB5C4890F8370030B9BE
:101A300001205A4981F8370081F8380015E05748ED
:101A400090F83700022810D10620544981F8370059
:101A5000012081F8380008E000205049087781F81B
:101A6000370041F288304E49C8874C48407C98B9CD
:101A70004B48008B28B14A48008B401E48490883D8
:101A80000AE001204549487447F230504449088330
:101A90000120424981F83900444890F82D0004287B
:101AA0000FD03F48008F28B13D48008F401E3C4971
:101AB000088706E00120394988754FF47A70384963
:101AC00008873EE03648406B28B13548406B401EE1
:101AD0003349486317E001203949087039480078D4
:101AE0002D490870384800782F490870012037497F
:101AF000087037482A494863002028494875012062
:101B000081F83000C8751CE032480078102816D1E2
:101B10002348B0F8640038B12148B0F86400401E92
:101B20001F49A1F864000AE011202A4908701B200F
:101B30001D4908704FF47A701949A1F8640000E05B
:101B400000BF00BF1448007810281FD0124800784A
:101B500011281BD010480078122817D00E480078A2
:101B6000132813D00C48007815280FD00A480078A5
:101B700014280BD0084800780F2807D006480078B2
:101B80000E2803D0044800781F2877D10448B0F805
:101B90004200C8B302481FE0C0000020A00300209C
:101BA000E0030020C2000020EC00002058040020C8
:101BB00008000020ED000020E4040020DB000020ED
:101BC000F2000020D3000020EF0000204B00002096
:101BD00020BF020048000020B0F84200401EFE492D
:101BE000A1F842000846B0F84200B0F5FA6F0CDBED
:101BF0000120FA490870FA480078032827DA012002
:101C0000F84981F8210022E011E0F348B0F84200E1
:101C1000B0F5FA6F1BDA0020F0490870F048007840
:101C2000032814DA0020EF4981F821000FE040F684
:101C3000C410E949A1F84200E9480078401CE8498D
:101C4000087008460078032801DB03200870E54887
:101C500090F82F00012814D1DF48006E30B1DE4823
:101C6000006E401EDC4908660BE007E0DE48DA49FA
:101C700008660020DB4981F82F0002E00020D849E7
:101C80000870D848407E01282AD1D348C068B8B12E
:101C9000D148C068401ED049C8600846C0684EF6AA
:101CA0006021B0FBF1F201FB1200C8B9CF480089F6
:101CB000401ECE4908810120CA4981F838000FE052
:101CC0000020CA490881C7494876C94880894EF62C
:101CD00060214843C049C8600020C24981F8220001
:101CE000704708B5C3480078022855D1BF4890F81E
:101CF0002D0001280ED0BD4890F82D00022809D0F3
:101D0000BA4890F82D00062804D0B84890F82D0065
:101D1000032809D10220B3490873002081F8250067
:101D20000920B24981F82E000120AE4981F8270030
:101D3000B14800780A2803D0AF4800780B2803D1B7
:101D40000120A84981F828004FF40051AB480AF05F
:101D5000A2FEE8B1AA48407A042803D00221A7488D
:101D60000AF0B3FEC820A7490880A74908800020D0
:101D7000A64908704FF42F70A54908800020A54996
:101D800008704FF47A70A44908800020A3490880A5
:101D90000A20FAF753FE27E0944890F82D00012816
:101DA0000ED0924890F82D00022809D08F4890F864
:101DB0002D00062804D08D4890F82D0003280AD164
:101DC00001208849087342F2D00083490885012028
:101DD000844981F825000020FAF730FE002081496F
:101DE00081F8270081F828007E48C07B01287DD13A
:101DF0007E4890F82D00072879D2DFE800F07804BB
:101E00005455BB78EB00774890F82F00022849D151
:101E10007648808C401C754988840846808C8049AF
:101E200008807248806B401C704988630846808C2B
:101E30000A2190FBF1F201FB120020BB6B48806B82
:101E4000000E8DF800006948806B000C8DF80100D1
:101E50006648008F000A8DF80200644890F8380048
:101E60008DF803006F4A04216846F9F79BFD6E4820
:101E7000007830B9F9F770FDF9F7A7FB01206A493E
:101E80000870F9F717FC59484088401E57494880A8
:101E90000846008C401E088400205249C8730B205D
:101EA00062490870E0E000BF4E4890F82F00022819
:101EB0005FD14C48C07C012804D14C48C088401EEA
:101EC0004A49C8804948808C401C48498884084653
:101ED000808C534908804548806B401C4349886387
:101EE0000846808C0A2190FBF1F201E0BDE0B7E0EA
:101EF00001FB120020BB3D48806B000E8DF80000F6
:101F00003A48806B000C8DF801003848008F000AB9
:101F10008DF80200354890F838008DF80300414AEA
:101F200004216846F9F73EFD3F48007830B9F9F7DB
:101F300013FDF9F74AFB01203B490870F9F7BAFB9A
:101F40002A48008C401E294908840846C08C401C41
:101F5000C88400202349C873354800780C2802D172
:101F60003249087005E032480078232801D12F4912
:101F7000087079E02F48007801282AD11B48408852
:101F8000A0B11A484088401E184948800846808CF5
:101F9000401C88840846808C214908801348806B47
:101FA000401C1249886303F06EFE0FE00F48808CDE
:101FB000401C0E4988840846808C194908800B48CB
:101FC000806B401C0949886303F0CFFF002005495E
:101FD000C87349E030E00000E0030020DC0000208E
:101FE000EB000020A0030020E09304005804002030
:101FF000E404002028000020C0000020000C014064
:10200000B0120020CE000020520100205801002014
:102010005E01002068010020700100207201002094
:10202000D600002000A00608A0000020EC00002040
:10203000ED000020E50000200C480088401C0B4902
:10204000088000200A49C87308480088142803D172
:1020500008200849087002E007200649087003E0DC
:1020600000200349C87300BF00BF08BD580400200A
:10207000A0030020EC00002070B505460E46144673
:1020800031462846F8F79BFDE0B2F8F7CBFC70BD6F
:102090002DE9FF4F83B08046894649464046F8F710
:1020A0008EFD0598A0EB08050698A0EB0906002D0B
:1020B00002DB0120029003E04FF0FF3002906D42FE
:1020C000002E02DB0120019003E04FF0FF30019071
:1020D00076424FEA450A4FEA460BB54219DDABEBB3
:1020E0000504002712E049464046109AFFF7C4FF56
:1020F000002C05DBA4EB0A04019848441FFA80F980
:102100005C44029840441FFA80F87F1CAF42EADD2D
:1021100018E0AAEB0604002712E049464046109A50
:10212000FFF7AAFF002C05DBA4EB0B040298404448
:102130001FFA80F85444019848441FFA80F97F1C24
:10214000B742EADD07B0BDE8F08F2DE9F04706465B
:102150000F4691469A46089CB04624E02078802895
:1021600020DA25780D2D01D1464619E0002514E02E
:1021700005EB4500F64911F81000217888420AD194
:1021800005EB4500F24B03EB4000421CF9B2304630
:10219000F8F7D6FD03E0681C85B2772DE8DB00BFB9
:1021A000701D86B2641C20780028D7D1BDE8F08766
:1021B0002DE9F04706460F4691469A46089CB046E0
:1021C00024E02078802820DA25780D2D01D146469C
:1021D00019E0002514E005EB4500DD4911F8100079
:1021E000217888420AD105EB4500D94B03EB40002A
:1021F000421CF9B23046F8F7A3FD03E0681C85B233
:10220000772DE8DB00BFB01D86B2641C2078002863
:10221000D7D1BDE8F0872DE9F04706460F46914635
:102220009A46089DB04651E02878802824DA2C7818
:102230000D2C01D146461BE0002416E004EB84007F
:1022400000EBC400C349085C297888420BD104EB39
:10225000840000EBC400BF4B1844421CF9B2304666
:10226000F8F7A0FD03E0601C84B2772CE6DB00BF2A
:102270006D1CB01D86B229E0002420E004EBC400F0
:1022800000EB4000B449085C2978884215D104EB82
:10229000C40000EB4000B0490844407869788842A7
:1022A0000BD104EBC40000EB4000AB4B1844C21C44
:1022B000F9B23046F8F716FD03E0601C84B2C82C72
:1022C000DCDB00BFAD1C06F10C0086B228780028CC
:1022D000AAD1BDE8F0872DE9F04706460F469146A2
:1022E0009A46089DB04651E02878802824DA2C7858
:1022F0000D2C04D1464607F1100087B217E00024E8
:1023000012E004EB04109549085C2978884209D151
:1023100004EB0410914B1844421CF9B23046F8F714
:1023200076FD03E0601C84B2772CEADB00BF6D1CF5
:1023300006F1080086B229E0002420E0C4EBC400C6
:1023400000EB80008649085C2978884215D1C4EBEF
:10235000C40000EB800082490844407869788842D4
:102360000BD1C4EBC40000EB80007D4B1844C21CB1
:10237000F9B23046F8F788FC03E0601C84B2C82C40
:10238000DCDB00BFAD1C06F1100086B22878002807
:10239000AAD1BDE8F0872DE9F04706460F469046E2
:1023A0009946089C37E0207880280CDA2578202D83
:1023B00003DDA5F1200085B200E00025641C06F1D4
:1023C000080086B227E000251FE0C5EB051000EBF2
:1023D00080006449085C2178884214D1C5EB05105F
:1023E00000EB80005F4908444078617888420AD158
:1023F000C5EB051000EB80005A4B1844C21CF9B223
:102400003046F8F715FC681C85B2C82DDDDBA41C2E
:10241000A6F1180086B220780028C4D1BDE8F08764
:10242000024600201009002805DD092803DC00F120
:102430003003D8B208E00A2805DB0F2803DC00F1DE
:102440003703D8B200E030200870491C02F00F00BA
:10245000002805DD092803DC00F13003D8B208E0CC
:102460000A2805DB0F2803DC00F13703D8B200E0AF
:102470003020087070472DE9F04705460E46144697
:102480009946B9F10B0F62D2DFE809F06106153306
:102490006EADFEFDFCFBFA003020281820704FF0D6
:1024A00000006070A070E07020716071A071E07138
:1024B0002072607268E30A2200232846314616F033
:1024C00084FC303020704FF00A024FF000032846A1
:1024D000314616F07AFC3020101860704FF0000082
:1024E000A070E07020716071A071E0712072607264
:1024F0004AE3642200232846314616F066FC303059
:1025000020704FF064024FF000032846314616F069
:102510005CFC174619460A220023384616F055FC83
:10252000303060704FF00A024FF000032846314609
:1025300016F04BFC30201018A0704FF00000E07037
:1025400020716071A071E071207260721CE31AE367
:1025500014A9020854AB020894B6020834B0020869
:10256000C4C5020826CD02084FF47A72002328461B
:10257000314616F02AFC303020704FF47A724FF05A
:1025800000032846314616F020FC174619466422FF
:102590000023384616F019FC303060704FF06402AA
:1025A0004FF000032846314616F00FFC1746194637
:1025B0000A220023384616F008FC3030A0704FF095
:1025C0000A024FF000032846314616F0FEFB302089
:1025D0001018E0704FF0000020716071A071E07180
:1025E00020726072D0E242F2107200232846314617
:1025F00016F0EBFB3030207042F210724FF0000307
:102600002846314616F0E1FB174619464FF47A7218
:102610000023384616F0D9FB303060704FF47A72E0
:102620004FF000032846314616F0CFFB17461946F7
:1026300064220023384616F0C8FB3030A0704FF0FB
:1026400064024FF000032846314616F0BEFB1746E1
:1026500019460A220023384616F0B7FB3030E070E6
:102660004FF00A024FF000032846314616F0ADFB4A
:102670003020101820714FF000006071A07104E04C
:10268000DDE150E1D2E063E003E0E07120726072CE
:102690007AE2FE4A00232846314616F096FB303097
:1026A0002070FA4A4FF000032846314616F08DFBA1
:1026B0001746194642F210720023384616F085FB81
:1026C0003030607042F210724FF0000328463146FD
:1026D00016F07BFB174619464FF47A7200233846F2
:1026E00016F073FB3030A0704FF47A724FF0000395
:1026F0002846314616F069FB174619466422002326
:10270000384616F062FB3030E0704FF064024FF054
:1027100000032846314616F058FB174619460A2290
:102720000023384616F051FB303020714FF00A027A
:102730004FF000032846314616F047FB30201018B2
:1027400060714FF00000A071E071207260721BE2B6
:10275000CF4A00232846314616F037FB3030207030
:10276000CB4A4FF000032846314616F02EFB1746A1
:102770001946C64A0023384616F027FB30306070F1
:10278000C24A4FF000032846314616F01EFB17469A
:10279000194642F210720023384616F016FB30300C
:1027A000A07042F210724FF000032846314616F036
:1027B0000CFB174619464FF47A720023384616F080
:1027C00004FB3030E0704FF47A724FF0000328467B
:1027D000314616F0FAFA17461946642200233846A5
:1027E00016F0F3FA303020714FF064024FF000031E
:1027F0002846314616F0E9FA174619460A22002300
:10280000384616F0E2FA303060714FF00A024FF0AD
:1028100000032846314616F0D8FA30201018A0716F
:102820004FF00000E07120726072ADE1994A002320
:102830002846314616F0C9FA30302070954A4FF0DC
:1028400000032846314616F0C0FA17461946904A4A
:102850000023384616F0B9FA303060708C4A4FF0D9
:1028600000032846314616F0B0FA17461946874A43
:102870000023384616F0A9FA3030A070834A4FF092
:1028800000032846314616F0A0FA1746194642F2D0
:1028900010720023384616F098FA3030E07042F299
:1028A00010724FF000032846314616F08EFA174694
:1028B00019464FF47A720023384616F086FA303003
:1028C00020714FF47A724FF000032846314616F01B
:1028D0007CFA1746194664220023384616F075FA2A
:1028E000303060714FF064024FF0000328463146EB
:1028F00016F06BFA174619460A220023384616F0DE
:1029000064FA3030A0714FF00A024FF000032846FD
:10291000314616F05AFA30201018E0714FF00000DE
:102920002072607230E15C4A00232846314616F07E
:102930004CFA30302070584A4FF000032846314698
:1029400016F043FA17461946524A0023384616F045
:102950003CFA303060704F4A4FF000032846314651
:1029600016F033FA17461946494A0023384616F03E
:102970002CFA3030A070464A4FF00003284631460A
:1029800016F023FA17461946404A0023384616F037
:102990001CFA3030E0703D4A4FF0000328463146C3
:1029A00016F013FA1746194642F210720023384601
:1029B00016F00BFA3030207142F210724FF0000323
:1029C0002846314616F001FA174619464FF47A7236
:1029D0000023384616F0F9F9303060714FF47A72FE
:1029E0004FF000032846314616F0EFF91746194616
:1029F00064220023384616F0E8F93030A0714FF019
:102A000064024FF000032846314616F0DEF91746FF
:102A100019460A220023384616F0D7F93030E07103
:102A20004FF00A024FF000032846314616F0CDF968
:102A30003020101820724FF000006072A4E0174A96
:102A400000232846314616F0C0F930302070134A72
:102A50004FF000032846314616F0B7F917461946DD
:102A60000D4A0023384616F0B0F9303060700A4A3B
:102A70004FF000032846314616F0A7F917461946CD
:102A8000044A0023384616F0A0F909E0A0860100A8
:102A900040420F008096980000E1F50500CA9A3B7D
:102AA0003030A070F84A4FF000032846314616F047
:102AB0008CF917461946F54A0023384616F085F971
:102AC0003030E070F14A4FF000032846314616F0EE
:102AD0007CF917461946EE4A0023384616F075F978
:102AE00030302071EA4A4FF000032846314616F094
:102AF0006CF91746194642F210720023384616F058
:102B000064F93030607142F210724FF000032846D1
:102B1000314616F05AF9174619464FF47A720023D7
:102B2000384616F052F93030A0714FF47A724FF0F7
:102B300000032846314616F048F917461946642224
:102B40000023384616F041F93030E0714FF064024E
:102B50004FF000032846314616F037F9174619465C
:102B60000A220023384616F030F9303020724FF038
:102B70000A024FF000032846314616F026F93020AD
:102B80001018607200E000BF00BFBDE8F08710B50C
:102B9000C04890F82000012805D12222FF210846D4
:102BA000F8F723F804E0222200210846F8F71DF880
:102BB00010BD10B5B84890F82D00042805D1512259
:102BC000FF210846F8F711F804E0512200210846D9
:102BD000F8F70BF810BD10B5AE48407C012805D1C0
:102BE0005222FF210846F8F700F804E052220021A3
:102BF0000846F7F7FAFF10BD10B5A848C07850B9DD
:102C0000A44890F83D00012805D16C22FF21084618
:102C1000F7F7EBFF04E06C2200210846F7F7E5FF29
:102C200010BD10B59D48C07918B19A48007E0128A2
:102C30000AD12922FF210846F7F7D7FF2A22FF21D0
:102C40000846F7F7D2FF09E0292200210846F7F7E6
:102C5000CCFF2A2200210846F7F7C7FF10BD10B5A8
:102C600000248D48808AA0420AD08A4890F82B0020
:102C7000012805D18848047D0020864981F82B0071
:102C80008748407A042834D0012308228321772002
:102C9000F7F76BFF8048808A282805DA7722012120
:102CA0000846F7F7A2FF24E07B48808A282809DB42
:102CB0007948808A572805DA782201210846F7F7F3
:102CC00094FF16E07448808A572809DB7248808A8E
:102CD000642805DA792201210846F7F786FF08E023
:102CE0006D48808A642804DB7A2201210846F7F7C0
:102CF0007CFF10BD1FB56BA207CA01AB07C36548B7
:102D000090F83900012822D16248407C012805D181
:102D10005222FF210846F7F768FF04E05222002103
:102D20000846F7F762FF5C4890F82D00042805D1AB
:102D30005122FF210846F7F758FF04E051220021F5
:102D40000846F7F752FF0020524981F839005148F0
:102D5000807D012838D156480078012806D0022805
:102D600012D0032819D0042829D11FE008220021FD
:102D70000846F7F73AFF0522FF210846F7F735FF27
:102D800002204B4908701BE00622FF210846F7F796
:102D90002CFF03204649087012E00722FF21084655
:102DA000F7F723FF04204249087009E00822FF21B9
:102DB0000846F7F71AFF01203D49087000E000BF00
:102DC00000BF0020334988753A4800780B285AD153
:102DD000304890F8230001287ED137480078232816
:102DE0007CD12C48807E012811D134A04EF67D7311
:102DF0000022032100901020FFF70DFA2648448D91
:102E0000032301AA20460021FFF735FB10E02EA086
:102E10004EF67D730022032100901020FFF7FBF98E
:102E20001D48048D032301AA20460021FFF723FB40
:102E3000184890F8220001280DD10220154981F888
:102E4000220024A04EF67D730022032100904F2023
:102E5000FFF7E1F99BE00F4890F82200062804D024
:102E60000C4890F8220000280CD10020094981F874
:102E7000220001A84EF67D730022032100904F200E
:102E8000FFF7C9F983E0C8E08096980040420F0040
:102E9000A0860100A003002058040020FE040020AA
:102EA000B012002030303030303030303030000060
:102EB000F2000020C0000020ED000020CEDED0A7F0
:102EC000B4CECAFD00000000D3D0D0A7B4CECAFD56
:102ED00000000000202020005DE0FFE7FE480078B1
:102EE0000C2854D1FD48007C012850D1FC48807E3C
:102EF000012811D1FBA04EF67D7300220121009024
:102F00000420FFF788F9F948448D032301AA2046DD
:102F10000021FFF7B0FA10E0F5A04EF67D73002215
:102F2000012100900420FFF776F9F048048D032377
:102F300001AA20460021FFF79EFAE94890F82200F6
:102F400001280ED10220E64981F82200AFF27C0070
:102F50004EF67D730022012100901D20FFF75BF9E2
:102F600015E0DF4890F8220020B1DD4890F82200FB
:102F700006280CD10020DA4981F8220001A84EF67B
:102F80007D730022012100901D20FFF744F90020ED
:102F9000D34981F82300D24890F8380001283CD169
:102FA000CF48007F012812D1CD4890F83700012882
:102FB0000DD10220CA4981F83700CFA04EF67D73AB
:102FC0000022042100901D20FFF725F921E0C448CC
:102FD000007F012804D1C24890F83700062803D0AA
:102FE000BF4890F83700A0B90020BD4981F83700EC
:102FF000BE480489022301AA20460021FFF73BFABC
:1030000001A84EF67D730022042100901D20FFF7D9
:1030100002F90020B24981F838001FBD08B54EF60C
:103020007D70F7F77DFDB5A04EF67D730022062179
:1030300000901420FFF74FF9B4A04EF67D730022E4
:10304000022100901420FFF746F908BD7FB5AFF2CA
:10305000AC1207CA01AB07C3002500244EF67D70F1
:10306000F7F75EFDFFF7FBFDFFF7C6FDFFF7D9FDA4
:103070001722FF210846F7F7B8FDA8A04EF67D738A
:103080000022072100900420FFF7C5F8A548008A18
:103090000A2190FBF1F084B2032301AA204600210B
:1030A000FFF7E9F901A84EF67D7300220721009091
:1030B0001E20FFF7B0F89CA04EF67D73002207217A
:1030C00000903020FFF7A7F89648008A0A2190FB6D
:1030D000F1F201FB120084B2012301AA2046002173
:1030E000FFF7C9F901A84EF67D7300220721009071
:1030F0003620FFF790F88DA04EF67D730022072151
:1031000000903F20FFF787F88948008820B900BF6A
:1031100000208849087001E086480578032301AA49
:1031200028460021FFF7A7F901A84EF67D7300227B
:10313000072100905620FFF76EF87FA04EF67D73B2
:103140000022072100906820FFF765F8032301AAF9
:103150007A4800880021FFF78EF901A84EF67D73AA
:103160000022072100906E20FFF755F874A04EF65C
:103170007D730022052100900420FFF74CF8694878
:103180000688032301AA30460021FFF774F901A83D
:103190004EF67D730022052100901F20FFF73BF8BB
:1031A00062A04EF67D730022052100903320FFF7C8
:1031B00032F865A04EF67D73002205210090402074
:1031C000FFF729F857484688022301AA3046002114
:1031D000FFF751F901A84EF67D73002205210090FA
:1031E0006620FFF718F851A04EF67D7300220521E6
:1031F00000907720FFF70FF855A04EF67D73002260
:10320000032100900420FFF706F8464880880A2131
:1032100090FBF1F084B2022301AA20460021FFF7BF
:103220002AF901A84EF67D730022032100901C208C
:10323000FEF7F1FF3CA04EF67D73002203210090C3
:103240002820FEF782FF374880880A2190FBF1F2A0
:1032500001FB120084B2012301AA20460021FFF7DE
:103260000AF901A84EF67D730022032100902D205B
:10327000FEF7D1FF2DA04EF67D73002203210090B2
:103280003320FEF7C8FF34A04EF67D7300220321E1
:1032900000904020FEF7BFFF2248C0880A2190FB23
:1032A000F1F084B2022301AA20460021FFF7E3F8DF
:1032B00001A84EF67D730022032100905A20FEF7EC
:1032C000AAFF19A04EF67D7300220321009066200C
:1032D000FEF73BFF134843E0ED000020FE04002012
:1032E000A0030020CEDED0A700000000580400207C
:1032F000D3D0D0A70000000020200000B8C4C9C669
:10330000D2BDC1C6CCE5D1E900000000BAC7BBA45C
:10331000C9FAC3FCBDA1BFB500000000D2D1CAE408
:1033200000000000940900202E0000006D6C0000D9
:103330009C000020E80000202F000000A2000020D8
:10334000D7DCC1BF00000000CAD7B4CEC1BF0000A7
:10335000B3D6D0F800000000D7B7BCD300000000FF
:10336000C0880A2190FBF1F201FB120084B2012314
:1033700001AA20460021FFF77EF801A84EF67D73D2
:103380000022032100906B20FEF745FFAFF264009E
:103390004EF67D730022032100907720FEF73BFF5D
:1033A000FEA04EF67D730022012100900420FEF75E
:1033B00032FFFC480689022301AA30460021FFF7AC
:1033C0005AF801A84EF67D730022012100901E20BC
:1033D000FEF721FFF4A04EF67D730022012100903C
:1033E0002D20FEF718FFF1A04EF67D73002201217B
:1033F00000904020FEF70FFFEA484689032301AA08
:1034000030460021FFF737F801A84EF67D73002201
:10341000012100906420FEF7FEFEAFF2F0004EF6B0
:103420007D730022012100907720FEF7F4FE7FBD1E
:103430001FB5AFF2905207CA01AB07C34EF67D70BD
:10344000F7F76EFBFFF70BFCFFF7D6FBFFF7E9FB87
:103450001722FF210846F7F7C8FBD6A04EF67D736A
:103460000022072100900420FEF7D5FECD48848974
:10347000032301AA20460021FEF7FDFF01A84EF616
:103480007D730022072100905220FEF7C4FECDA0DC
:103490004EF67D730022052100900420FEF7BBFE4E
:1034A000C048C489032301AA20460021FEF7E3FF98
:1034B00001A84EF67D730022052100905220FEF7F0
:1034C000AAFEB848847C022301AA20460021FEF708
:1034D000D2FF01A84EF67D73002203210090042044
:1034E000FEF799FEBBA04EF67D73002203210090EB
:1034F0001020FEF790FEAB48C47C022301AA2046B0
:103500000021FEF7B8FF01A84EF67D7300220321CB
:1035100000901C20FEF77FFEAFA04EF67D730022C8
:10352000032100902820FEF776FE9E48047D0223AA
:1035300001AA20460021FEF79EFF01A84EF67D73EA
:103540000022032100903420FEF765FEA3A04EF672
:103550007D730022032100904020FEF75CFE91481D
:10356000447D022301AA20460021FEF784FF01A822
:103570004EF67D730022032100904620FEF74BFE9D
:1035800097A04EF67D730022032100905420FEF791
:1035900042FE8448847D022301AA20460021FEF7D2
:1035A0006AFF01A84EF67D730022012100900420DD
:1035B000FEF731FE87A04EF67D73002201210090B8
:1035C0001020FEF728FE7748C47D022301AA20467A
:1035D0000021FEF750FF01A84EF67D730022012165
:1035E00000901C20FEF717FE7BA04EF67D73002294
:1035F000012100902820FEF70EFE6A48047E022377
:1036000001AA20460021FEF736FF01A84EF67D7381
:103610000022012100903420FEF7FDFD6FA04EF640
:103620007D730022012100904020FEF7F4FD5D48EB
:10363000447E022301AA20460021FEF71CFF01A8B8
:103640004EF67D730022012100904620FEF7E3FD37
:103650005448807E092856D2DFE800F055050F193E
:10366000232D37414B0060A04EF67D7300220121CF
:1036700000905420FEF7CFFD4FE05EA04EF67D7324
:103680000022012100905420FEF7C5FD45E05BA01B
:103690004EF67D730022012100905420FEF7BBFD01
:1036A0003BE058A04EF67D7300220121009054208B
:1036B000FEF7B1FD31E056A04EF67D7300220121E8
:1036C00000905420FEF7A7FD27E054A04EF67D732E
:1036D0000022012100905420FEF79DFD1DE052A024
:1036E0004EF67D730022012100905420FEF793FDD9
:1036F00013E050A04EF67D7300220121009054206B
:10370000FEF789FD09E04EA04EF67D7300220121EF
:1037100000905420FEF77FFD00BF00BF1FBD2DE9C4
:10372000FC41AFF678000068019000254EF67D70F0
:10373000F7F7F6F9FFF793FAFFF75EFAFFF771FA7A
:1037400041A04EF67D730022062100900846FEF748
:1037500062FDA84616E03D4911F8080001A9FEF7F0
:103760005FFE01A808EB48011E22009002EB8100D9
:103770004EF67D7300220621FEF74DFD08F1010093
:1037800000F0FF08B8F1080FE5DB31A04EF67D73BD
:10379000002203210090062060E00000CBF8CAB1AF
:1037A00000000000940900206D696E00BCABCFDE04
:1037B000D6B50000D7B7BCD3D3D0D0A7B4CECAFDFE
:1037C00000000000D7B7BCD3CEDED0A7B4CECAFD70
:1037D00000000000D4C20000C8D500003A0000007C
:1037E000B9D8BBFA00000000BBFAD0B5B9CAD5CF32
:1037F00000000000B6C2C8FB00000000BCABCFDE7A
:1038000000000000C6F8C5DDCEDED2BA0000000020
:10381000CEB4D7B0D2A9BAD000000000B5E7C1BF7E
:10382000BAC4BEA100000000B9DCB5C0CDD1C2E46D
:1038300000000000CAE4D2BABDE1CAF800000000EE
:10384000CEDEB1A8BEAF000049443A00A904002072
:10385000D7DCCAA3D3E0C1BFA3BA0000FEF7DBFCEC
:10386000FE48806BFE49081A0A21B0FBF1F542F2CE
:103870001070B5FBF0F0D8B3052301AA284600214B
:10388000FEF7F9FD01A84EF67D730022032100909A
:103890003C20FEF7C0FCAFF270504EF67D73002264
:1038A000032100905A20FEF7B6FCEC48806BEC49EF
:1038B000081A0A21B0FBF1F201FB1204012301AA4C
:1038C00020460021FEF7D7FD01A84EF67D730022A9
:1038D000032100905E20FEF79EFCAFF2B0504EF642
:1038E0007D730022032100906420FEF794FCFFE02A
:1038F000FFE74FF47A70B5FBF0F0D8B3042301AAC8
:1039000028460021FEF7B7FD01A84EF67D73002280
:10391000032100903C20FEF77EFCAFF2F4504EF6FF
:103920007D730022032100905420FEF774FCCB48E5
:10393000806BCB49081A0A21B0FBF1F201FB12049B
:10394000012301AA20460021FEF795FD01A84EF6AD
:103950007D730022032100905820FEF75CFCAFF23B
:1039600034604EF67D730022032100905E20FEF746
:1039700052FCBDE0FFE76420B5FBF0F0D8B30323B1
:1039800001AA28460021FEF776FD01A84EF67D73B8
:103990000022032100903C20FEF73DFCAFF278604E
:1039A0004EF67D730022032100904E20FEF733FC7B
:1039B000AA48806BAA49081A0A21B0FBF1F201FB60
:1039C0001204012301AA20460021FEF754FD01A89C
:1039D0004EF67D730022032100905220FEF71BFC5F
:1039E000AFF2B8604EF67D7300220321009058209C
:1039F000FEF711FC7CE0FFE70A20B5FBF0F0D8B33E
:103A0000022301AA28460021FEF735FD01A84EF643
:103A10007D730022032100903C20FEF7FCFBAFF2F7
:103A2000F8604EF67D730022032100904820FEF7D7
:103A3000F2FB8A48806B8A49081A0A21B0FBF1F22E
:103A400001FB1204012301AA20460021FEF713FD09
:103A500001A84EF67D730022032100904C20FEF752
:103A6000DAFBAFF238704EF67D730022032100902E
:103A70005220FEF7D0FB3BE0FFE7012301AA2846D6
:103A80000021FEF7F8FC01A84EF67D730022032109
:103A900000903C20FEF7BFFBAFF274704EF67D73D2
:103AA0000022032100904220FEF7B5FB6B48806B9B
:103AB0006B49081A0A21B0FBF1F201FB1204012341
:103AC00001AA20460021FEF7D6FC01A84EF67D7320
:103AD0000022032100904620FEF79DFBAFF2B47058
:103AE0004EF67D730022032100904C20FEF793FBDD
:103AF0005CA04EF67D730022012100900620FEF7A7
:103B00008AFB5A4800884FF47A7190FBF1F0C11794
:103B10000646012301AAFEF7AEFC01A84EF67D730E
:103B20000022012100903020FEF775FBAFF608005F
:103B30004EF67D730022012100903620FEF76BFBCC
:103B40004A4800884FF47A7190FBF1F201FB1200B1
:103B5000642190FBF1F0C1170646012301AAFEF78C
:103B60008AFC01A84EF67D730022012100903C20C2
:103B7000FEF751FBAFF650004EF67D730022012197
:103B800000904220FEF747FB38480088642190FBF4
:103B9000F1F201FB12000A2190FBF1F0C117064679
:103BA000012301AAFEF767FC01A84EF67D730022EF
:103BB000012100904820FEF72EFBAFF694004EF650
:103BC0007D730022012100904E20FEF724FB274840
:103BD00000880A2190FBF1F201FB1200C117064692
:103BE000012301AAFEF747FC01A84EF67D730022CF
:103BF000012100905420FEF70EFBBDE8FC811FB5AB
:103C0000AFF6605207CA01AB07C319480078012814
:103C10007ED14EF67D70F6F783FFFFF720F8FEF7B2
:103C2000EBFFFEF7FEFF182201210020F6F7DDFF73
:103C300010480488042301AA20460021FEF71BFC3B
:103C400001A84EF67D730022062100900D20FEF79C
:103C500042FB09A04EF67D7300220FE058040020BD
:103C6000F0490200B0E6B1BEA3BA5600F40000204D
:103C70004B0000202A000020C4EA0000062100902A
:103C80002D20FEF728FBFE488478022301AA204657
:103C90000021FEF7F0FB01A84EF67D7300220621FD
:103CA00000903D20FEF717FBAFF2D8404EF67D7333
:103CB0000022062100904D20FEF70DFBF048C4784D
:103CC000022301AA20460021FEF7D5FB01A84EF6EB
:103CD0007D730022062100905D20FEF7FCFAAFF212
:103CE00008504EF67D730022062100906D20FEF7ED
:103CF000F2FAE3484479022301AA20460021FEF7A4
:103D0000BAFB01A84EF67D7300220221009000E06C
:103D100021E02D20FEF7DFFAAFF240504EF67D7322
:103D20000022022100904120FEF7D5FAD448847980
:103D3000022301AA20460021FEF79DFB01A84EF6B2
:103D40007D730022022100904D20FEF7C4FA02206C
:103D5000CC4908705AE0FEF782FFFEF74DFFFEF7F0
:103D600060FFC7480488042301AA20460021FEF70B
:103D700082FB01A84EF67D730022062100900D20E3
:103D8000FEF7A9FABE488478022301AA2046002142
:103D9000FEF771FB01A84EF67D730022062100900C
:103DA0003D20FEF798FAB648C478022301AA2046BF
:103DB0000021FEF760FB01A84EF67D73002206216C
:103DC00000905D20FEF787FAAD484479022301AAEE
:103DD00020460021FEF74FFB01A84EF67D7300221E
:103DE000022100902D20FEF776FAA548847902235F
:103DF00001AA20460021FEF73EFB01A84EF67D7386
:103E00000022022100904D20FEF765FA1FBD1FB56C
:103E1000AFF6707207CA01AB07C39A480078012851
:103E20007DD14EF67D70F6F77BFEFEF718FFFEF7AC
:103E3000E3FEFEF7F6FE182201210020F6F7D5FE7C
:103E40005E22FF210846F6F7D0FE8FA04EF67D7366
:103E50000022072100900520FEF7DDF98DA04EF627
:103E60007D730022032100900F20FEF76EF9844835
:103E70000488042301AA20460021FEF7FCFA01A8C9
:103E80004EF67D730022052100900D20FEF7C3F948
:103E9000AFF21C204EF67D730022052100902D20EC
:103EA000FEF7B9F976488478022301AA204600215A
:103EB000FEF7E1FA01A84EF67D730022052100907D
:103EC0003D20FEF7A8F9AFF2F4604EF67D730022B4
:103ED000052100904D20FEF79EF96948C478022321
:103EE00001AA20460021FEF7C6FA01A84EF67D730E
:103EF0000022052100905D20FEF78DF9AFF22870B9
:103F00004EF67D730022052100906D20FEF783F9A7
:103F10005B484479022301AA2046002100E029E001
:103F2000FEF7A9FA01A84EF67D7300220221009047
:103F30002D20FEF770F9AFF25C704EF67D73002213
:103F4000022100904120FEF766F94D488479022352
:103F500001AA20460021FEF78EFA01A84EF67D73D5
:103F60000022022100904D20FEF755F9022045491C
:103F7000087087E1FEF773FEFEF73EFEFEF751FE86
:103F800046480078062879D2DFE800F0780346B486
:103F9000FAF843480488042301AA20460021FEF7CA
:103FA0006AFA01A84EF67D730022052100900D20CB
:103FB000FEF731F937A04EF67D7300220321009001
:103FC0000F20FEF7C2F8AFF6D0404EF67D73002208
:103FD000032100903E20FEF7B8F8AFF6E4404EF61D
:103FE0007D730022032100905E20FEF7AEF8AFF64D
:103FF000F8404EF67D730022114600902E20FEF709
:10400000A4F8AFF60C504EF67D73002211460090D6
:104010004E20FEF79AF834E121488478022301AA61
:1040200020460021FEF727FA01A84EF67D730022F4
:10403000052100903D20FEF7EEF81948C4780223D0
:1040400001AA20460021FEF716FA01A84EF67D735C
:104050000022052100905D20FEF7DDF811A04EF64C
:104060007D730022032100900F20FEF76EF80FA051
:104070004EF67D7300220321009019E000E100005C
:104080002A0000204B000020CAB1BCE4C8B7C8CF4A
:10409000000000002D2D2D2D000000003800002014
:1040A0003A00002020202020000000002D2D0000DC
:1040B0003E20FEF74AF8AFF6C0504EF67D73002260
:1040C000032100905E20FEF740F8AFF6D4504EF684
:1040D0007D730022114600902E20FEF736F8AFF6D1
:1040E000E8504EF67D730022114600904E20FEF7F8
:1040F0002CF8C6E0FE48C478022301AA204600211D
:10410000FEF7B9F901A84EF67D7300220521009053
:104110005D20FEF780F8AFF274004EF67D7300224A
:10412000032100900F20FEF710F8AFF634604EF632
:104130007D730022032100903E20FEF706F8AFF2C7
:1041400094004EF67D730022032100905E20FDF75F
:10415000FCFFAFF65C604EF67D73002211460090C6
:104160002E20FDF7F2FFAFF670604EF67D73002251
:10417000114600904E20FDF7E8FF82E040E0FFE7A7
:10418000DB484479022301AA20460021FEF773F997
:1041900001A84EF67D730022022100902D20FEF72B
:1041A0003AF8D4A04EF67D730022032100900F2030
:1041B000FDF7CBFFD1484EF67D730022032100901E
:1041C0003E20FDF7C2FFCD484EF67D73002203214D
:1041D00000905E20FDF7B9FFAFF230104EF67D7310
:1041E0000022114600902E20FDF7AFFFC3484EF687
:1041F0007D730022114600904E20FDF7A6FF40E09F
:10420000BB488479022301AA20460021FEF733F936
:1042100001A84EF67D730022022100904D20FDF78B
:10422000FAFFB4A04EF67D730022032100900F2008
:10423000FDF78BFFB1484EF67D73002203210090FD
:104240003E20FDF782FFAD484EF67D73002203212C
:1042500000905E20FDF779FFA8484EF67D7300229E
:10426000114600902E20FDF770FFAFF2C0104EF601
:104270007D730022114600904E20FDF766FF00E09E
:1042800000BF00BF1FBD7FB59C4A303A07CA01ABD3
:1042900007C39B48007801285FD14EF67D70F6F782
:1042A0003FFCFEF7DCFCFEF7A7FCFEF7BAFC5C2245
:1042B000FF210846F6F799FC92A04EF67D73002286
:1042C000052100901920FDF7A6FF91A04EF67D7301
:1042D0000022042100904E20FDF737FF002414E057
:1042E0008C48055D012301AA28460021FEF7C3F88A
:1042F00001A84E21009001EBC4004EF67D73002210
:104300000521FDF722FF601CC4B2032CE8DB82A06C
:104310004EF67D730022022100901920FDF77BFFED
:10432000002414E07F48055D012301AA28460021EE
:10433000FEF7A1F801A84E21009001EBC4004EF653
:104340007D7300220221FDF700FF601CC4B2032C24
:10435000E8DB02206A490870C0E1FEF780FCFEF746
:104360004BFCFEF75EFC70480078072873D2DFE84C
:1043700000F072043B73AAFDFC0065A04EF67D734D
:104380000022042100904E20FDF7DFFE5AA04EF6D9
:104390007D730022042100905620FDF7D6FE56A022
:1043A0004EF67D730022042100905E20FDF7CDFEC5
:1043B00051A04EF67D730022012100904E20FDF7A2
:1043C000C4FE4DA04EF67D730022012100905620C0
:1043D000FDF7BBFE48A04EF67D7300220121009040
:1043E0005E20FDF7B2FE46E143A04EF67D7300224B
:1043F000042100904E20FDF7A8FE45A04EF67D73E7
:104400000022042100905620FDF79FFE3AA04EF6B0
:104410007D730022042100905E20FDF796FE36A0F9
:104420004EF67D730022012100904E20FDF78DFE97
:1044300031A04EF67D730022012100905620FDF739
:1044400084FE2DA04EF67D730022012100905E2097
:10445000FDF77BFE0FE10DE127A04EF67D730022F4
:10446000042100904E20FDF770FE23A04EF67D73D0
:104470000022042100905620FDF767FE24A04EF68E
:104480007D730022042100905E20FDF75EFE1AA0DD
:104490004EF67D730022012100904E20FDF755FE5F
:1044A00015A04EF67D730022012100905620FDF7E5
:1044B0004CFE11A04EF67D730022012100905E207B
:1044C000FDF743FED7E00CA04EF67D7300220421D9
:1044D00000904E20FDF739FE07A04EF67D730022B6
:1044E000042100905620FDF730FE03A01EE00000DE
:1044F0003A0000202020202020000000D42E0108B7
:104500004B000020C9E8D6C3C3DCC2EB00000000AA
:104510005F00000042000020C8B7C8CFC3DCC2EB78
:104520000000000045000020F20000204EF67D73E0
:104530000022042100905E20FDF707FEAFF230005C
:104540004EF67D730022012100904E20FDF7FDFD07
:10455000AFF25C004EF67D730022012100905620E0
:10456000FDF7F3FDAFF2700001E046E008E04EF623
:104570007D730022012100905E20FDF7E6FD7AE0C8
:10458000AFF28C004EF67D730022042100904E2085
:10459000FDF7DBFDAFF2A0004EF67D730022042193
:1045A00000905620FDF7D1FDAFF2B4004EF67D73BA
:1045B0000022042100905E20FDF7C7FDAFF2C80085
:1045C0004EF67D730022012100904E20FDF7BDFDC7
:1045D000AFF2C4004EF67D730022012100905620F8
:1045E000FDF7B3FDAFF2F0004EF67D73002201211E
:1045F00000905E20FDF7A9FD3DE0AFF204104EF6FD
:104600007D730022042100904E20FDF79EFDAFF245
:1046100018104EF67D730022042100905620FDF7FD
:1046200094FDAFF22C104EF67D7300220421009011
:104630005E20FDF78AFDAFF240104EF67D7300223A
:10464000012100904E20FDF780FDAFF254104EF690
:104650007D730022012100905620FDF776FDAFF218
:1046600050104EF67D730022012100905E20FDF770
:104670006CFD00E000BF00BF002414E0FC48055DB5
:10468000012301AA28460021FDF7F5FE01A84E21CD
:10469000009001EBC4004EF67D7300220521FDF76A
:1046A00054FD601CC4B2032CE8DB002414E0F14884
:1046B000055D012301AA28460021FDF7DCFE01A8C3
:1046C0004E21009001EBC4004EF67D7300220221C2
:1046D000FDF73BFD601CC4B2032CE8DB7FBD7FB55A
:1046E000E54A07CA01AB07C30024E4480078012863
:1046F0007ED14EF67D70F6F713FAFEF7B0FAFEF7AC
:104700007BFAFEF78EFADEA04EF67D7300220721BB
:1047100000900420FDF77FFDDCA04EF67D730022A3
:10472000042100900846FDF776FDDA488378DA48E0
:1047300001AAD0E902512846FDF79DFE01A84EF6D8
:104740007D730022042100902E20FDF764FDD3A08C
:104750004EF67D730022022100900420FDF75BFDE0
:10476000AFF2B8604EF67D730022022100901C204B
:10477000FDF751FDCBA04EF67D7300220221009083
:104780002820FDF748FDC4484588C248037801AA9F
:1047900028460021FDF76FFE01A84EF67D7300222A
:1047A000022100904020FDF736FDBA48007800EB6A
:1047B0004000402101EB4000C4B2AFF210704EF651
:1047C0007D730022022100902046FDF724FD04F1B4
:1047D0000C00C4B2B0488588AE48437801AA284688
:1047E0000021FDF748FE01A84EF67D73002200E08F
:1047F00033E0022100902046FDF70DFDA648007829
:10480000012813D1A9A04EF67D7300220421009047
:104810007120FDF700FD984830304EF67D73002280
:10482000022100907120FDF7F6FC12E09248303032
:104830004EF67D730022042100907120FDF7EBFC01
:104840009AA04EF67D730022022100907120FDF7A0
:10485000E2FC02208949087034E0FEF700FAFEF716
:10486000CBF9FEF7DEF98C480078012813D18FA030
:104870004EF67D730022042100907120FDF7CBFCE1
:104880007D4830304EF67D73002202210090712069
:10489000FDF7C1FC16E080480078022812D1764866
:1048A00030304EF67D730022042100907120FDF718
:1048B000B2FC7EA04EF67D73002202210090712092
:1048C000FDF7A9FC7FBD7FB56B4A07CA01AB07C3E3
:1048D00000256A480078012876D14EF67D70F6F7FB
:1048E0001FF9FEF7BCF9FEF787F9FEF79AF95E2289
:1048F000FF210846F6F779F967480078012809D1C1
:104900006BA04EF67D730022032100903820FDF746
:104910004FFC0CE060480078022808D164A04EF6F5
:104920007D730022012100904C20FDF741FC54A032
:104930004EF67D730022072100900A20FDF76BFCE4
:1049400052A04EF67D730022042100900A20FDF74C
:1049500062FC002416E05748065D012301AA304698
:104960000021FDF788FD01A804EB440138220090E6
:1049700002EB41004EF67D7300220421FDF718FC86
:10498000601CC4B243488078A042E4DC43A04EF6E9
:104990007D730022022100900A20FDF73CFCAFF657
:1049A000F4004EF67D730022022100902220FDF7D4
:1049B00032FC3CA04EF67D730022022100902E2096
:1049C000FDF729FC002418E076E03A48801F065DD8
:1049D000012301AA30460021FDF74DFD01A804EB9B
:1049E00044014C22009002EB41004EF67D73002200
:1049F0000221FDF7DDFB601CC4B226480078A0420E
:104A0000E3DC2448007800EB40004C2101EB40003F
:104A1000C5B2AFF668104EF67D73002202210090F9
:104A20002846FDF7C5FB05F10C00C5B2002416E0D1
:104A30002048C01E065D012301AA30460021FDF773
:104A40001AFD01A804EB4401009005EB41004EF66D
:104A50007D7300220221FDF7ABFB601CC4B20D4840
:104A60004078A042E4DC0220044908708EE1000096
:104A70004200002045000020A42E01084B00002029
:104A8000C7EBC8B7C8CFD0C5CFA20000D7A1D4BA52
:104A9000BAC50000FE04002098040020B2A1C7F8A7
:104AA00000000000B4B2BAC5000000003C3D3D006B
:104AB0002D000000C6040020FEF7D1F8FEF79CF898
:104AC000FEF7AFF8FE480078012802D002286ED128
:104AD000A9E0002424E0AFF2E05004EB44013822C6
:104AE000009002EB41004EF67D7300220321FDF79A
:104AF0005FFBF448065D012301AA30460021FDF763
:104B0000BAFC01A804EB44013822009002EB4100FA
:104B10004EF67D7300220421FDF74AFB601CC4B2EF
:104B2000E9488078A042D6DCE84800780B2877D2A4
:104B3000DFE800F07606111C27323E49545F6A0018
:104B4000AFF294004EF67D730022032100903820CE
:104B5000FDF72EFB65E0AFF2A8004EF67D73002254
:104B6000032100903E20FDF723FB5AE0AFF2C00086
:104B70004EF67D730022032100904420FDF718FBC0
:104B80004FE0AFF2D4004EF67D7300220321009077
:104B90004A20FDF70DFB44E0AFF2EC004EF67D73CA
:104BA0000022032100905020FDF702FB39E0EBE0EA
:104BB000AFF204104EF67D730022032100905620C0
:104BC000FDF7F6FA2DE0AFF218104EF67D730022D5
:104BD000032100905C20FDF7EBFA22E0AFF23010E9
:104BE0004EF67D730022032100906220FDF7E0FA6B
:104BF00017E0AFF244104EF67D73002203210090BF
:104C00006820FDF7D5FA0CE0AFF25C104EF67D732C
:104C10000022032100906E20FDF797FA01E0FFE7E4
:104C200000BF00BFB1E0002447E0A648801F065D3A
:104C3000012301AA30460021FDF71DFC01A804EB69
:104C400044014C22009002EB41004EF67D7300229D
:104C50000221FDF7ADFAAFF2607004EB44014C2283
:104C6000009002EB41004EF67D7300220121FDF71A
:104C70009FFA96480078401EA0420ED1AFF2D010A5
:104C800004EB44014C22009002EB41004EF67D7390
:104C900000220121FDF78CFA0DE0AFF2A47004EBC5
:104CA00044014C22009002EB41004EF67D7300223D
:104CB0000121FDF77DFA601CC4B283480078A04250
:104CC000B3DC8148007800EB40004C2101EB400050
:104CD000C5B2AFF628404EF67D7300220221009047
:104CE0002846FDF765FA05F10C00C5B2002446E040
:104CF000AFF2FC7004EB4401009005EB41004EF66E
:104D00007D7300220121FDF753FA6E48C01E065D37
:104D1000012301AA30460021FDF7ADFB01A804EBF9
:104D20004401009005EB41004EF67D730022022104
:104D3000FDF73EFA64480078011964480078401E87
:104D400081420DD1AFF2982004EB4401009005EBB5
:104D500041004EF67D7300220121FDF729FA0CE097
:104D6000AFF66C0004EB4401009005EB41004EF6F9
:104D70007D7300220121FDF71BFA601CC4B252486A
:104D80004078A042B4DC00E000BF00BF7FBD08B5A2
:104D90004EF67D70F5F7C4FE4DA04EF67D730022F1
:104DA000042100901920FDF736FA08BD1FB54C4AC2
:104DB00007CA01AB07C300244A480078012862D122
:104DC0004EF67D70F5F7ACFEFDF749FFFDF714FFD9
:104DD000FDF727FF0622FF210846F5F706FF42A050
:104DE0004EF67D730022052100902C20FDF773FA0A
:104DF0003F48008840F2E731884202DB08463C49E0
:104E000008803B4800880A2190FBF1F084B202231D
:104E100001AA20460021FDF72EFB01A84EF67D7366
:104E20000022022100902C20FDF755FA31A04EF609
:104E30007D730022022100903C20FDF74CFA2C48A3
:104E400000880A2190FBF1F201FB120084B20123D9
:104E500001AA20460021FDF70EFB01A84EF67D7346
:104E60000022022100904420FDF735FA22A04EF6E0
:104E70007D730022022100904E20FDF72CFA0220C3
:104E80001849087072E0FDF7EAFEFDF7B5FEFDF780
:104E9000C8FE0522FF210846F5F7A7FE1448008842
:104EA00040F2E731884202DB084611490880104889
:104EB00000880A2190FBF1F084B2022301AA1DE0D0
:104EC00098040020C6040020FE040020F200002008
:104ED000C7EBC9E8D6C3D7A1D4BABAC52100000030
:104EE000A42E01084B000020C5C52020C6F80000F4
:104EF000580400202E0000006D6C000020460021A8
:104F0000FDF7B9FA01A84EF67D7300220221009048
:104F10002C20FDF7E0F9AFF224004EF67D7300225D
:104F2000022100903C20FDF7D6F9FE4800880A21B6
:104F300090FBF1F201FB120084B2012301AA20468A
:104F40000021FDF798FA01A84EF67D730022022198
:104F500000904420FDF7BFF9AFF264004EF67D7378
:104F60000022022100904E20FDF7B5F91FBD00B5CB
:104F700089B0ED49D1E900028968CDE907210690A1
:104F80000020059004900390E848007801287CD127
:104F90004EF67D70F5F7C4FDFDF761FEFDF72CFEC2
:104FA000FDF73FFE5E22FF210846F5F71EFEE048B2
:104FB0004EF67D730022072100900420FDF72BF9A7
:104FC000DC48008D64281CDB03200390039800EB71
:104FD0008000C0F11600029000EBD070C0F34700D3
:104FE0000490D4480078012848D1D3A000900498B8
:104FF0001C304EF67D73002206210290FDF7D8F892
:105000003CE0CC48008D0A281CDB0220039003986A
:1050100000EB8000C0F11600029000EBD070C0F3EE
:1050200047000490C3480078012827D1C3A000900E
:1050300004981C304EF67D73002206210290FDF785
:10504000B7F81BE001200390039800EB8000C0F14B
:105050001600029000EBD07040100490B548007824
:1050600001280BD1AFF65830009004981C304EF652
:105070007D73002206210290FDF79AF8AD48008D5D
:10508000029006AA0021039B00E0ECE2FDF7F3F991
:1050900006A8009004981C304EF67D73002207216C
:1050A0000290FDF785F8AFF2B0104EF67D73002246
:1050B000072100903320FDF748F8A1A04EF67D733C
:1050C0000022072100904020FDF7A5F89948408D67
:1050D0000A281CDB02200390039800EB8000C0F13B
:1050E0001700029000EBD070C0F347000490914885
:1050F0000078022827D191A00090049858304EF6ED
:105100007D73002206210290FDF752F81BE001207A
:105110000390039800EB8000C0F11700029000EBB1
:10512000D070401004908348007802280BD1AFF66D
:1051300020400090049858304EF67D7300220621DE
:105140000290FDF735F87B48408D029006AA0021B9
:10515000039BFDF790F906A80090049858304EF68E
:105160007D73002207210290FDF722F8AFF278202C
:105170004EF67D730022072100906F20FCF7E5FFBB
:105180006B4818304EF67D730022042100900846CB
:10519000FDF741F8002003906648C08D0A2190FB7E
:1051A000F1F201FB120018B10398801CC0B2039009
:1051B0006048C08D642190FBF1F020B10398801C01
:1051C000C0B2039003E00398401CC0B20390039860
:1051D00000EB8000C0F11600029000EBD070C0F32D
:1051E000470004905348C08D0A2190FBF1F080B233
:1051F00005900598092811DD022003904D4800789C
:1052000004281DD14DA0009004981C304EF67D73EB
:10521000002203210290FCF7CBFF11E00120039054
:105220004448007804280BD1AFF61C500090049835
:105230001C304EF67D73002203210290FCF7B8FF6C
:1052400006AA0021039B0598FDF715F906A8009012
:1052500004981C304EF67D73002204210290FCF766
:10526000A7FF3448C08D0A2190FBF1F201FB120028
:1052700080B20590059890B304981C30039901EB17
:1052800081010844401CC0B204902A4800780428D8
:1052900008D12AA04EF67D730022032100900498C5
:1052A000FCF786FFAFF2B4304EF67D730022042186
:1052B00000900498FCF749FF0498401DC0B2049088
:1052C000012306AA00210598FDF7D5F806A84EF699
:1052D0007D730022042100900498FCF769FFAFF26F
:1052E000E8304EF67D730022042100903320FCF755
:1052F0002CFF0F4810304EF67D73002204210090E1
:105300004020FCF788FF002003900A48808D0A2186
:1053100090FBF1F201FB120018B10398801CC0B29F
:10532000039011E058040020A42E01084B00002037
:1053300040330108A80400205F5F5F005F5F00004A
:10534000CAD7B4CE00000000FE48808D642190FBD7
:10535000F1F020B10398801CC0B2039003E00398E1
:10536000401CC0B20390039800EB8000C0F117000E
:10537000029000EBD070C0F347000490F148808D9C
:105380000A2190FBF1F080B205900598092812DD02
:1053900002200390EB48007803281ED1AFF264008E
:1053A0000090049858304EF67D730022032102903D
:1053B000FCF7FEFE11E001200390E248007803288C
:1053C0000BD1AFF6B4600090049858304EF67D7360
:1053D000002203210290FCF7EBFE06AA0021039BAA
:1053E0000598FDF748F806A80090049858304EF646
:1053F0007D73002204210290FCF7DAFED148808DF3
:105400000A2190FBF1F201FB120080B20590059891
:1054100098B304985830039901EB81010844401C6B
:10542000C0B20490C7480078032809D1AFF2F40055
:105430004EF67D730022032100900498FCF7B8FE1D
:10544000AFF250504EF67D73002204210090049874
:10545000FCF77BFE0498401DC0B20490012306AA0D
:1054600000210598FDF707F806A84EF67D73002287
:10547000042100900498FCF79BFEB3A04EF67D73C8
:105480000022042100906F20FCF75FFEB0484EF62A
:105490007D730022012100900420FCF7BCFEA94886
:1054A000008E0A281DDB02200390039800EB800089
:1054B000C0F11100029000EBD070C0F347000490DF
:1054C000A0480078052828D1AFF2901000900498E9
:1054D0001C304EF67D73002211460290FCF768FEE8
:1054E0001BE001200390039800EB8000C0F1110045
:1054F000029000EBD070401004909248007805288C
:105500000BD1AFF6F470009004981C304EF67D730A
:10551000002211460290FCF74BFE8A48008E029052
:1055200006AA0021039BFCF7A6FF06A8009004989A
:105530001C304EF67D73002201210290FCF738FEEC
:1055400083480C304EF67D730022012100902E20FE
:10555000FCF7FBFD7E4860304EF67D730022012192
:1055600000904020FCF757FE7648408E64281DDBF3
:1055700003200390039800EB8000C0F11700029015
:1055800000EBD070C0F3470004906E480078062806
:1055900049D1AFF25C200090049858304EF67D73EC
:1055A000002211460290FCF703FE3CE06548408E65
:1055B0000A281DDB02200390039800EB8000C0F155
:1055C0001700029000EBD070C0F3470004905D48D4
:1055D0000078062827D1AFF29C200090049858301C
:1055E0004EF67D73002211460290FCF7E1FD1AE0B1
:1055F00001200390039800EB8000C0F11700029097
:1056000000EBD070401004904E48007806280AD174
:1056100050A00090049858304EF67D730022114639
:105620000290FCF7C5FD4748408E029006AA002173
:10563000039BFCF720FF06A80090049858304EF614
:105640007D73002201210290FCF7B2FD3EA04EF6D0
:105650007D730022012100906F20FCF776FD02206F
:105660003D4908700DE3FDF7FAFAFDF7C5FAFDF7BD
:10567000D8FA0123062232211C20F5F776FA0123FD
:1056800006226E215820F5F770FA012303223221F9
:105690001C20F5F76AFA012303226E215820F5F742
:1056A00064FA012300222D211C20F5F75EFA012364
:1056B00000226E215820F5F758FA22480078072872
:1056C0007ED2DFE800F07D0482FDD2FCFB001D48A5
:1056D000008D642819DB03200390039800EB800001
:1056E000C0F11600029000EBD070C0F347000490A8
:1056F000AFF2BC30009004981C304EF67D7300224F
:1057000006210290FCF754FD43E00E48008D0A2864
:1057100027DB02200390039800EB8000C0F1160005
:10572000029000EBD070C0F347000490AFF2F43069
:10573000009004981C304EF67D73002206210290E2
:105740000CE00000A80400206D6C2F680000000031
:105750009C3701085F0000004B000020FCF728FD8B
:1057600017E001200390039800EB8000C0F11600C1
:10577000029000EBD07040100490AFF2280000902F
:1057800004981C304EF67D73002206210290FCF72F
:105790000FFD0123072232211C20F5F7E6F9FE4810
:1057A000008D029006AA0021039BFCF764FE06A868
:1057B000009004981C304EF67D730022072100E013
:1057C0005DE20290FCF7F4FC5AE2F348408D0A28AF
:1057D00019DB02200390039800EB8000C0F1170052
:1057E000029000EBD070C0F347000490AFF2B440D9
:1057F0000090049858304EF67D73002206210290E6
:10580000FCF7D6FC17E001200390039800EB800022
:10581000C0F11700029000EBD07040100490AFF27E
:10582000CC000090049858304EF67D73002206217B
:105830000290FCF7BDFC012307226E215820F5F7EA
:1058400094F9D548408D029006AA0021039BFCF7ED
:1058500012FE06A80090049858304EF67D73002280
:1058600007210290FCF7A4FC0AE200200390CA483A
:10587000C08D0A2190FBF1F201FB120018B10398D0
:10588000801CC0B20390C448C08D642190FBF1F02D
:1058900020B10398801CC0B2039003E00398401C21
:1058A000C0B20390039800EB8000C0F11600029094
:1058B00000EBD070C0F34700049002E071E11CE1FE
:1058C00079E00123042232211C20F5F74EF9B24879
:1058D000C08D0A2190FBF1F080B20590059809284F
:1058E0000EDD02200390AFF2AC50009004981C3003
:1058F0004EF67D73002203210290FCF759FC0DE067
:1059000001200390AFF2B410009004981C304EF6C2
:105910007D73002203210290FCF74AFC06AA0021B5
:10592000039B0598FCF7A7FD06A8009004981C307F
:105930004EF67D73002204210290FCF739FC964854
:10594000C08D0A2190FBF1F201FB120080B205909C
:10595000059878B304981C30039901EB8101084441
:10596000401CC0B20490AFF22C604EF67D73002252
:10597000032100900498FCF71BFCAFF688204EF63C
:105980007D730022042100900498FCF7DEFB04984C
:10599000401DC0B20490012306AA00210598FCF71F
:1059A0006AFD06A84EF67D7300220421009004983B
:1059B000FCF7FEFB64E1002003907748808D0A210C
:1059C00090FBF1F201FB120018B10398801CC0B2E9
:1059D00003907148818D642091FBF0F020B1039811
:1059E000801CC0B2039003E00398401CC0B2039037
:1059F000039800EB8000C0F11700029000EBD0701C
:105A0000C0F347000490012304226E215820F5F7CB
:105A1000ACF86148818D0A2091FBF0F080B20590CE
:105A2000059809280EDD02200390AFF2F060009087
:105A3000049858304EF67D73002203210290FCF743
:105A4000B7FB0DE001200390AFF2F820009004981E
:105A500058304EF67D73002203210290FCF7A8FB1C
:105A600006AA0021039B0598FCF705FD06A80090F7
:105A7000049858304EF67D73002204210290FCF702
:105A800097FB4548818D0A2291FBF2F002FB101032
:105A900080B20590059878B304985830039901EBCB
:105AA00081010844401CC0B20490AFF270704EF601
:105AB0007D730022032100900498FCF779FBAFF678
:105AC000CC304EF67D730022042100900498FCF740
:105AD0003CFB0498401DC0B20490012306AA00219B
:105AE0000598FCF7C8FC06A84EF67D730022042139
:105AF00000900498FCF75CFBC2E02748008E0A285F
:105B000019DB02200390039800EB8000C0F1110024
:105B1000029000EBD070C0F347000490AFF2E47045
:105B2000009004981C304EF67D73002211460290BE
:105B3000FCF73EFB17E001200390039800EB800088
:105B4000C0F11100029000EBD07040100490AFF251
:105B5000FC30009004981C304EF67D7300221146F4
:105B60000290FCF725FB01231A462D211C20F4F797
:105B7000FCFF0948008E029006AA0021039BFCF757
:105B80007AFC06A8009004981C304EF67D73002223
:105B90000121029002E00000A8040020FCF708FBAD
:105BA0006EE0FE48408E642819DB032003900398C2
:105BB00000EB8000C0F11700029000EBD070C0F342
:105BC00047000490AFF690000090049858304EF6CD
:105BD0007D73002211460290FCF7EAFA35E0EF48A7
:105BE000408E0A2819DB02200390039800EB800006
:105BF000C0F11700029000EBD070C0F34700049092
:105C0000AFF6C8000090049858304EF67D7300221D
:105C100011460290FCF7CCFA17E00120039003989C
:105C200000EB8000C0F11700029000EBD070401034
:105C30000490AFF2E0400090049858304EF67D7327
:105C4000002211460290FCF7B3FA01231A466E2196
:105C50005820F4F78AFFD148408E029006AA00210E
:105C6000039BFCF708FC06A80090049858304EF6F9
:105C70007D73002201210290FCF79AFA00E000BF38
:105C800000BF09B000BD7FB5C54A07CA01AB07C355
:105C90000024C44800780A287DD1C3480078012830
:105CA0007AD14EF67D70F4F73BFFC048407C012866
:105CB00005D15222FF210846F4F797FF04E0522253
:105CC00000210846F4F791FFB94890F82D00042808
:105CD00005D15122FF210846F4F787FF04E0512245
:105CE00000210846F4F781FFB04890F82000012811
:105CF00005D12222FF210846F4F777FF04E0222293
:105D000000210846F4F771FFFCF7A9FFFCF774FFC8
:105D1000FCF787FFA7A04EF67D73002206210090B6
:105D20002020FCF778FA9D48058D032301AA284618
:105D30000021FCF7A0FB01A84EF67D73002206218E
:105D400000905020FCF767FAAFF654604EF67D7372
:105D50000022062100906A20FCF75DFA97484EF673
:105D60007D730022032100902020FCF754FA904814
:105D700040880A2190FBF1F084B2022301AA204658
:105D80000021FCF778FB01A84EF67D730022032169
:105D90000090502001E0E7E030E0FCF73CFAAFF67D
:105DA000AC604EF67D730022032100905C20FCF76E
:105DB00032FA7F4840880A2190FBF1F201FB120081
:105DC00084B2012301AA20460021FCF754FB01A85C
:105DD0004EF67D730022032100906220FCF71BFA2F
:105DE000AFF6EC604EF67D730022032100906A202E
:105DF000FCF711FA02206C490870B5E07048007891
:105E00000028FAD16948407C012805D15222FF219F
:105E10000846F4F7EAFE04E0522200210846F4F7AF
:105E2000E4FE634890F82D00042805D15122FF219B
:105E30000846F4F7DAFE04E0512200210846F4F7A0
:105E4000D4FE5A4890F82000012805D12222FF21D3
:105E50000846F4F7CAFE04E0222200210846F4F7BF
:105E6000C4FEFCF7FCFEFCF7C7FEFCF7DAFE4B486D
:105E7000058D032301AA28460021FCF7FCFA01A89E
:105E80004EF67D730022062100905020FCF7C3F9E6
:105E9000474840880A2190FBF1F084B2022301AA0E
:105EA00020460021FCF7E7FA01A84EF67D73002298
:105EB000032100905020FCF7AEF9AFF6C8704EF603
:105EC0007D730022032100905C20FCF7A4F9384880
:105ED00040880A2190FBF1F201FB120084B20123F9
:105EE00001AA20460021FCF7C6FA01A84EF67D73F0
:105EF0000022032100906220FCF78DF900202B493D
:105F000088753048007C78BB042301AA2E4800889D
:105F10000021FCF7B0FA01A84EF67D7300220121A2
:105F200000901020FCF777F9042301AA2748008885
:105F30000021FCF7A0FA01A84EF67D730022012192
:105F400000903D20FCF767F9042301AA204800884F
:105F50000021FCF790FA01A84EF67D730022012182
:105F600000906A20FCF757F97FBD7FB50C4A07CA3D
:105F700001AB07C300240B4800780B287ED10A48E8
:105F8000007801287BD14EF67D70F4F7C9FD0748F3
:105F9000407C012822D15222FF211BE0A8040020CE
:105FA000A42E0108C00000204B000020A003002008
:105FB00058040020D7DC2020C1BF0000483301086E
:105FC00028000020FE040020640100204C01002075
:105FD0001C0100200846F4F708FE04E052220021CC
:105FE0000846F4F702FEFE4890F82D00042805D17B
:105FF0005122FF210846F4F7F8FD04E05122002168
:106000000846F4F7F2FDF74890F82000012805D182
:106010002222FF210846F4F7E8FD04E022220021B5
:106020000846F4F7E2FDFCF71AFEFCF7E5FDFCF785
:10603000F8FDED484EF67D73002207210090042004
:10604000FCF7E9F8E948058D032301AA2846002159
:10605000FCF711FA01A84EF67D730022072100908B
:106060001D20FCF7D8F8E2A04EF67D730022072130
:1060700000903020FCF7CFF8DB4801E0A3E235E1E7
:1060800024384EF67D730022072100903C20FCF757
:10609000C2F8D348808C0A2190FBF1F084B203232C
:1060A00001AA20460021FCF7E6F901A84EF67D730F
:1060B0000022072100905620FCF7ADF8CDA04EF647
:1060C0007D730022072100906820FCF7A4F8C448E3
:1060D000808C0A2190FBF1F201FB120084B20123B3
:1060E00001AA20460021FCF7C6F901A84EF67D73EF
:1060F0000022072100906E20FCF78DF8BCA04EF620
:106100007D730022072100907720FCF784F8BA48BD
:106110004EF67D730022042100900846FCF77BF8C0
:10612000AF480589022301AA28460021FCF7A3F9FC
:1061300001A84EF67D730022042100901D20FCF77B
:106140006AF8AD480C304EF67D73002204210090B1
:106150002A20FCF760F8A44818304EF67D73002220
:10616000042100903C20FCF756F8A44840890A21FD
:1061700090FBF1F084B2022301AA20460021FCF733
:106180007AF901A84EF67D7300220421009059206F
:10619000FCF741F897A04EF67D7300220421009091
:1061A0006520FCF738F8954840890A2190FBF1F208
:1061B00001FB120084B2012301AA20460021FCF752
:1061C0005AF901A84EF67D730022042100906B203D
:1061D000FCF721F886A04EF67D7300220421009082
:1061E0007720FCF718F88648007C01287AD17E4891
:1061F00010304EF67D730022012100903C20FCF708
:106200000AF87E48C0880A2190FBF1F084B202238C
:1062100001AA20460021FCF72EF901A84EF67D7355
:106220000022012100905420FBF7F5FF71A04EF6EB
:106230007D730022012100906020FBF7ECFF6F4886
:10624000C0880A2190FBF1F201FB120084B2012305
:1062500001AA20460021FCF70EF901A84EF67D7335
:106260000022012100906620FBF7D5FFAFF6283011
:106270004EF67D730022012100906C20FBF7CBFFCE
:106280005848807E012812D157485C384EF67D73FD
:106290000022012100900420FBF7BDFF5048458DEE
:1062A000032301AA28460021FCF7E5F811E04E4837
:1062B00050384EF67D730022012100900420FBF738
:1062C000AAFF4748058D032301AA28460021FCF7B1
:1062D000D2F801A84EF67D730022012100901D2006
:1062E000FBF799FF022047490870B2E14648007861
:1062F0000028FAD13B48407C012805D15222FF21D9
:106300000846F4F772FC04E0522200210846F4F734
:106310006CFC334890F82D00042805D15122FF2150
:106320000846F4F762FC04E0512200210846F4F725
:106330005CFC2C4890F82000012805D12222FF2186
:106340000846F4F752FC04E0222200210846F4F744
:106350004CFCFCF784FCFCF74FFCFCF762FC234888
:10636000058D032301AA28460021FCF784F801A823
:106370004EF67D730022072100901D20FBF74BFF96
:106380001748808C0A2190FBF1F084B2032301AA04
:1063900020460021FCF76FF801A84EF67D7300221D
:1063A000072100905620FBF736FF12A04EF67D73B2
:1063B0000022072100906820FBF72DFF0848808C01
:1063C0000A2190FBF1F201FB120084B2012301AA21
:1063D00020460021FCF74FF801A84EF67D7315E02A
:1063E00058040020A003002040330108A804002026
:1063F0006D6C00002E0000009C370108E4040020B2
:10640000FE0400204B00002028000020002207216D
:1064100000906E20FBF7FFFEFE48007F01280ED1A2
:10642000FC4890F83700012809D1FBA04EF67D7397
:106430000022042100901D20FBF7EDFE1DE0F54831
:10644000007F012804D1F34890F83700062803D0D4
:10645000F04890F8370080B9F0480589022301AA76
:1064600028460021FCF707F801A84EF67D730022AC
:10647000042100901D20FBF7CEFEE94840890A2147
:1064800090FBF1F084B2022301AA20460021FBF721
:10649000F2FF01A84EF67D730022042100905920DE
:1064A000FBF7B9FEAFF2B4004EF67D730022042173
:1064B00000906520FBF7AFFED94840890A2190FB88
:1064C000F1F201FB120084B2012301AA204600214F
:1064D000FBF7D1FF01A84EF67D7300220421009046
:1064E0006B20FBF798FECF48007C01287DD1CC487B
:1064F000C0880A2190FBF1F084B2022301AA204651
:106500000021FBF7B8FF01A84EF67D7300220121A0
:1065100000905420FBF77FFEAFF228104EF67D73FB
:106520000022012100906020FBF775FEBC48C08866
:106530000A2190FBF1F201FB120084B2012301AAAF
:1065400020460021FBF797FF01A84EF67D7300223D
:10655000012100906620FBF75EFEAE48807E012898
:1065600011D1B1484EF67D73002201210090042024
:10657000FBF751FEA948458D032301AA28460021B7
:10658000FBF779FF11E0A8480C304EF67D7300222E
:10659000012100900420FBF73EFEA048058D032357
:1065A00001AA28460021FBF766FF9A4890F82200CE
:1065B000012809D19D484EF67D73002201210090EB
:1065C0001D20FBF728FE44E0924890F8220020B1FD
:1065D000904890F8220006283BD101A84EF67D7322
:1065E0000022012100901D2000E002E0FBF713FED5
:1065F0002FE0042301AA8E4800880021FBF73BFF0F
:1066000001A84EF67D730022012100906A20FBF75D
:1066100002FE042301AA874800880021FBF72BFF14
:1066200001A84EF67D730022012100903D20FBF76A
:10663000F2FD042301AA804800880021FBF71BFF1C
:1066400001A84EF67D730022012100901020FBF777
:10665000E2FD7FBD7FB5754A303A07CA01AB07C37B
:106660007648007801287CD14EF67D70F4F758FA10
:10667000FCF7F5FAFCF7C0FAFCF7D3FA6548407C62
:10668000012805D15222FF210846F4F7AEFA04E0B2
:10669000522200210846F4F7A8FA604890F82D002D
:1066A000042805D15122FF210846F4F79EFA04E0A0
:1066B000512200210846F4F798FA61A04EF67D7346
:1066C0000022072100900420FBF7A5FD5DA04EF6F7
:1066D0007D730022012100905A20FBF79CFD5AA0F7
:1066E0004EF67D730022072100901120FBF7F3FD89
:1066F00056A04EF67D730022012100905020FBF73A
:10670000EAFD002407E004F1140001221146FBF722
:10671000B3FC601CC4B23C2CF5DB012406E0FF2274
:1067200021461420FBF7A8FC601CC4B2072CF6DB42
:1067300047A04EF67D730022072100905A20FBF7F8
:106740006AFD36488589042301AA28460021FBF703
:1067500092FE01A84EF67D73002204210090542081
:1067600000E040E0FBF757FD3BA04EF67D730022B2
:10677000042100906E20FBF74EFD042301AA374848
:1067800000880021FBF777FE01A84EF67D730022FA
:10679000022100905420FBF73EFD2FA04EF67D73A2
:1067A0000022022100906E20FBF735FD042301AA90
:1067B0002B4800880021FBF75EFE01A84EF67D7392
:1067C0000022012100905420FBF725FD22A04EF667
:1067D0007D730022012100906E20FBF71CFD02203A
:1067E0001649087040E0FCF73AFAFCF705FAFCF7A6
:1067F00018FA0A488589042301AA28460021FBF7D4
:106800003AFE01A84EF67D73002204210090542028
:1068100028E00000A00300202020000058040020F1
:10682000E4040020FE040020E4320108D42E010814
:10683000640100204C0100201C0100204B000020BE
:106840006B700000740000005E0000003E0000005D
:10685000D1B92020C1A600006B7061008E0000201D
:1068600092000020FBF7D7FC7FBD1FB5FB4A07CA8B
:1068700001AB07C34EF67D70F4F752F9F8484EF6B7
:106880007D730022072100907320FBF7C4FCF548BC
:10689000048D032301AA20460021FBF7ECFD01A88B
:1068A0004EF67D730022072100906120FBF7B3FCB8
:1068B000AFF2C4404EF67D730022072100904D20B8
:1068C000FBF7A9FCE8A04EF67D730022072100909B
:1068D0003720FBF7A0FCE648848C022301AA20465F
:1068E0000021FBF7C8FD01A84EF67D7300220721A9
:1068F00000901620FBF78FFCAFF20C504EF67D7324
:106900000022072100900620FBF785FCD9484EF6AF
:106910007D730022042100907320FBF77CFCD64895
:106920008489022301AA20460021FBF7A4FD01A8C7
:106930004EF67D730022042100906020FBF76BFC73
:10694000CC480C304EF67D73002204210090532079
:10695000FBF761FCC9A04EF67D7300220421009074
:106960003720FBF758FCC4484489022301AA20467B
:106970000021FBF780FD01A84EF67D730022042163
:1069800000901620FBF747FCAFF29C504EF67D734B
:106990000022042100900620FBF73DFCB048103097
:1069A0004EF67D730022012100907320FBF733FC2B
:1069B000B148C488022301AA20460021FBF75BFDF1
:1069C00001A84EF67D730022012100906020FBF7A4
:1069D00022FCAC484EF67D7300220121009053202A
:1069E000FBF719FCA34820304EF67D7300220121ED
:1069F00000902B20FBF70FFC9D48048D022301AA79
:106A000020460021FBF737FD01A84EF67D730022DA
:106A1000012100901620FBF7FEFB1FBD7FB58F4ABA
:106A200007CA01AB07C30024974800780B287CD124
:106A300096480078012879D14EF67D70F4F770F809
:106A40009348407C012805D15222FF210846F4F7E3
:106A5000CCF804E0522200210846F4F7C6F8844836
:106A600090F82D00042805D15122FF210846F4F7A3
:106A7000BCF804E0512200210846F4F7B6F8844837
:106A800090F82000012805D12222FF210846F4F7C2
:106A9000ACF804E0222200210846F4F7A6F8FCF73F
:106AA000DEF8FCF7A9F8FCF7BCF87AA04EF67D7387
:106AB0000022072100901020FBF7ADFB6C48808C72
:106AC0000A2190FBF1F084B2032301AA20460021A1
:106AD000FBF7D1FC01A84EF67D7300220721009040
:106AE0004F20FBF798FBAFF2F4604EF67D73002267
:106AF000072100906120FBF78EFB5D48808C0A2106
:106B000090FBF1F201FB120084B2012301AA20469E
:106B10000021FBF7B0FC01A84EF67D73002207218F
:106B200000906820FBF777FB01E0D4E188E0AFF24A
:106B300040704EF67D730022072100906E20FBF717
:106B40006AFB57A04EF67D730022052100901020AD
:106B5000FBF761FB4648C0880A2190FBF1F084B244
:106B6000022301AA20460021FBF785FC01A84EF66E
:106B70007D730022052100904F20FBF74CFBAFF204
:106B80008C704EF67D730022052100905B20FBF790
:106B900042FB3748C0880A2190FBF1F201FB12004A
:106BA00084B2012301AA20460021FBF764FC01A85E
:106BB0004EF67D730022052100906120FBF72BFB30
:106BC000AFF2D4704EF67D7300220521009067204D
:106BD000FBF721FB2E48807E012812D125482C305E
:106BE0004EF67D730022032100901020FBF713FB6B
:106BF0001F48458D032301AA28460021FBF73BFCD3
:106C000011E01C481C304EF67D73002203210090D9
:106C10001020FBF700FB1648058D032301AA284628
:106C20000021FBF728FC01A84EF67D73002203210A
:106C300000904F20FBF7EFFA0220144908704AE158
:106C40001A4800780028FAD11148407C01282FD139
:106C50005222FF210846F3F7C8FF2EE0A42E0108B8
:106C600040330108A8040020D2D1CAE4C8EB0000D8
:106C7000580400209C370108E4040020D7B7BCD397
:106C8000C1BF000048570108C00000204B00002091
:106C9000A0030020D2D1CAE4C8EBC1BF00000000AD
:106CA000D7D420BFD820C1BF00000000280000209A
:106CB000522200210846F3F798FFF74890F82D007C
:106CC000042805D15122FF210846F3F78EFF04E086
:106CD000512200210846F3F788FFF04890F8200081
:106CE000012805D12222FF210846F3F77EFF04E0A8
:106CF000222200210846F3F778FFFBF7B0FFFBF7ED
:106D00007BFFFBF78EFFE448808C0A2190FBF1F0BB
:106D100084B2032301AA20460021FBF7ACFB01A8A3
:106D20004EF67D730022072100904F20FBF773FA87
:106D3000AFF640104EF67D730022072100906120CF
:106D4000FBF769FAD448808C0A2190FBF1F201FB31
:106D5000120084B2012301AA20460021FBF78BFB1D
:106D600001A84EF67D730022072100906820FBF7F2
:106D700052FAC948C0880A2190FBF1F084B202237C
:106D800001AA20460021FBF776FB01A84EF67D7391
:106D90000022052100904F20FBF73DFAAFF6AC1022
:106DA0004EF67D730022052100905B20FBF733FA3D
:106DB000B948C0880A2190FBF1F201FB120084B2AD
:106DC000012301AA20460021FBF755FB01A84EF63E
:106DD0007D730022052100906120FBF71CFAAF486B
:106DE000807E012811D1AE484EF67D73002203212A
:106DF00000901020FBF70FFAA748458D032301AA46
:106E000028460021FBF737FB11E0A54810384EF665
:106E10007D730022032100901020FBF7FCF99E48AF
:106E2000058D032301AA28460021FBF724FB9B487C
:106E300090F82200012809D19A484EF67D7300226D
:106E4000032100904F20FBF7E6F911E0934890F8FA
:106E50002200062803D0914890F8220040B901A8EA
:106E60004EF67D730022032100904F20FBF7D3F9EB
:106E70008D48007C78BB042301AA8C48008800213F
:106E8000FBF7F9FA01A84EF67D730022012100906C
:106E90001020FBF7C0F9042301AA854800880021CF
:106EA000FBF7E9FA01A84EF67D730022012100905C
:106EB0003D20FBF7B0F9042301AA7E480088002199
:106EC000FBF7D9FA01A84EF67D730022012100904C
:106ED0006A20FBF7A0F97FBD7FB5724A303A07CA36
:106EE00001AB07C374480078012840D14EF67D708D
:106EF000F3F716FEFBF7B3FEFBF77EFEFBF791FE02
:106F00005C22FF210846F3F770FE6CA04EF67D73FD
:106F10000022062100902120FBF7DDF96AA04EF641
:106F20007D730022022100903520FBF7D4F9002464
:106F300017E00020654908550846055D012301AAB0
:106F400028460021FBF797FA01A83521009001EBB4
:106F5000C4004EF67D7300220321FBF7BCF9601CD0
:106F6000C4B2032CE5DB02205349087077E058488F
:106F70000078012804D002281ED0032854D137E01D
:106F800051A04EF67D730022022100903520FBF7C0
:106F9000A2F950A04EF67D730022022100903D2000
:106FA000FBF799F94BA04EF67D7300220221009069
:106FB0004520FBF790F938E046A04EF67D7300229D
:106FC000022100903520FBF786F93FA04EF67D7335
:106FD0000022022100903D20FBF77DF93DA04EF6F6
:106FE0007D730022022100904520FBF774F91CE01C
:106FF00038A04EF67D730022022100903520FBF769
:107000006AF934A04EF67D730022022100903D20E3
:10701000FBF761F92CA04EF67D730022022100904F
:107020004520FBF758F900E000BF00BF002414E042
:107030002648055D012301AA28460021FBF71BFA1B
:1070400001A83521009001EBC4004EF67D730022AB
:107050000321FBF740F9601CC4B2032CE8DB7FBDC1
:107060007FB5104A303A07CA01AB07C300244EF679
:107070007D70F3F755FDFBF7F2FDFBF7BDFDFBF768
:10708000D0FD064890F82000012825D12222FF21BA
:107090000846F3F7AAFD24E058040020A0030020CE
:1070A000C8370108D42E0108FE0400206401002026
:1070B0004C0100201C0100204B000020CBF8B6A89A
:1070C000C3DCC2EB000000005F00000045000020B0
:1070D000F200002020000000222200210846F3F7E1
:1070E00084FDFE488578022301AA28460021FBF78B
:1070F000C2F901A84EF67D730022072100900420FA
:10710000FBF789F8F6A04EF67D7300220721009068
:107110001020FBF780F8F148C578022301AA284621
:107120000021FBF7A8F901A84EF67D730022072184
:1071300000901C20FBF76FF8EAA04EF67D7300224A
:10714000072100902820FBF766F8E44845790223E0
:1071500001AA28460021FBF78EF901A84EF67D739F
:107160000022072100903420FBF755F8DEA04EF6F0
:107170007D730022072100904020FBF74CF8D74890
:107180008579022301AA28460021FBF774F901A89A
:107190004EF67D730022072100904620FBF73BF856
:1071A000D2A04EF67D730022052100900420FBF74B
:1071B00032F8AFF24C504EF67D730022032100905E
:1071C0001D20FBF728F8CC48808C0A2190FBF1F0B9
:1071D00084B2032301AA20460021FBF74CF901A841
:1071E0004EF67D730022032100904120FBF713F837
:1071F000AFF600604EF67D7300220321009053200D
:10720000FBF709F8BC48808C0A2190FBF1F201FBE6
:10721000120084B2012301AA20460021FBF72BF9BA
:1072200001A84EF67D730022032100905920FAF741
:10723000F2FFAFF644604EF67D730022032100900A
:107240006220FAF7E8FFAFF2CC504EF67D730022D1
:10725000012100900420FAF7DEFFA748C0880A2128
:1072600090FBF1F084B2022301AA20460021FBF733
:1072700002F901A84EF67D730022012100902E2014
:10728000FAF7C9FFAFF694604EF67D730022012134
:1072900000903A20FAF7BFFF9748C0880A2190FB78
:1072A000F1F201FB120084B2012301AA2046002161
:1072B000FBF7E1F801A84EF67D7300220121009052
:1072C0004020FAF7A8FFAFF6D8604EF67D73002293
:1072D000012100904820FAF79EFF88484EF67D7302
:1072E0000022012100905820FAF795FF8248058D71
:1072F000022301AA28460021FBF7BDF801A84EF69B
:107300007D730022012100907620FAF784FF7FBD73
:107310001FB57B4A07CA01AB07C34EF67D70F3F772
:10732000FFFBFBF79CFCFBF767FCFBF77AFC3D22BD
:1073300001210020F3F759FC68488478022301AA50
:1073400020460021FBF797F801A84EF67D73002236
:10735000062100900420FAF75EFF61A04EF67D73CF
:107360000022062100901020FAF755FF5B48C478F0
:10737000022301AA20460021FBF77DF801A84EF662
:107380007D730022062100901C20FAF744FF55A0CF
:107390004EF67D730022062100902820FAF73BFF6D
:1073A0004E484479022301AA20460021FBF763F8E6
:1073B00001A84EF67D730022062100903420FAF7D2
:1073C0002AFF49A04EF67D7300220621009040203E
:1073D000FAF721FF41488479022301AA20460021BF
:1073E000FBF749F801A84EF67D73002206210090B4
:1073F0004620FAF710FF43A04EF67D7300220321CA
:1074000000900420FAF707FF1FBD1FB53C4A07CACA
:1074100001AB07C34EF67D70F3F782FBFBF71FFC51
:10742000FBF7EAFBFBF7FDFB3D2201210020F3F710
:10743000DCFB2A488478022301AA20460021FBF7BE
:107440001AF801A84EF67D73002206210090042050
:10745000FAF7E1FE22A04EF67D730022062100908D
:107460001020FAF7D8FE1D48C478022301AA20464E
:107470000021FBF700F801A84EF67D7300220621DB
:1074800000901C20FAF7C7FE16A04EF67D7300226E
:10749000062100902820FAF7BEFE10484479022306
:1074A00001AA20460021FAF7E6FF01A84EF67D73F7
:1074B0000022062100903420FAF7ADFE0AA04EF615
:1074C0007D730022062100904020FAF7A4FE0348B5
:1074D0008479022301AA2046002119E02A00002015
:1074E000D4C20000C8D500003A000000CAE4D2BAF5
:1074F000BDE1CAF82121000058040020BC37010872
:10750000A42E0108BBFAD0B5B9CAD5CF21210000FD
:10751000FAF7B1FF01A84EF67D7300220621009014
:107520004620FAF778FEFEA04EF67D730022032176
:1075300000900420FAF76FFE1FBD1FB5FA4A07CA74
:1075400001AB07C34EF67D70F3F7EAFAFBF787FB52
:10755000FBF752FBFBF765FB3D2201210020F3F70F
:1075600044FBF2488478022301AA20460021FAF75E
:1075700082FF01A84EF67D730022062100900420B0
:10758000FAF749FEAFF2A8004EF67D7300220621FD
:1075900000901020FAF73FFEE448C478022301AAC5
:1075A00020460021FAF767FF01A84EF67D730022FE
:1075B000062100901C20FAF72EFEAFF2D8004EF6FE
:1075C0007D730022062100902820FAF724FED74878
:1075D0004479022301AA20460021FAF74CFF01A8B2
:1075E0004EF67D730022062100903420FAF713FE38
:1075F000AFF20C104EF67D73002206210090402061
:10760000FAF709FEC9488479022301AA204600211D
:10761000FAF731FF01A84EF67D7300220621009093
:107620004620FAF7F8FDC2A04EF67D730022032132
:1076300000900420FAF7EFFD1FBD1FB5BA4A07CA34
:1076400001AB07C34EF67D70F3F76AFAFBF707FB51
:10765000FBF7D2FAFBF7E5FA3D2201210020F3F710
:10766000C4FAB2488478022301AA20460021FAF71E
:1076700002FF01A84EF67D7300220621009004202F
:10768000FAF7C9FDAFF2A8104EF67D73002206216D
:1076900000901020FAF7BFFDA448C478022301AA85
:1076A00020460021FAF7E7FE01A84EF67D7300227E
:1076B000062100901C20FAF7AEFDAFF2D8104EF66E
:1076C0007D730022062100902820FAF7A4FD974838
:1076D0004479022301AA20460021FAF7CCFE01A832
:1076E0004EF67D730022062100903420FAF793FDB8
:1076F000AFF20C204EF67D73002206210090402050
:10770000FAF789FD89488479022301AA20460021DD
:10771000FAF7B1FE01A84EF67D7300220621009013
:107720004620FAF778FD84A04EF67D7300220321EF
:1077300000900420FAF76FFD1FBD1FB57A4A07CAF3
:1077400001AB07C34EF67D70F3F7EAF9FBF787FA52
:10775000FBF752FAFBF765FA3D2201210020F3F70F
:1077600044FA72488478022301AA20460021FAF7DD
:1077700082FE01A84EF67D730022062100900420AF
:10778000FAF749FDAFF2A8204EF67D7300220621DC
:1077900000901020FAF73FFD6448C478022301AA44
:1077A00020460021FAF767FE01A84EF67D730022FD
:1077B000062100901C20FAF72EFDAFF2D8204EF6DD
:1077C0007D730022062100902820FAF724FD5748F7
:1077D0004479022301AA20460021FAF74CFE01A8B1
:1077E0004EF67D730022062100903420FAF713FD37
:1077F000AFF20C304EF67D7300220621009040203F
:10780000FAF709FD49488479022301AA204600219C
:10781000FAF731FE01A84EF67D7300220621009092
:107820004620FAF7F8FC47A04EF67D7300220321AC
:1078300000900420FAF7EFFC1FBD1FB53A4A07CAB3
:1078400001AB07C34EF67D70F3F76AF9FBF707FA51
:10785000FBF7D2F9FBF7E5F93D2201210020F3F710
:10786000C4F932488478022301AA20460021FAF79D
:1078700002FE01A84EF67D7300220621009004202E
:10788000FAF7C9FCAFF2A8304EF67D73002206214C
:1078900000901020FAF7BFFC2448C478022301AA04
:1078A00020460021FAF7E7FD01A84EF67D7300227D
:1078B000062100901C20FAF7AEFCAFF2D8304EF64D
:1078C0007D730022062100902820FAF7A4FC1748B7
:1078D0004479022301AA20460021FAF7CCFD01A831
:1078E0004EF67D730022062100903420FAF793FCB7
:1078F000AFF20C404EF67D7300220621009040202E
:10790000FAF789FC09488479022301AA204600215C
:10791000FAF7B1FD01A84EF67D730022062117E0AB
:10792000B6C2C8FB21210000A42E01082A000020B5
:10793000BCABCFDE21210000C6F8C5DDCEDED2BA59
:1079400021210000CEB4D7B0D2A9BAD021210000A5
:1079500000904620FAF75FFCF7A04EF67D730022F8
:10796000032100900420FAF756FC1FBD08B54EF61F
:107970007D70F3F7D5F8FBF772F9FBF73DF9FBF7EC
:1079800050F93D2201210020F3F72FF9EDA04EF62A
:107990007D730022032100900420FAF73CFC08BD0F
:1079A0001FB5EB4A07CA01AB07C34EF67D70F3F76C
:1079B000B7F8FBF754F9FBF71FF9FBF732F93D2253
:1079C00001210020F3F711F9E2488478022301AA8B
:1079D00020460021FAF74FFD01A84EF67D730022E4
:1079E000062100900420FAF716FCAFF20C504EF678
:1079F0007D730022062100901020FAF70CFCD54878
:107A0000C478022301AA20460021FAF734FD01A818
:107A10004EF67D730022062100901C20FAF7FBFB36
:107A2000AFF240504EF67D730022062100902820D0
:107A3000FAF7F1FBC7484479022301AA2046002146
:107A4000FAF719FD01A84EF67D7300220621009079
:107A50003420FAF7E0FBAFF270504EF67D7300224F
:107A6000062100904020FAF7D6FBBA488479022319
:107A700001AA20460021FAF7FEFC01A84EF67D730C
:107A80000022062100904620FAF7C5FBB2A04EF670
:107A90007D730022032100901320FAF7BCFB1FBD69
:107AA0001FB5AB4A07CA01AB07C3AF48007801282E
:107AB0007ED14EF67D70F3F733F8FBF7D0F8FBF785
:107AC0009BF8FBF7AEF8A9A04EF67D7300220721C4
:107AD00000900420FAF79FFBA7480478012301AA2D
:107AE00020460021FAF7C7FC01A84EF67D7300225C
:107AF000072100904920FAF75BFBAFF634204EF6E1
:107B00007D730022062100904920FAF751FB9BA0CB
:107B10004EF67D730022072100905320FAF77BFB7D
:107B20009548C078012809D196A04EF67D730022B1
:107B3000072100907020FAF76EFB08E092A04EF645
:107B40007D730022072100907020FAF764FB8FA05C
:107B50004EF67D730022052100900420FAF75BFBAE
:107B600085484478012301AA20460021FAF783FCC6
:107B700001A84EF67D730022052100904920FAF7F6
:107B800017FB85A04EF67D7300220521009053203F
:107B9000FAF741FB7848407901280AD179A04EF6DE
:107BA0007D730022052100907020FAF734FB09E074
:107BB00061E075A04EF67D730022052100907020D3
:107BC000FAF729FB76A04EF67D7300220321009080
:107BD0000420FAF720FB6848C489032301AA204641
:107BE0000021FAF748FC01A84EF67D73002203211C
:107BF00000903D20FAF7DCFAAFF63C304EF67D738C
:107C00000022032100905320FAF705FB5A4880799F
:107C1000012809D15BA04EF67D730022032100905C
:107C20007020FAF7F8FA08E057A04EF67D730022AC
:107C3000032100907020FAF7EEFA5CA04EF67D73F7
:107C40000022012100900420FAF7E5FA4A488478DE
:107C5000022301AA20460021FAF70DFC01A84EF6E6
:107C60007D730022012100904320FAF7A1FA02203F
:107C70003D490870E4E1FAF7F2FFFAF7BDFFFAF7C1
:107C8000D0FF4D480078C01E0D2853D2DFE800F029
:107C900007ACF23A52FEF05252525252EF00AFF697
:107CA000D8304EF67D730022062100904920FAF765
:107CB0007FFA31480478012301AA20460021FAF70F
:107CC000DAFB01A84EF67D730022072100904920BF
:107CD000FAF76EFA2848C078012809D129A04EF693
:107CE0007D730022072100907020FAF794FA08E0D3
:107CF00025A04EF67D730022072100907020FAF730
:107D00008AFA9CE1AFF634404EF67D7300220621DC
:107D100000904920FAF74CFA1748C07801284FD153
:107D200026A04EF67D730022072100907020FAF7FE
:107D300072FA4EE082E10000B5E7C1BFBAC4BEA14D
:107D400021210000B9DCC2B7CDD1C2E4212100005D
:107D5000A42E01082A000020D7DCCAE4D7A2C1BFA4
:107D6000B1A8BEAF212100004B000020B2A1C7F88E
:107D7000CEBBCAFD00000000FE040020CDF8C2E723
:107D800000000000B9D80000BFAA0000B2A1B4B240
:107D9000CEBBCAFD00000000B2E9D1AF0000000078
:107DA000D7D4BFD8C1F7CBD900000000D7A1D4BA2F
:107DB000BAC5CEBBCAFD000049000020D1F20000C8
:107DC000F9A04EF67D730022072100907020FAF78B
:107DD00022FAAFF600504EF67D7300220421009087
:107DE0004920FAF7E5F92AE1F048C07801280AD1DC
:107DF000AFF270004EF67D730022072100907020D4
:107E0000FAF709FA09E0AFF280004EF67D7300221E
:107E1000072100907020FAF7FEF9AFF654504EF6A5
:107E20007D730022042100904920FAF7C1F9DF4850
:107E30004478012301AA20460021FAF71CFB01A87F
:107E40004EF67D730022052100904920FAF7B0F923
:107E5000D648407901280ED1AFF2D8004EF67D7396
:107E60000022052100907020FAF7D5F90DE039E0E5
:107E700085E00BE0AEE0AFF2F0004EF67D7300223D
:107E8000052100907020FAF7C6F9D8E0AFF6BC5093
:107E90004EF67D730022042100904920FAF788F9FC
:107EA000C248407901280AD1AFF2F0004EF67D7346
:107EB0000022052100907020FAF7ADF908E0BAA081
:107EC0004EF67D730022052100907020FAF7A3F989
:107ED000B7484EF67D730022022100903D20FAF74C
:107EE00067F9ACE0B148407901280AD1AFF26C10D3
:107EF0004EF67D730022052100907020FAF78BF971
:107F000009E0AFF27C104EF67D730022052100904F
:107F10007020FAF780F9A7484EF67D7300220221FF
:107F200000903D20FAF744F9A048C489032301AA30
:107F300020460021FAF79FFA01A84EF67D73002231
:107F4000032100903D20FAF733F998488079012801
:107F50000AD1AFF2D0104EF67D73002203210090BB
:107F60007020FAF758F909E0AFF2E4104EF67D738D
:107F70000022032100907020FAF74DF95FE08C4851
:107F80004EF67D730022022100903D20FAF710F991
:107F90008648807901280AD1AFF2E0104EF67D7351
:107FA0000022032100907020FAF735F908E07EA046
:107FB0004EF67D730022032100907020FAF72BF912
:107FC0007DA04EF67D730022114600904320FAF703
:107FD000EFF834E07548807901280AD1AFF25C20CF
:107FE0004EF67D730022032100907020FAF713F9FA
:107FF00009E0AFF26C204EF67D7300220321009061
:108000007020FAF708F96DA04EF67D730022114634
:1080100000904320FAF7CCF864488478022301AA40
:1080200020460021FAF727FA01A84EF67D730022B8
:10803000012100904320FAF7BBF800E000BF00BF29
:108040001FBD1FB55A4A303A07CA01AB07C35C4887
:10805000007801287DD14EF67D70F2F761FDFAF7C8
:10806000FEFDFAF7C9FDFAF7DCFD56A04EF67D736A
:108070000022072100900420FAF7CDF84B48C07A7F
:1080800001280AD1AFF2CC204EF67D7300220721E1
:1080900000903A20FAF7BFF808E043A04EF67D734F
:1080A0000022072100903A20FAF7B5F848A04EF6D2
:1080B0007D730022072100905020FAF7ACF83B486E
:1080C000C07950B9AFF244304EF67D7300220721DB
:1080D00000907020FAF79FF809E0AFF254304EF6A6
:1080E0007D730022072100907020FAF794F83A4837
:1080F0004EF67D730022052100900420FAF78BF8DC
:108100002A48807A01280AD1AFF288304EF67D7372
:108110000022052100903A20FAF77DF809E0AFF23D
:1081200098304EF67D730022052100903A20FAF730
:1081300072F82AA04EF67D7300220521009050208F
:10814000FAF769F81948007A01280CD1AFF2CC305F
:1081500000E0CCE04EF67D730022052100907020F7
:10816000FAF759F809E0AFF2E0304EF67D730022DD
:10817000052100907020FAF74EF80C48007B01288A
:1081800038D118A04EF67D73002203210090042000
:10819000FAF741F816A04EF67D73002203210090F5
:1081A0003A20FAF705F838E0B7E10000FE040020B5
:1081B000D42E010838530108202000005F5F000022
:1081C0004B000020BBFAD0B5B1A8BEAF0000000044
:1081D000C9F9D2F40000000004380108BFDBBACFAF
:1081E00000000000D7DCCAE4D7A2C1BF0000000035
:1081F00031353000AFF214004EF67D7300220321BA
:1082000000900420FAF707F8FCA04EF67D730022D8
:10821000032100903A20F9F7CBFFF9484EF67D7321
:108220000022032100905020F9F7F5FFF548407A2D
:1082300001280AD1AFF2B4404EF67D73002203212B
:1082400000907020F9F7E7FF09E0AFF2C4404EF666
:108250007D730022032100907020F9F7DCFFEAA073
:108260004EF67D730022012100900420F9F7D3FF20
:10827000E448007C01280AD1AFF2F8404EF67D7345
:108280000022012100903A20F9F7C5FF09E0AFF282
:1082900008504EF67D730022012100903A20F9F734
:1082A000BAFFDCA04EF67D73002201210090502021
:1082B000F9F7B1FFD348407C01280AD1AFF23C5016
:1082C0004EF67D730022012100907020F9F7A3FF84
:1082D00009E0AFF24C504EF67D7300220121009070
:1082E0007020F9F798FF0220CC490870C3E2FAF732
:1082F000B6FCFAF781FCFAF794FCC94800780A3812
:10830000092878D2DFE800F037CEF9830577F8F74F
:10831000F600BC48C07A01280AD1AFF260504EF690
:108320007D730022072100903A20F9F774FF09E0DD
:10833000AFF28C104EF67D730022072100903A2098
:10834000F9F769FFAF48C07950B9AFF2C8504EF69F
:108350007D730022072100907020F9F75CFF09E08F
:10836000AFF2DC504EF67D730022072100907020A2
:10837000F9F751FF7EE2A348C07A01280AD1AFF293
:10838000FC504EF67D730022072100903A20F9F749
:1083900042FF09E0AFF210604EF67D730022072124
:1083A00000903A20F9F737FF9648C07950B9AFF2FC
:1083B000F4504EF67D730022072100907020F9F7EB
:1083C0002AFF09E0AFF220204EF67D73002207213C
:1083D00000907020F9F71FFF8A48807A01280BD19E
:1083E000AFF260604EF67D730022052100903A20C6
:1083F000F9F711FF0AE03CE2AFF274604EF67D73CC
:108400000022052100903A20F9F705FF32E27D486D
:10841000C07950B9AFF294604EF67D730022072107
:1084200000907020F9F7F7FE09E0AFF2A4604EF675
:108430007D730022072100907020F9F7ECFE71484F
:10844000807A01280AD1AFF28C604EF67D7300224B
:10845000052100903A20F9F7DEFE09E0AFF2B820DE
:108460004EF67D730022052100903A20F9F7D3FEE5
:108470006448007A01280AD1AFF2F8604EF67D73A5
:108480000022052100907020F9F7C5FE09E0AFF247
:1084900008704EF67D730022052100907020F9F7D8
:1084A000BAFEE7E15748807A01280AD1AFF22C7072
:1084B0004EF67D730022052100903A20F9F7ABFEBD
:1084C00009E0AFF23C704EF67D730022052100906A
:1084D0003A20F9F7A0FE4B48007A01280ED1AFF2FE
:1084E00024704EF67D730022052100907020F9F76C
:1084F00092FE0DE08AE13DE140E0D3E0AFF258307A
:108500004EF67D730022052100907020F9F783FE5E
:108510003C48007B012818D142484EF67D7300226A
:10852000022100903A20F9F743FE032301AA962086
:108530000021F9F7A0FF01A84EF67D730022032168
:1085400000903A20F9F734FE17E036484EF67D7376
:108550000022022100903A20F9F72AFE032301AA03
:1085600001200021F9F787FF01A84EF67D73002254
:10857000032100903A20F9F71BFE7BE12148007AA5
:1085800001280AD1AFF604004EF67D7300220521C2
:1085900000907020F9F73FFE09E0AFF614004EF6A8
:1085A0007D730022052100907020F9F734FE1548F4
:1085B000007B01283AD1AFF2D4304EF67D73002211
:1085C000032100900420F9F726FE17484EF67D732C
:1085D0000022022100903A20F9F7EAFD032301AAC4
:1085E00096200021F9F747FF01A84EF67D7300227F
:1085F000032100903A20F9F7DBFD39E030303100FB
:10860000F4370108FE040020D1B9C1A6CFD4CABEF8
:1086100000000000B2E2CAD4000000004B000020BD
:1086200049000020D42E010838530108AFF24C4015
:108630004EF67D730022032100900420F9F7EBFD34
:10864000FE484EF67D730022022100903A20F9F791
:10865000AFFD032301AA01200021F9F70CFF01A8B7
:108660004EF67D730022032100903A20F9F7A0FD19
:10867000F348407A01280AD1AFF6F8004EF67D7330
:108680000022032100907020F9F7C5FD09E0AFF644
:1086900008104EF67D730022032100907020F9F738
:1086A000BAFDE7E0E648007B012818D1E5484EF620
:1086B0007D730022022100903A20F9F779FD03230F
:1086C00001AA96200021F9F7D6FE01A84EF67D7387
:1086D0000022032100903A20F9F76AFD17E0D948FB
:1086E0004EF67D730022022100903A20F9F760FDDA
:1086F000032301AA01200021F9F7BDFE01A84EF6CF
:108700007D730022032100903A20F9F751FDCC48F7
:10871000407A01280AD1AFF65C104EF67D73002234
:10872000032100907020F9F776FD09E0AFF2885040
:108730004EF67D730022032100907020F9F76BFD47
:10874000BF48007C01280AD1AFF6C8104EF67D73F1
:108750000022012100903A20F9F75DFD09E0AFF613
:10876000D8104EF67D730022012100903A20F9F7CF
:1087700052FD7FE0B248407A01280AD1AFF6FC10E2
:108780004EF67D730022032100907020F9F743FD1F
:1087900009E0AFF60C204EF67D7300220321009015
:1087A0007020F9F738FDA648007C01280AD1AFF601
:1087B000F4104EF67D730022012100903A20F9F763
:1087C0002AFD09E0AFF220604EF67D730022012100
:1087D00000903A20F9F71FFD9948407C01280AD102
:1087E000AFF660204EF67D730022012100907020CC
:1087F000F9F711FD09E0AFF670204EF67D73002207
:10880000012100907020F9F706FD33E08C48007CD0
:1088100001280AD1AFF694204EF67D730022012183
:1088200000903A20F9F7F7FC09E0AFF6A4204EF6E5
:108830007D730022012100903A20F9F7ECFC80487A
:10884000407C01280AD1AFF68C204EF67D730022C1
:10885000012100907020F9F7DEFC09E0AFF2B8606A
:108860004EF67D730022012100907020F9F7D3FCB1
:1088700000BF00BF00BF1FBD1FB5724A303A07CA14
:1088800001AB07C37048007801287DD14EF67D709A
:10889000F2F746F9FAF7E3F9FAF7AEF96B4804880C
:1088A000042301AA20460021F9F7E5FD01A84EF6B0
:1088B0007D730022072100900420F9F7ACFC64A02E
:1088C0004EF67D730022072100901C20F9F7A3FCCF
:1088D0005E488478022301AA20460021F9F7CBFDE7
:1088E00001A84EF67D730022072100902220F9F79F
:1088F00092FC57A04EF67D730022072100902E2097
:10890000F9F789FC5148C478022301AA20460021C6
:10891000F9F7B1FD01A84EF67D7300220721009002
:108920003420F9F778FC4BA04EF67D730022072126
:1089300000904020F9F76FFC44484479022301AAD3
:1089400020460021F9F797FD01A84EF67D7300221D
:10895000072100904620F9F75EFC3FA04EF67D739C
:108960000022072100905220F9F755FC37488479FE
:10897000022301AA20460021F9F77DFD01A84EF649
:108980007D730022072100E0A8E000905820F9F74D
:1089900042FC30A04EF67D73002207210090642037
:1089A000F9F739FC2948C479022301AA204600219D
:1089B000F9F761FD01A84EF67D73002207210090B2
:1089C0006A20F9F728FC25A04EF67D7300220521C8
:1089D00000900420F9F7ECFB042301AA2148008849
:1089E0000021F9F748FD01A84EF67D73002205210C
:1089F00000902220F9F7DCFB1BA04EF67D730022CD
:108A0000052100903A20F9F7D3FB1848848A032304
:108A100001AA20460021F9F72EFD01A84EF67D732C
:108A20000022052100904020F9F7C2FB10A04EF66D
:108A30007D7300220421009008461FE0385301088E
:108A4000FE040020D42E01084B0000202A00002044
:108A50002F000000200000003A000000566F6C74E8
:108A60003A000000BA0000202D0000005804002049
:108A70005072657373757265313A0000F9F798FBAF
:108A8000FE488489042301AA20460021F9F7F3FC5B
:108A900001A84EF67D730022042100904020F9F7D2
:108AA00087FBF748007910B9F548807848B1F5A000
:108AB0004EF67D730022022100900420F9F778FB26
:108AC00008E0F4A04EF67D730022022100900420FD
:108AD000F9F76EFB0220F3490870D2E0FAF7BFF80D
:108AE000FAF78AF8F0480488042301AA20460021F6
:108AF000F9F7C1FC01A84EF67D7300220721009012
:108B00000420F9F788FBE8488478022301AA20466C
:108B10000021F9F7B0FC01A84EF67D730022072171
:108B200000902220F9F777FBDF48C478022301AADE
:108B300020460021F9F79FFC01A84EF67D73002224
:108B4000072100903420F9F766FBD74844790223C7
:108B500001AA20460021F9F78EFC01A84EF67D738C
:108B60000022072100904620F9F755FBCE48847972
:108B7000022301AA20460021F9F77DFC01A84EF648
:108B80007D730022072100905820F9F744FBC64866
:108B9000C479022301AA20460021F9F76CFC01A840
:108BA0004EF67D730022072100906A20F9F733FB0F
:108BB000042301AABD4800880021F9F75CFC01A844
:108BC0004EF67D730022052100902220F9F7F0FA7D
:108BD000AA48848A032301AA20460021F9F74BFC06
:108BE00001A84EF67D730022052100904020F9F780
:108BF000DFFAA34890F82A0078B9042301AA0020DC
:108C00000146F9F738FC01A84EF67D7300220421D5
:108C100000904020F9F7CCFA1AE0984884890423A0
:108C200001AA20460021F9F726FC01A84EF67D7323
:108C30000022042100904020F9F7BAFA9C480078FD
:108C4000032805DB00209A4908708D4981F82A0025
:108C50008B48007910B98A48807848B189A04EF6CF
:108C60007D730022022100900420F9F7A1FA08E0A8
:108C700088A04EF67D730022022100900420F9F7AF
:108C800097FA1FBD1FB58B4A07CA01AB07C38548BA
:108C9000007801287ED14EF67D70F1F741FFF9F79B
:108CA000DEFFF9F7A9FFF9F7BCFF83A04EF67D734D
:108CB0000022072100902920F9F7ADFA81480078B9
:108CC000012809D1AFF60C304EF67D730022042145
:108CD00000903720F9F76CFA7BA04EF67D730022E6
:108CE000052100900420F9F796FA7A4804780223C7
:108CF00001AA20460021F9F7BEFB01A84EF67D73BC
:108D00000022052100903720F9F752FA6D480078CB
:108D1000022809D1AFF65C304EF67D7300220421A3
:108D200000907620F9F744FA6BA04EF67D7300228E
:108D3000052100904420F9F76EFA66484478022332
:108D400001AA20460021F9F796FB01A84EF67D7393
:108D50000022052100907620F9F72AFA5948007878
:108D6000032809D1AFF6AC304EF67D730022022104
:108D700000903720F9F71CFA5AA04EF67D730022B6
:108D8000032100900420F9F746FA52488478022320
:108D900001AA00E052E020460021F9F76CFB01A88F
:108DA0004EF67D730022032100903720F9F700FA78
:108DB0004FA04EF67D730022032100904420F9F766
:108DC0002AFA40480078042808D14C484EF67D73B2
:108DD0000022032100907620F9F7B7F948A04EF65B
:108DE0007D730022012100900420F9F714FA354820
:108DF0000078052808D141484EF67D7300220121F4
:108E000000903520F9F7A1F940A04EF67D730022BD
:108E1000012100904420F9F7FEF92A48007806283D
:108E200008D136484EF67D7300220121009076204D
:108E3000F9F78BF902201B490870F3E1F9F70FFFEE
:108E4000F9F7DAFEF9F7EDFE1E48007807287DD223
:108E5000DFE800F07C04A0EFEDECEB00AFF6A440FF
:108E60004EF67D730022042100903720F9F7A0F917
:108E7000AFF6BC404EF67D7300224DE05804002052
:108E8000A00300207A6967626565206F70656E20B7
:108E9000000000007A696762656520636C6F736526
:108EA000000000004B0000202A000020BA00002033
:108EB00051000020A42E0108CAE4D7A2C6C0BCDB22
:108EC0000000000048000020F0FE20202020D1F704
:108ED00000000000F2040020D5F2BEB2C6C0B7D632
:108EE00000000000B6F1D0C4C5BBCDC20000000038
:108EF000CBC4D6ABBCA1C1A600000000AC4A01089F
:108F0000CCDBCDB4C6C0BCDB00000000C8B7C8CF06
:108F1000C6C0BCDB00000000042100907620F9F7F9
:108F200047F9AFF66C504EF67D7300220221009097
:108F30003720F9F73DF9F9484EF67D7300220321F9
:108F400000907620F9F701F9F44800E068E14EF668
:108F50007D730022012100903520F9F7F6F8EF48E3
:108F60004EF67D730022012100907620F9F7EDF88E
:108F7000EB480478022301AA20460021F9F77BFA86
:108F800001A84EF67D730022052100903720F9F7E5
:108F90000FF946E1AFF6E0504EF67D730022042152
:108FA00000903720F9F704F9AFF6F0504EF67D73D4
:108FB0000022042100907620F9F7FAF8AFF6086055
:108FC0004EF67D730022022100903720F9F7F0F869
:108FD000D2484EF67D730022032100907620F9F7E7
:108FE000B4F8CE484EF67D73002201210090352062
:108FF000F9F7ABF8C9484EF67D73002201210090C5
:109000007620F9F7A2F8C6484478022301AA204640
:109010000021F9F730FA01A84EF67D7300220521F0
:1090200000907620F9F7C4F8FBE0C1E086E04BE061
:10903000FFE7AFF67C604EF67D73002204210090BE
:109040003720F9F7B5F8AFF690604EF67D73002241
:10905000042100907620F9F7ABF8AFF6A0604EF649
:109060007D730022022100903720F9F7A1F8AB4868
:109070004EF67D730022032100907620F9F765F803
:10908000A6484EF67D730022012100903520F9F7A5
:109090005CF8A2484EF67D730022012100907620F4
:1090A000F9F753F89E488478022301AA204600214C
:1090B000F9F7E1F901A84EF67D7300220321009033
:1090C0003720F9F775F8ACE0AFF614704EF67D7303
:1090D0000022042100903720F9F76AF8AFF62870D3
:1090E0004EF67D730022042100907620F9F760F897
:1090F000AFF63C704EF67D730022022100903720BF
:10910000F9F756F887484EF67D7300220321009048
:109110007620F9F71AF881484EF67D730022012176
:1091200000903520F9F711F87C484EF67D73002247
:10913000012100907620F9F708F872E0AFF6887008
:109140004EF67D730022042100903720F9F730F8A5
:10915000AFF69C704EF67D730022042100907620BD
:10916000F9F726F8AFF6B0704EF67D7300220221B3
:1091700000903720F9F71CF868484EF67D730022FE
:10918000032100907620F8F7E0FF66484EF67D73E5
:109190000022012100903520F8F7D7FF5F484EF6F6
:1091A0007D730022012100907620F8F7CEFF38E091
:1091B000AFF6FC704EF67D7300220421009037203C
:1091C000F8F7F6FF58A04EF67D73002204210090B8
:1091D0007620F8F7EDFF54A04EF67D7300220221B1
:1091E00000903720F8F7E4FF4C484EF67D730022DC
:1091F000032100907620F8F7A8FF48484EF67D73CB
:109200000022012100903520F8F79FFF45484EF6D7
:109210007D730022012100907620F8F796FF00E090
:1092200000BF00BF1FBD1FB53C4A303A07CA01ABA3
:1092300007C33E48007801286ED14EF67D70F1F7E5
:109240006FFCF9F70CFDF9F7D7FCF9F7EAFCAFF280
:1092500098304EF67D730022072100902920F8F700
:10926000DAFF33A04EF67D730022042100900846F9
:10927000F8F7D1FF2A48C479022301AA2046002129
:10928000F9F7F9F801A84EF67D7300220421009049
:109290002220F8F78DFF28A04EF67D7300220321CF
:1092A00000902220F8F784FF24A04EF67D73002260
:1092B000042100904420F8F7AEFF1948047A0223F5
:1092C00001AA20460021F9F7D6F801A84EF67D73D1
:1092D0000022042100906220F8F76AFF19A04EF6E0
:1092E0007D730022022100900420F8F794FF0C48BF
:1092F000447A022301AA20460021F9F7BCF801A80C
:109300004EF67D730022022100904020F8F750FFB6
:1093100002200649087052E118E00000D42E01082E
:10932000F2040020AC4A0108202000004B0000207D
:10933000BEB2D6B9000000005F5F0000BBEEB6AF62
:1093400000000000C2FAD2E2B6C80000F9F787FCBC
:10935000F9F752FCF9F765FCFE4800780B2804D0B9
:109360000C285BD00D287DD1B3E0FB48C4790223E3
:1093700001AA20460021F9F77EF801A84EF67D7378
:109380000022042100902220F8F712FFAFF25800CB
:109390004EF67D730022032100902220F8F708FF8B
:1093A000AFF27C004EF67D73002203210090622014
:1093B000F8F7FEFEAFF290004EF67D730022012119
:1093C00000904020F8F7F4FEE348C079012809D165
:1093D000E2A04EF67D730022042100903120F8F7C0
:1093E0001AFF1AE0DC48C079022809D1DCA04EF649
:1093F0007D730022042100903120F8F70CFF0CE06F
:10940000D548C079032808D1D6A04EF67D73002236
:10941000042100903120F8F7FEFECFE0CE48047A18
:10942000022301AA20460021F9F725F801A84EF6EB
:109430007D730022042100906220F8F7B9FEAFF29C
:1094400018104EF67D730022032100902220F8F7B9
:10945000AFFEAFF21C104EF67D7300220321009088
:10946000622000E0A9E0F8F7A3FEAFF244104EF648
:109470007D730022012100904020F8F799FEB64844
:10948000007A012809D1B5A04EF67D73002204218F
:1094900000907120F8F7BFFE1AE0AF48007A02286A
:1094A00009D1AFA04EF67D730022042100907120F7
:1094B000F8F7B1FE0CE0A848007A032808D1A9A06B
:1094C0004EF67D730022042100907120F8F7A3FE70
:1094D00074E0A148447A022301AA20460021F8F74B
:1094E000CAFF01A84EF67D730022022100904020A1
:1094F000F8F75EFEAFF2D0104EF67D730022032126
:1095000000902220F8F754FEAFF2E4104EF67D737F
:109510000022032100906220F8F74AFEAFF2E81023
:109520004EF67D730022012100904020F8F740FEA6
:109530008948407A012812D18BA04EF67D73002213
:10954000022100905920F8F766FE89A04EF67D733F
:109550000022022100905920F8F75DFE2CE07E48A1
:10956000407A022812D180A04EF67D73002202219B
:1095700000905920F8F74FFE7FA04EF67D73002231
:10958000022100905920F8F746FE15E07248407A13
:10959000032811D174A04EF67D73002202210090A1
:1095A0005920F8F738FE76A04EF67D73002202218E
:1095B00000905920F8F72FFE00E000BF00BF1FBD4C
:1095C0001FB5714A07CA01AB07C37048007801286C
:1095D0007ED14EF67D70F1F7A3FAF9F740FBF9F76B
:1095E0000BFBF9F71EFBAFF2F8604EF67D7300221D
:1095F000072100902920F8F70EFE65A04EF67D7336
:109600000022052100900420F8F705FE5248C47896
:10961000022301AA20460021F8F72DFFAFF2E8202F
:109620004EF67D730022042100902E20F8F7C0FD35
:1096300001A84EF67D730022052100902E20F8F738
:10964000B7FD55A04EF67D73002205210090442001
:10965000F8F7E1FD40484479022301AA20460021A1
:10966000F8F709FF01A84EF67D730022052100904E
:109670006E20F8F79DFD4AA04EF67D730022022170
:1096800000900420F8F7C7FD33480479022301AAAB
:1096900020460021F8F7EFFE01A84EF67D73002268
:1096A000022100902E20F8F783FD3FA04EF67D7337
:1096B0000022022100904420F8F7ADFD264884796D
:1096C000022301AA20460021F8F7D5FE01A800E0F8
:1096D0000BE04EF67D730022022100906E20F8F719
:1096E00067FD0220294908702CE1F9F7B8FAF9F76B
:1096F00083FAF9F796FA17480078072806D0082861
:109700007DD009286BD00A287AD1DFE01248C478CE
:10971000022301AA20460021F8F7ADFE01A84EF66B
:109720007D730022052100902E20F8F741FDAFF255
:10973000F8304EF67D730022042100902E20F8F7B9
:1097400037FD0AA04EF67D730022042100906E20A2
:109750002EE0000048000020F2040020C7E10000D5
:10976000D6D00000D6D800002020202020200000E5
:10977000B2BBC2FAD2E20000D2BB2020B0E30000AC
:10978000C2FA2020D2E20000A42E01084B000020E3
:10979000D7F3C9CFD6AB0000D7F3CFC2D6AB00000A
:1097A000D3D2C9CFD6AB0000D3D2CFC2D6AB000044
:1097B000F8F7FEFCAFF24C004EF67D73002201215B
:1097C00000902E20F8F7F4FCAFF260004EF67D73A7
:1097D0000022012100906E20F8F7EAFCB1E0FA487F
:1097E0004479022301AA20460021F8F744FE01A88B
:1097F0004EF67D730022052100906E2001E02BE0E3
:109800009EE0F8F7D5FCAFF29C004EF67D73002287
:10981000042100902E20F8F7CBFCAFF2E4404EF686
:109820007D730022042100906E20F8F7C1FCAFF296
:10983000C4004EF67D730022012100902E20F8F71F
:10984000B7FCAFF2D8004EF67D73002201210090E4
:109850006E20F8F7ADFC74E0DB480479022301AA1E
:1098600020460021F8F707FE01A84EF67D7300227E
:10987000022100902E20F8F79BFCAFF210104EF65C
:109880007D730022042100902E20F8F791FCAFF2A6
:1098900024104EF67D730022042100906E20F8F70C
:1098A00087FCAFF26C504EF67D73002201210090D0
:1098B0002E20F8F77DFCAFF24C104EF67D7300229F
:1098C000012100906E20F8F773FC3AE0BE488479DD
:1098D000022301AA20460021F8F7CDFD01A84EF68B
:1098E0007D730022022100906E20F8F761FCAFF238
:1098F00084104EF67D730022042100902E20F8F78C
:1099000057FCAFF298104EF67D73002204210090B0
:109910006E20F8F74DFCAFF2AC104EF67D730022CE
:10992000012100902E20F8F743FCAFF2F4504EF6E0
:109930007D730022012100906E20F8F739FC00E0D1
:1099400000BF00BF1FBD1FB5A04A07CA01AB07C3B8
:109950009F48007801286FD14EF67D70F1F7E0F84E
:10996000F9F77DF9F9F748F9F9F75BF999A04EF69F
:109970007D730022072100902920F8F74CFC98A065
:109980004EF67D730022052100900A20F8F743FC73
:109990008D48847A022301AA20460021F8F76BFD46
:1099A00001A84EF67D730022052100903420F8F7BF
:1099B00032FC8D4800780E2808D18C484EF67D7315
:1099C0000022052100907020F8F725FC88A04EF6B3
:1099D0007D730022032100900A20F8F71CFC8248C6
:1099E00000780F2808D181484EF67D7300220321AC
:1099F00000907020F8F70FFC7B480078102809D100
:109A00007FA04EF67D730022012100900A20F8F716
:109A100002FC0CE074480078112808D17BA04EF6B7
:109A20007D730022012100900A20F8F7F4FB022048
:109A30006749087086E0FFE7F9F711F9F9F7DCF8F4
:109A4000F9F7EFF8684800780E38052878D2DFE893
:109A500000F003283C4659005B48847A022301AA9F
:109A600020460021F8F707FD01A84EF67D7300227D
:109A7000052100903420F8F7CEFB5C484EF67D734C
:109A80000022052100907020F8F7C5FB4F483030C8
:109A90004EF67D730022032100907020F8F7BBFB87
:109AA0004FE04A4830304EF67D7300220521009089
:109AB0007020F8F7B0FB4D484EF67D73002203216D
:109AC00000907020F8F7A7FB3BE04DA04EF67D73A9
:109AD0000022012100900A20F8F79DFB31E04EA002
:109AE0004EF67D730022012100900A20F8F793FBC7
:109AF00046A04EF67D730022012100900A20F8F75F
:109B00008AFB1EE0AFF29C304EF67D73002282216C
:109B100000906E20F8F73FFC34484EF67D7300222B
:109B2000A5210090AA20F8F736FC3EA04EF67D73E2
:109B30000022D22100900A20F8F72DFC01E0FFE777
:109B400000BF00BF1FBD08B54EF67D70F0F7E8FFFF
:109B5000F9F785F8F9F750F8F9F763F800203C2396
:109B60004FF4A07219460090F8F792FA35A04EF61D
:109B70007D730022462100905F20F8F70CFC18A0AE
:109B80004EF67D7300226E2100900A20F8F703FC48
:109B90002FA04EF67D730022732100906E20F8F7FF
:109BA000FAFB13A04EF67D730022A02100900A203C
:109BB000F8F7F1FB12A04EF67D730022D22100903F
:109BC0000A20F8F7E8FB08BDF2040020A42E0108E3
:109BD0004B000020CDD5C8CBBFC6BCBC00000000E8
:109BE000C6C0BCDBC8CB000048000020AC4A01085E
:109BF000C9CFB4ABC8B7C8CFC6C0BCDB000000003B
